:1000000000800020BD010000DDCA000095CA00008C
:1000100095CA000095CA000095CA000095CA000064
:1000200095CA000095CA000095CA0000DDCA00000C
:10003000DDCA000095CA00005DC1000061C2000079
:10004000DDCA0000DDCA0000DDCA0000DDCA000014
:10005000DDCA0000DDCA0000DDCA0000DDCA000004
:10006000DDCA0000DDCA0000DDCA0000DDCA0000F4
:10007000DDCA0000DDCA0000DDCA0000DDCA0000E4
:10008000DDCA0000DDCA0000DDCA0000DDCA0000D4
:10009000DDCA0000DDCA0000DDCA0000DDCA0000C4
:1000A00099A60000A5A60000DDCA0000DDCA000078
:1000B000DDCA0000DDCA0000DDCA0000DDCA0000A4
:1000C000DDCA0000DDCA0000DDCA0000DDCA000094
:1000D000DDCA0000DDCA0000DDCA0000DDCA000084
:1000E000DDCA0000DDCA0000DDCA0000DDCA000074
:1000F000DDCA000049EB0000DDCA000075EC00001D
:10010000DDCA0000B5D40000DDCA0000DDCA000071
:10011000DDCA0000DDCA0000DDCA0000DDCA000043
:10012000DDCA0000DDCA0000DDCA0000DDCA000033
:10013000DDCA0000DDCA0000DDCA0000DDCA000023
:10014000DDCA0000DDCA0000DDCA0000DDCA000013
:100150004DC3000061C3000075C3000089C30000E7
:10016000DDCA0000D1D70000DDCA0000DDCA0000F2
:10017000DDCA0000DDCA0000DDCA0000DDCA0000E3
:10018000DDCA0000DDCA0000DDCA0000DDCA0000D3
:10019000DDCA0000DDCA0000DDCA0000DDCA0000C3
:1001A000DDCA0000DDCA0000DDCA0000DDCA0000B3
:1001B000DDCA0000DDCA0000DDCA0000564B4CF26B
:1001C000205210B51A804DF628121A8000BF00BFC9
:1001D0000CF088FC514B4FF010621A60504A9A6044
:1001E000504ADA60504A136813F4807304D14F49BF
:1001F0000B604FF4A85313604D4B1A78110703D5C9
:100200001A7842F008021A704A4B4B492A221A7097
:100210004A4A4B4B8B4204D252F8040F43F8040B6A
:10022000F8E7484B484900228B4202D243F8042B9E
:10023000FAE74649464A002352F8230041F82300D2
:1002400001336F2BF8D1434B434A802103F8011B44
:100250009342FBD1414B3D4A1A60414B8A221A70AE
:10026000A3F5805324225A70A0221A709A7992071B
:10027000FCD59A79D406FCD43A4A937903F00C035E
:10028000082B384BF9D103221A7140225A719A79FE
:100290009006FCD5334A9179324B4906FBD5324A58
:1002A000324911600221516020221A709A7902F0BD
:1002B0000C020C2AFAD12E4B2E4A1A602E4B2F4AD2
:1002C0001A6000225A60072243F8042C2C4AC3F813
:1002D0000C2D62B60CF0B6FF144B1B68DA0705D57F
:1002E00028480CF083FD284B284A1A60284B1B78BD
:1002F0005B0609D5244C254B22689A4204D121483B
:100300000CF074FD002323600FF06EFF0CF0F0FB87
:100310000CF01EFBFEE700BF0E20054030800440BD
:10032000823F04000100002B10D0034014D0034092
:1003300002D0074000E007405C9BFF1F5C3A0100D1
:100340004088FF1F5C9BFF1F4CA3FF1F0082FF1F05
:100350000000000000E400E05FE400E008ED00E0E1
:100360000050064000400640448004400000030165
:1003700004800440C010050014E000E0FF76010096
:100380000000202078D83C5F1CE00340A5C3945AAD
:1003900000F00740FFFFFFFFFFFFFFFFFFFFFFFF32
:1003A000FFFFFFFFFFFFFFFFFFFFFFFFFFFFFFFF5D
:1003B000FFFFFFFFFFFFFFFFFFFFFFFFFFFFFFFF4D
:1003C000FFFFFFFFFFFFFFFFFFFFFFFFFFFFFFFF3D
:1003D000FFFFFFFFFFFFFFFFFFFFFFFFFFFFFFFF2D
:1003E000FFFFFFFFFFFFFFFFFFFFFFFFFFFFFFFF1D
:1003F000FFFFFFFFFFFFFFFFFFFFFFFFFFFFFFFF0D
:10040000FFFFFFFFFFFFFFFFFFFFFFFFDEF9FFFF23
:1004100010B5054C237833B9044B13B10448AFF33E
:1004200000800123237010BD5C9BFF1F00000000B3
:10043000603A0100084B10B51BB108490848AFF3FA
:1004400000800848036803B910BD074B002BFBD0A0
:10045000BDE81040184700BF00000000609BFF1F70
:10046000603A01005C9BFF1F0000000038B50446A5
:10047000104621700A491D460FF098FC01464FF0C6
:100480007E500FF047FD07490FF090FCE56060607B
:10049000256165610CF066FEE061204638BD00BF55
:1004A000DB0FC9400024744938B50446104621705A
:1004B00009491D460FF07AFC01464FF07E500FF0BF
:1004C00029FD06490FF072FCE560606025616561F9
:1004D0000CF048FEE06138BDDB0FC94000247449D0
:1004E00038B503780446032B20D8DFE803F01A1848
:1004F0001002C16840690FF04FFB0D490546606866
:100500000FF008FD014628460FF004FD38BD0849EC
:1005100040680FF0FFFCE1680FF048FC38BDC06890
:1005200038BDC16840690FF037FB38BD002038BDC9
:100530000024744970B504460E460CF013FE0546BF
:10054000E069281A0FF0DEFBE3682361E56166616C
:10055000A061014660680FF0DDFC0146A060104814
:100560000FF0D8FC0EF0AEFF0EF04EFC0FF0C0FA0C
:10057000054601464FF07E500FF00EFB61690FF00B
:1005800015FC2169064628460FF010FC014630464E
:100590000FF004FBE0602046BDE87040FFF7A0BF0D
:1005A000000080BF08B50E200CF0ACF8114B1B8882
:1005B000012B19D0104B1B88984213DB40F6FF71BA
:1005C0008842D4BFC3EB0001C3EB0101C1EB013191
:1005D000C3F57F630F33282091FBF3F1BDE808409A
:1005E0000CF016BC0021F3E70146BDE808401420DA
:1005F0000CF00EBC909DFF1F289CFF1F10B50446F9
:100600000BF082FE204610BD70B44C88A04220D969
:1006100001230133DBB21CB2660031F8144084427E
:100620001D46F6D3A04211D005F10045013D965B71
:1006300031F8151032F81530401AF21A00FB02F0AA
:10064000641A90FBF4F4E01870BC7047905B70BCC7
:10065000704702260125E5E700280CDA064A4342E6
:1006600082FB0320DA17C2EB600000EB4000A3EB33
:100670008000C0F10C007047ABAAAA2AF0B40E8823
:1006800086420DD203F10043013B31F813508542FD
:1006900002D9F0BCFFF7B8BF32F81300F0BC7047C6
:1006A0001088F0BC704700BF094B1B880C2B09D881
:1006B000084A80B252F8232028B143F6FE739842CC
:1006C00003D9108C7047108870470349FFF79CBF0F
:1006D000AE9BFF1F2015010024170100374A38493F
:1006E0001088384AF8B5384B12881B68834248DBBB
:1006F0009342A8BF134698420B60C8BF002342DD57
:10070000101AB0F5804FAABF9B03C3EB83330130AF
:1007100093FBF0F0FFF7C8FF2C4B2D4F1C883B6874
:10072000C0F3C61505FB04F47F2CA8BF7F249D42AF
:10073000064608D0274B1B88002B38D1264B1B8838
:10074000002B30D13D60254D2B689E4205D0214BBA
:100750001B885A1F032A1DD92E60214D2B689C42ED
:100760000ED0204B188848B11A4B1F4A1B88D35C07
:10077000834203D0C0B2E1B208F0E6F82C60F8BDC5
:10078000F8BD034608609A42D4BFC0EB0203C0EB39
:100790000303B5E7144AD05C2030C0B206F07F01F5
:1007A00008F0D2F8D8E7284608F042F9CAE70E4A1E
:1007B0002946D05C08F0C8F8C0E700BF289CFF1F9E
:1007C000809BFF1FE49DFF1F8C9DFF1F949BFF1FBD
:1007D000DC9BFF1F729DFF1F1E9CFF1FA89BFF1F1E
:1007E000209CFF1FC49DFF1F9889FF1F2DE9F04F1C
:1007F000172089B00CF0CAFEAF4B186016200CF021
:10080000C5FEAE4BAE4A1B8810600C2B00F03B813E
:10081000AC4BAD4A19880093AC4B52F821400022F2
:100820001A70AB4BAB4D1B88AB4A2E88013B32F99B
:100830001370002E5CD0A94BA94A1B88A9491278D5
:10084000013B31F91380002A40F0DF8011200CF0C9
:100850009DFEA54B0193D3F800A00646B24540F398
:10086000DF80A24BDFF8A4921B88A14A012BD9F8A4
:100870000030B2F800B09F4A02922046C8EB03084D
:1008800000F09A820FF03EFA029A52F82B100FF005
:100890008DFA014600200FF07FF90FF04DFCCAEBF6
:1008A0000802B045B8BFB0469042CAEB080880F2D3
:1008B000968200FB0888013298FBF2F08E4BDFF83D
:1008C00050820293D8F80030034403EBD3735B10DB
:1008D000C8F800302B88012B12D1884BDFF834B2D6
:1008E0000393874BDBF8005004934FF0000A47E076
:1008F0007D4B0193DFF814927F4BDFF81482029353
:100900007E4B03931D460F200CF040FE2B6898424F
:10091000824641DA754A1288012A00F01D82744A23
:1009200005931288734D049220460FF0EBF9049A58
:10093000DFF8E0B155F82210DBF800500FF036FA7E
:10094000014600200FF028F90FF0F6FBEF1B059B86
:100950005745A7EB0302B8BF5746FF1A9042BABFEC
:10096000013200FB0777474397FBF2F7D8F80020E6
:10097000634B0493BB1803EBD3735B10C8F80030D0
:10098000604B1B88013B032B00F2B082DFE813F0C1
:100990006301A901C4008601594B04931B68984266
:1009A00040F3C281514A1288012A00F0A682504ABF
:1009B000079311884F4A0691204605920FF0A2F93D
:1009C000059A0699DFF84CB152F82110DBF8005077
:1009D0000FF0ECF90FF0B0FB079B2F445745A7EB46
:1009E0000302A8BF5746FF1AD8F800309042BABF9A
:1009F00000FB07770132474397FBF2F73B4403EBD9
:100A0000D3735B10C8F80030BAE715200BF07AFEFC
:100A1000354B0193D3F800A00646B2453FF721AF0E
:100A2000354B0293D3F800A0B24580F289812F4B59
:100A3000DFF8D8901B882E4A012BD9F80030B2F885
:100A400000B02C4A03922046984400F070820FF0C8
:100A500059F9039A52F82B100FF0A8F90FF06CFB1C
:100A6000B045CAEB0802A8BFB046CAEB08089042DE
:100A7000B6BF00FB088800FB08F8013298FBF2F0D3
:100A8000DFF88C801EE7204B1B78002B3FF4C0AEB4
:100A90000C4B0D4A198800930C4B52F8210001228F
:100AA0001A700FF02FF94FF07C510FF07FF90FF013
:100AB00043FB0446B5E600BFD49BFF1FBE9DFF1F4E
:100AC000049EFF1FD89BFF1F5889FF1F8A9BFF1F93
:100AD0002089FF1F2C9DFF1F0C190100A889FF1FF3
:100AE000A29DFF1F00170100089EFF1F0C9CFF1F07
:100AF000C89BFF1F24190100009CFF1FB09DFF1F12
:100B0000249DFF1F2E89FF1F709DFF1F789BFF1FD5
:100B1000C89DFF1FAC9DFF1F28460FF0F3F8B24998
:100B20000FF044F9054650460FF0ECF8AF490FF0CE
:100B30003DF9014628460FF031F80FF0FDFA054661
:100B4000CBF80050D9F800000FF0DCF8A6490FF000
:100B50002DF9074630460FF0D5F8A4490FF026F9D5
:100B6000014638460FF01AF80FF0E6FAC9F800000F
:100B70009F4AA04B168819889F4AA04B12681B8871
:100B80009F4FC6EB050E3544039EC6F800E0461A9B
:100B9000084404990D6001990E6002993E8808602E
:100BA0009A4280F289810025C3EB060E954974456F
:100BB0000F6880F27681611C9F4205FB01F50EF102
:100BC000010E95FBFEF5C0F2BE81BE42A8BF3E46B7
:100BD000F61A01FB06F494FBFEF49A4200F3368108
:100BE000BB42C0F23381884C20680FF08BF88749F4
:100BF0000FF0DCF886490EF0D1FF0FF09DFAA0F55A
:100C0000FF531C3B082B98BF4FF40050D8F800301E
:100C1000184400282060C0F24281B0F5804F80F275
:100C200052817C4B1B781BB1B0F5005F40F05381C3
:100C3000794D2B78002B40F05481784D20682B683B
:100C4000714C984204D080B207F05CFF23682B609F
:100C500009B0BDE8F08F28460FF054F870490FF046
:100C6000A5F8054650460FF04DF86E490FF09EF876
:100C7000014628460EF092FF0FF05EFA0546CBF8CB
:100C80000050D9F800000FF03DF865490FF08EF8DC
:100C9000074630460FF036F862495FE728460FF006
:100CA00031F85A490FF082F8054650460FF02AF8FD
:100CB0005D490FF07BF8014628460EF06FFF0FF0FC
:100CC0003BFA0546CBF80050D9F800000FF01AF8AF
:100CD0004E490FF06BF8074630460FF013F85249B3
:100CE0003CE728460FF00EF850490FF05FF8054634
:100CF00050460FF007F84E490FF058F801462846C5
:100D00000EF04CFF0FF018FA0546CBF80050D9F85A
:100D100000000EF0F7FF45490FF048F8074630464F
:100D20000EF0F0FF424919E7D8F80030DFF810B1B3
:100D300003EBD3735B10DBF80050C8F800301FE6FC
:100D4000DFF80081DFF80091D8F8003003EBD373AF
:100D50005B10C8F80030BDE5364A06931188364A64
:100D6000059120460492DFF8D8B00EF0CBFF049A2C
:100D70000599DBF8005052F821100FF017F80FF02A
:100D8000DBF9EF1B069B5745A7EB0302B8BF57469D
:100D9000FF1AD8F800309042BABF013200FB077743
:100DA000474397FBF2F73B4403EBD373234A049288
:100DB0005B10C8F80030E3E50EF0A4FF029A52F889
:100DC0002B100EF0F3FF0FF0B7F9CAEB0802B04595
:100DD000B8BFB0468242CAEB08083FF76AAD00FBD5
:100DE00008F898FBF2F069E5CDCC4C3FCDCC4C3EF9
:100DF000A489FF1F2C89FF1FD49BFF1F889DFF1F05
:100E0000C09BFF1F049EFF1F8C89FF1F9A99193FEB
:100E1000CDCC4C45BA9EFF1F1D9CFF1F2489FF1F90
:100E20003333733FCDCC4C3DCDCCCC3E6666663F74
:100E3000CDCCCC3DC89BFF1F24190100249DFF1F72
:100E4000AC9DFF1FC89DFF1F789BFF1F009B1B8849
:100E5000002B3FF4C8AE2B1B002BB8BF5B42092B05
:100E600047DD05F500500130001B0EF04BFF3B49FC
:100E70003B4C0EF09BFF054620680EF043FF3949BE
:100E80000EF094FF014628460EF088FE0FF054F94C
:100E9000D8F80030184400282060BFF6BEAE00220B
:100EA00013E09F4205FB04F5B8BF002195FBFEF55A
:100EB0004BDA91FBFEF490E6B242D4BFC3EB0205DD
:100EC000C3EB060570E643F6FF72274B22601B78E2
:100ED000002B3FF4ADAE04F0B3FF244B01221A7097
:100EE000ABE604F0A9FF00232B70A6E6D9F80000BA
:100EF0003EE64FF400501A4C88E61D491D4A069301
:100F000020460D8805920EF0FDFE059ADFF868B0C8
:100F100052F82510DBF800500EF048FF0146002083
:100F20000EF03AFE0FF008F92F44069B56E50EF03E
:100F3000E9FE039A52F82B100EF038FF014600200C
:100F40000EF02AFE8AE51E4642E6B742D4BFC3EB46
:100F50000701C3EB060104FB01F1AAE7CDCCCC3EAF
:100F60008C89FF1F9A99193FBA9EFF1F1D9CFF1F76
:100F7000C89BFF1F24190100AC9DFF1F08B5244B1F
:100F80001B88FBB1234B1B78FBB1234B1B78E3B1D0
:100F9000224B1B78CBB1224B1B78B3B1214B22489B
:100FA0001A78C2B9214A2249008812880968024485
:100FB000B1EB620F09DD01221A706420BDE8084020
:100FC00004F052BF174A117801B908BD1370BDE88B
:100FD000084007F061BD154A164900881288096863
:100FE0000244B1EB620FF0DD00221A7007F054FDED
:100FF000642004F039FF642004F036FF642004F01C
:1010000033FF4FF41670BDE808400CF0CDB800BFB8
:101010002E9DFF1F0F9EFF1FDE9DFF1FDF9DFF1FE9
:10102000E09DFF1FAC9BFF1FC09BFF1F889DFF1F04
:10103000D49BFF1F049EFF1F38B5114C2320257839
:101040000BF060FB0F4A42F82500131F02F1C400A9
:10105000002253F8041F83420A44FAD123780A4934
:1010600007480A4C0133DBB2322B81FB025108BF27
:101070000023D217C2EB21120370226038BD00BFDB
:10108000969BFF1F389CFF1F1F85EB51849DFF1F00
:101090002DE9F04FB84CB94D2068B94F83B00EF030
:1010A00031FEB8490EF082FE064610200CF06EFAB2
:1010B0000EF028FEB4490EF079FE31460EF06EFDBA
:1010C0000FF03AF82988206088423B8843DA9E4630
:1010D0005B1A7F2B4FF0000247DDD2015E1C92FBB2
:1010E000F6F2AA4EDFF8C882B6F800C0C8F80020B1
:1010F000BCF1190F00F0DF80BCF11A0F00F017816E
:10110000BCF11E0F00F020810126B146A04A1288D2
:10111000002A00F09D808842C0F207817045D4BF4C
:10112000C1EB0000C1EB0E009A42BABF02FB000007
:101130000133504390FBF3F3964A1360964B1888A3
:10114000C0B9964A1288AAB9954B197801B11A709C
:1011500003B0BDE8F08F9842D4BFC1EB0002C1EBF1
:1011600003029E465B1A7F2BB7DCC2EBC21292FBD6
:10117000F3F2B6E72988D4F800E0DFF80082DFF860
:10118000F8A171456CDCDFF818C29CF80020002A39
:101190002ED14FF0010B04288CF800B028D1002E7E
:1011A00040F094817D4B18880028D1D0B9F1000F10
:1011B000CED023682C883A88A34280F26581002330
:1011C000141B7E2C774DD5BFC3EB8313C3EBC31326
:1011D0005B00013493FBF4F42B680134A34203D089
:1011E000C0B2E1B207F0B0FB2C6003B0BDE8F08FF5
:1011F000012800F0F680022800F0EB800328D1D10E
:10120000694B1B88092BCDD0002ECBD023682E88AC
:101210003A88B34280F27B810023961B7E2EDFF852
:101220008CA1D5BFC3EB8313C3EBC3135B000136A3
:1012300093FBF6F6DAF800300136B34203D0F1B290
:101240004A2007F081FBCAF80060ABE716469146DA
:10125000BCF11E0F7FF472AF0022DFF858817EE0F0
:101260004F4B1A78002A3FF473AF002401281C70FA
:1012700000F0A480022840F00E81002E00F0A38030
:101280004A4D2B68002B00F09E800420214607F079
:101290005BFB424B2C60188800283FF459AFB9F132
:1012A000000F3FF455AFC0B2002107F04DFB3D4B9E
:1012B00000221A604CE7DFF8FC8098F80020C2B1E9
:1012C000DFF8D890B9F800A0BAF1000F11D0DFF81C
:1012D000E89099F800B0934578D05FFA8AF07F21C2
:1012E00007F032FB98F80030B6F800C089F80030FB
:1012F00010E0DFF8C49099F800A0924566D0274B23
:101300000021187807F020FB98F80030B6F800C0EC
:1013100089F800301E4B1A88002A97D0BCF11E0FA6
:1013200040F006810026B14619E00020FCE6DFF817
:10133000848098F80020002A0BBF012600264FF079
:1013400000094FF00109E1E6DFF86880104B98F8DA
:1013500000601A88B6FA86F676094FF0000998F808
:101360000030002B3FF4E8AE2988B7F800E0206891
:10137000C1EB0E03CFE600BFCC9BFF1F349DFF1FC8
:10138000309DFF1F9A99193FCDCCCC3EBE9DFF1FCB
:10139000EC9DFF1F309CFF1FD29BFF1FCE9DFF1FA8
:1013A000C79DFF1FB49BFF1F729DFF1F349CFF1F33
:1013B000A49DFF1F709DFF1F9A9BFF1F1EB1614DD3
:1013C0002B68002B7BD1604B188865E70026B1465F
:1013D0009CE6002E3FF4E6AEDFF868A1DAF80020C4
:1013E0002EE0002E3FF4DEAEB7F80080F045D4BF0B
:1013F000C1EB0802C1EB0E02C1EB0808B8F17E0F89
:10140000DFF840A1D5BFC2EB8212C2EBC21252007C
:1014100008F1010892FBF8F8DAF8002008F1010859
:10142000424506D05FFA88F10120009307F08CFA5C
:10143000009B1888CAF8008002287FF4DFAE42467D
:101440002168B5F800803888414559DA0021C8EB99
:101450000008B8F17E0FD3BFC1EB8111C1EBC11100
:1014600008F10108490091FBF8F808F101089045DE
:1014700006D05FFA88F10420009307F065FA009B1C
:101480001888CAF80080B9E69342D4BFC4EB0303BE
:10149000C4EB020394E6032827D12C4B1B88092BAD
:1014A00091D0002E8FD0274D2B68002B8BD04A2057
:1014B000214607F049FA244B2C601888ECE62146B7
:1014C00007F042FA204B2C601888E5E640207F2187
:1014D0008DE80C0007F038FA019B009A18885845EF
:1014E0001CD002287FF48AAE76E704287FF46BAF25
:1014F000002E3FF468AF2146402007F025FA62E74E
:101500008142D4BFC8EB0101C8EB00019FE79342C1
:10151000D4BFC6EB0303C6EB02037EE6B8F80010A7
:10152000DAF800E0B7F800808E45FFF665AF5DE7BA
:101530002988B7F800E020680026C1EB0E03B14609
:10154000E9E500BF349CFF1FCE9DFF1F729DFF1F6A
:1015500008B5114B1B88022B09D0052B07D0032B94
:1015600015D0042B0BD00D4B01221A7008BD7F2122
:10157000412007F0E9F9094B01221A7008BD7F21CB
:10158000092007F0E1F9054B01221A7008BD40213E
:10159000092007F0D9F9E6E72E9CFF1FEC9BFF1FFF
:1015A00038B5244B1B881D2B40D0234B1B88012BA7
:1015B00025D0224A224B14881B68224AA342128853
:1015C00028DB214909889342D4BFC4EB0303C4EB51
:1015D0000203121B914224DA01FB0333541C93FBD8
:1015E000F4F41A4B1A4D1B88052B06D02B689C422D
:1015F00003D0E1B2052007F0A7F92C6038BD154BE8
:10160000154A1B681488154AC3F53B630833A34287
:101610001288D6DA0C490988121B91424FF0000358
:10162000DADB03FB01F393FBF2F4DAE7064B1C88E9
:10163000D7E700BFBE9DFF1F2C9DFF1FA89DFF1F6A
:101640008C9BFF1FBC9DFF1FC29DFF1F2E9CFF1F79
:10165000849BFF1F389DFF1F2C9CFF1FAA9DFF1F0F
:1016600038B5124D124C2B88052B12D022684AB97E
:10167000022B0ED0033B012B13D90E4A002313700B
:10168000236038BD0021052007F05EF92B88022B6E
:1016900004D10021412007F057F9EEE7052BE9D1ED
:1016A000F7E70021092007F04FF9E6E72E9CFF1F1E
:1016B000849BFF1FEC9BFF1F08B5284B1B78ABB129
:1016C00015200BF01FF8264A264B128818601D2A99
:1016D00015D0254A1288DAB1012A2BD0234B1B786A
:1016E000002B3AD0BDE80840FFF7BABF11200BF03D
:1016F0004DFF1B4A1B4B128818601D2AE9D11C4B59
:101700001B88002BEAD01B4B1B78002BE6D008E08F
:10171000174A1288002AE1D0174A1B6812889A4299
:10172000DCDC124B1B780BB9FFF712FFBDE8084059
:10173000FFF736BF0F200BF029FF0D4B0F4A1B8818
:10174000106033B10E4BC0F53B601B8808309842E7
:10175000E7DA064B1B78002BC4D108BDA29DFF1F02
:10176000BE9DFF1F8C9BFF1F2C9DFF1FEC9BFF1F2F
:101770002E9CFF1F709DFF1FA89DFF1F389DFF1F00
:101780002C9CFF1F38B510200BF000FFC830B0F5BF
:10179000FA7FC0F2EF80B0F57A6F0146A8BF4FF430
:1017A0007A6101F51673B3F57A6FA8BF4FF47A63C7
:1017B0009BB289B28E4A8F4C11802220238007F081
:1017C00047FA21888C4D8D4C242007F041FA0E20D9
:1017D0000AF098FF40F6FF71C8308842A8BF08465B
:1017E00020EAE07000F5FA6283B28A42A8BF0A4696
:1017F0000220194622802B8007F02AFA2188042033
:1018000007F026FA17200BF0C1FE044616200BF055
:10181000BDFEA042B8BF204600F1C801B1F5FA7F75
:10182000C0F2A380B1F57A6FA8BF4FF47A6101F5D9
:101830004873B3F57A6FA8BF4FF47A639BB289B24D
:101840006F4A704C11800A20238007F001FA21882A
:101850000C2007F0FDF90F200BF098FEC0F53F615A
:101860000E31B1F5AF6F7DDBB1F5FA6FA8BF4FF464
:10187000FA6189B2C0F54460634B0E30B0F5AF6FCA
:1018800019806CDBB0F5FA6FA8BF4FF4FA6083B231
:101890005E4CA420238007F0DBF9A620218807F006
:1018A000D7F90B200BF04AFC002868D011200BF070
:1018B0006DFE00F1C801B1F52F7F6EDA40F21453CE
:1018C0004FF42F71524A1180524C0620238007F0AA
:1018D000BFF92188082007F0BBF900244FF4AF7549
:1018E000E1B24D4808F04CFF01348542A8BF0546DF
:1018F0000C2CF5D101200BF049FE044600200BF022
:1019000045FE323CA0F1320344496FF4957000FB70
:1019100003F300FB04F081FB034281FB0041DB1772
:10192000C017C3EB6223C0EB612003F5AF7200F573
:10193000AF739342A8BF13469D42A8BF1D46A5F1B1
:101940001401312938DC40F26C7332213448354AB5
:10195000018013602A20BDE8384007F079B94FF4C0
:10196000AF6395E74FF4AF6184E740F214534FF44F
:10197000FA7165E740F24C434FF4FA711AE715200B
:101980000AF0C0FE00F59671B1F52F7F96DB41F2AB
:101990005C2399421FDD194694E741F25C2399428A
:1019A000F9DC1B4A00F5487089B2B0F52F7F118031
:1019B00019DA4FF42F7387E740F23A72A5F5B9753B
:1019C000194B02FB05F583FB0523ED17A5EB63130C
:1019D00089B23233BAE70E4A00F5617089B2B0F5C8
:1019E0002F7F1180E5DB8342A8BF03469BB26BE7E4
:1019F000349DFF1F309DFF1F289CFF1FE49DFF1F8C
:101A0000889DFF1FC09BFF1F2C9CFF1FAA9DFF1FCF
:101A1000A89DFF1FBC9DFF1F1C9CFF1F67BBCF46DF
:101A2000DC9DFF1F9489FF1FB5814E1B2DE9F84FE8
:101A30000C200AF033FE0C200BF0E8FAA149142028
:101A40000BF0F4FAA049A14808F02CFB0221032076
:101A50000BF082FB022104200BF07EFB022105200B
:101A60000BF07AFB022106200BF076FB01210A2005
:101A70000BF072FB012109200BF06EFB01210D2000
:101A80000BF06AFB012128200BF066FB01211420DA
:101A90000BF062FB02210B200BF05EFB01210C20FE
:101AA0000BF05AFB0C2000210BF042FB04200BF042
:101AB00045FB70B305200BF041FB044680B30024C6
:101AC0002046834D287005F0D1FC2B78EBB92046D9
:101AD00007F0E8F87F4B80491B88804D0988804AD1
:101AE0002970A3F5AF7140F23A7303FB01F382FB57
:101AF0000312DB177B4E7C48A3EB621332335A216F
:101B0000336008F079FE90B9FEE7BDE8F84F08F0C1
:101B1000D9B906200BF012FB0028CBD10124D0E765
:101B200003200BF00BFBB0FA80F04009C9E76F4AC5
:101B30006F481268DFF800B200230121FEF7B4FC01
:101B40000B200BF0FBFA011E0CBF012300238BF8C6
:101B5000003002D111200BF0FFFADFF8A091654FA1
:101B6000DFF8D881644E0023C9F800303B60C8F824
:101B700000304FF0040A14E00AF0C4FD3B6818443A
:101B800038600AF0010080F0010004F05DF933884C
:101B9000002B14BF4B20DC200BF006FBBAF1010A2E
:101BA0001BD00F200BF0F2FCD8F8003003440E20BD
:101BB000C8F800300AF0A6FDD9F800309BF80020E4
:101BC0000344C9F800301520002AD5D111200BF0AC
:101BD000DDFC3B6818443860D3E7D8F80030D9F80A
:101BE000002046493868DFF858E1DFF858C1002B7B
:101BF000B8BF0333002AB8BF033292100A604049CD
:101C0000404A098812880028B8BF03309B10801012
:101C100038605F1A1944CEF80070CCF80010DFF875
:101C200028E1394F3949C8F80030C2EB000C0244B2
:101C3000CEF800C03A600B600CB1FFF7A3FD33880B
:101C40005BB94FF4FA7004F00FF904F0F9F805F0FD
:101C50001FFF4FF4AF600BF0A7FA2D4B01240420B7
:101C60001C600BF06BFA10B92A4B28701C702A4BC1
:101C70001B881C2B1CD0294C04F1C80523200AF01A
:101C800041FD44F8040F01200BF08EFAA542F5D176
:101C9000234A244B1078187006F00EFF04F0CCF89D
:101CA00045F6BF5220492148BDE8F84F0AF0E2BA94
:101CB0001F4B18880028DED01E4BC0B2197806F0E2
:101CC00043FED8E7001B374640420F006890FF1FD5
:101CD000B29BFF1FDC9DFF1FC09DFF1FFC9BFF1FD2
:101CE000B5814E1B9489FF1F1C9CFF1F2889FF1F75
:101CF000509DFF1F789BFF1F7E9DFF1F909BFF1F26
:101D0000A489FF1F2C89FF1F009CFF1FF49DFF1F4C
:101D1000B89DFF1F9E9BFF1FBE9DFF1F349CFF1F92
:101D20003C9DFF1F229DFF1FA5050000D49DFF1FA6
:101D3000049CFF1FCA9BFF1FA29DFF1FAC9DFF1F9E
:101D4000B09DFF1F249DFF1F089EFF1F2DE9F04F30
:101D50008BB007ADB54F2C460AAE611BC9B2B44873
:101D600008F00EFD3B88834294BF0020012004F858
:101D7000010BA642F1D1AF48AF4A9DF81C70AF49A4
:101D800007709DF81E00AE4D10709DF820209DF844
:101D90002430AC4EAC4C0A709DF8221029700025FE
:101DA0003370257073B9002940F00581A7491AB135
:101DB0000B78002B40F0EC81002800F0BF8102235B
:101DC000237005E0002A40F0A78005239F49237077
:101DD000DFF8D0B2DFF8D0829DF81D209DF82100F9
:101DE000DFF8C892DFF8C8A2994D9A4F9A4E0B704F
:101DF0009DF81FC09DF823109DF827309DF826E020
:101E00008BF8002088F800009DF82520297001201B
:101E10003A70337089F800C08AF800E00BF0B6FB26
:101E20008E4A8F4B11688842CCBF012200221A7063
:101E300076DD8C4B1B88182B72D88B4AB2F800E0E9
:101E40000C3B0093BEF1000F72D1884A9BF800C092
:101E500092F800B098F8008099F800209AF8009065
:101E600094F800A02C78ABEB4C0BC2EB0B0BA8EB5F
:101E7000880EDE44C9EB897BC9EB8B09DFF8F4B12E
:101E8000F14497F800E0BBF800B009EB440934785E
:101E9000CE4404FB0BEE4FF00C09754C19FB0AEE17
:101EA000C4F800E0B8F1000F0BD036784EB1714E97
:101EB0003688042E0CBF0EF1020E0EF1040EC4F88B
:101EC00000E06D4CDFF8EC912488B9F800A06B4E6F
:101ED000DFF8E4913688D9F80090009B033C04EBCE
:101EE0004404CAEBCA0A0EEB84043444D144644E61
:101EF0000C3C56F829601C44A319BCF1000F28D0F3
:101F00002C7834B3002A5AD1B8FA88F85D4C4FEADD
:101F1000581884F8008023E0062323704B4957E7C4
:101F2000514AB2F800E000230093BEF1000F8CD0BC
:101F3000BEF1010F47D0BEF1020F00F0C1804C4C42
:101F40009BF800C099F8002098F80080D4F800E0D1
:101F5000A8E74C4C002525700AB13A781ABB00223C
:101F6000494C884222704949C4BF494AC2F800E03E
:101F70000A68934213D0474A474C10680590059869
:101F8000206012680692454C069A24880B60121A4B
:101F9000A24284BF424A13600BB0BDE8F08F3E48B6
:101FA0003C4A0068EDE7BCF1000FD8D1B8F1000F52
:101FB000D5D10122D4E704232370244908E7314A0C
:101FC00000241470CBE7294A9BF800C092F800E087
:101FD00098F8008099F8002094F800B09AF80090E2
:101FE0002C780194AEEB4C0EC2EB0E0EA8EB8804DD
:101FF0007444C9EBC909D944A31EDFF878A0DFF8FF
:10200000BCE0019C97F800B05EF829E0BAF800A0A7
:1020100096F8009003EB44045C4409FB0A4909F17B
:102020001809134CCE44C4F800E03BE7DC9DFF1FC9
:102030001C9CFF1FDE9DFF1FDF9DFF1FE09DFF1FFC
:10204000E19DFF1FE29DFF1F299DFF1F329DFF1F86
:10205000109EFF1F119EFF1FC69DFF1F9489FF1F2B
:10206000709DFF1FBE9DFF1F889BFF1FA689FF1F3E
:10207000789DFF1FDA9BFF1F949DFF1F989BFF1FFA
:1020800054150100EE9DFF1FEF9DFF1FE49BFF1FF6
:10209000F89DFF1FF89EFF1F089CFF1FCC9DFF1F90
:1020A000009EFF1F0C9EFF1F0E9EFF1F0D9EFF1F19
:1020B0000F9EFF1FB49DFF1F309CFF1FD41801000F
:1020C000374A9BF800C092F800B0247899F80020B5
:1020D00098F800800394ABEB4C049AF80090314BD5
:1020E00095F800A0CDF804A0A8EB880BA41A5C44D6
:1020F0004FF0050B1BFB094B039C97F800A0CDF894
:1021000008A0C9EBC909B3F800A009EB0403BDF8A6
:102110000490029C0BF1050B1EFB09BE96F800B063
:10212000DFF8A490A6440BFB0AEE59F823901E4C4E
:102130000EF10C0ECE44C4F800E0B3E65FBB0B78A2
:10214000012B2BD9194A23701288002A3FF440AE84
:10215000174A1288013A92B2062A3FF639AE154A5A
:102160001278002A3FF434AE134A1268012A7FF431
:102170002FAE1248124A0068124E82FB0025C21789
:10218000C2EB650202EB4202A0EB820232801FE644
:10219000032323701CE60123237019E63B4617E650
:1021A000A689FF1FDA9BFF1F789DFF1FA09DFF1FC1
:1021B0003E9DFF1F2A9CFF1FB89DFF1F009EFF1F13
:1021C000ABAAAA2A7C9DFF1FFC1A01002DE9F04F43
:1021D0003A4B1B788BB0002B6BD10E200AF092FA91
:1021E0000DF090FD01463648364E374DFEF7A2F908
:1021F0003348FEF775F90DF09FFF80F30C00306057
:10220000FFF7A4FD2C68012C7AD0022C00F0A782E5
:10221000032C00F0B5832D4E2D4C33682D4A2E4EE5
:102220000993099B316812882360591A013A914237
:10223000274F00F28F82294E32689A1A0D2A00F237
:102240008282274E32689A1A132A00F27782254E2C
:1022500032689A1A252A1AD9234B1B88002B40F082
:102260005D81224B1B78002B40F05881FEF7E4FE85
:102270001F4B1B881B3B9BB2022B04D81D4B1B78AA
:10228000002B40F04E8103F001FE236833601A4DAD
:102290002A689B1A502B00F20D82184B1B88012BC9
:1022A00000F0258206F0E4FB06F012FA0BB0BDE860
:1022B000F08F07F08FFC0BB0BDE8F08FB29BFF1FD3
:1022C000509DFF1F8C9DFF1FB89DFF1FF89EFF1F95
:1022D0004C9DFF1F9089FF1F249CFF1F149CFF1F14
:1022E000F49BFF1FF89BFF1F2E9DFF1FAC9BFF1F42
:1022F000BE9DFF1F709DFF1F409DFF1F909DFF1FF4
:10230000DFF82093A04AB9F800001378834204D084
:10231000C3B21846137006F0E7FADFF804839B4A4D
:10232000B8F800301178994204D0994F39780029D3
:1023300040F0E486974A33681288974E9A42C0F27A
:10234000FA80964A1278002A40F0F580DFF8D8A289
:10235000BAF8003023B9924B1B88002B00F0EE84B2
:10236000904A914B11881B88904A0B4412685B106D
:1023700093428F4A126880F2908400219342B4BF46
:1023800001230B4604910093ACBF4FF0010B8B4629
:1023900005910E200AF0B6F9864B874A1B6817682C
:1023A00003930133A7F25232002B8446029240F38A
:1023B000CC86802BA8BF8023804A81491278019166
:1023C000002A00F0C2800978914200F0BE80B8F87F
:1023D0000010DFF84CE2994201F0E1806C49AEF860
:1023E0000030784B4FF0010E81F800E01978DFF8EB
:1023F0003CE2019B8EF800101A70009B002B00F04D
:102400001781BAF80030002B00F012816E4B1B6868
:102410005A1C002A40F39D86802A00F399866B4C53
:102420006B496C482488098800682144B0EB610F2F
:10243000C1F22A83A3F148020F2A02D8473BA9F828
:1024400000300E200AF05EF96FF454731F44874287
:1024500002DC614B00221A7000200BF097F85F4AF3
:102460005F4B11685F4C1B888842D4BF0022012259
:102470002270002B00F008845B4B1C78944240D003
:1024800088423EDD59490C78002C00F01E875849DF
:1024900091F800C0BCF1000F40F01587554F009730
:1024A000554F56480297534F007887F800C0524F57
:1024B0004FF0010E87F800C081F800E0002841F0DD
:1024C000C5804F490978002900F0E1874D49039103
:1024D0000C460978002940F0D7874B48464F0078D2
:1024E000397001210297217058B14248404900904B
:1024F000002008700099029F0870039901243C7025
:1025000008701A70414B1B88A3F11B02012A40F28C
:10251000B9851D2B00F003863D4C7EE6FEF72EFDAF
:10252000A4E63C4B1B78002B3FF4ADAE2B68012B8F
:102530007FF4A9AEA9E63168374A06910698374973
:10254000106002220B602A6000E71E49DFF8DCE021
:10255000097800293FF44DAF9EF8000081423FF416
:1025600048AF03984B2840F3E1871833802BB8F825
:102570000000A8BF802398423FF43BAF2848038067
:1025800003480123037034E7229DFF1FFC9BFF1FBC
:102590009E9BFF1F289CFF1FF89EFF1FAC9BFF1FE9
:1025A0001A9CFF1FC09BFF1F889DFF1FD49BFF1F0E
:1025B000049EFF1FF89DFF1F909BFF1FEE9DFF1FB6
:1025C000E09BFF1FEF9DFF1F789DFF1F349DFF1FA6
:1025D000309DFF1FCC9BFF1F289DFF1F9489FF1F6D
:1025E0003E9DFF1FC69BFF1F7C9BFF1F0F9EFF1F73
:1025F000809DFF1FD09DFF1F2A9CFF1F109EFF1F65
:102600000C9EFF1F7D9BFF1F709DFF1FBE9DFF1F28
:102610004C9DFF1FC69DFF1FF09BFF1F489DFF1F86
:10262000C09DFF1F3C9DFF1FE89BFF1FE19BFF1FFD
:10263000029B9C45BFF605AF864B1B88002B3FF4E1
:1026400000AFBBF1000F7FF4E1AE834B1B881BB1E1
:10265000059B002B7FF4DAAE049B002B3FF4F1AE18
:102660007E4B1A78002A7FF4ECAEDFF8649299F87A
:10267000004001221A70002C40F02D83784B1B780B
:10268000002B02F0C680774B1B78002B02F09A8358
:10269000754B1B78002B7FF4D4AE744B1B78002B4A
:1026A0003FF4CFAEB8F8003071490A3BA8F80030CB
:1026B0000A70C6E604F022FF6E4B1B7873B96E4BAE
:1026C0001B785BB96D4B1B7843B96D4B1B782BB9ED
:1026D0006C4B1B7813B903F0AFFB01E003F0B8FBC0
:1026E00023682B60684B1B88012B7FF4DBAD674AA6
:1026F000674B116867481A78A1F118032A2101FB7A
:1027000003F10160002A00F0A982634C236899421A
:1027100000F3528310DA61480278002A40F07C8787
:102720005F4A1068D0F17F0048BF0330801001304D
:102730001B1A994242F3BF86216091E2FEF7BCFF6B
:102740002368336083E5FEF751F8FEF7A1FC2368A8
:10275000336076E5FDF7C2FF3B6833606BE5514AB5
:1027600034681188A14204DB464B1B78002B00F033
:102770005D834D4E4D48336807934D4B079A006873
:102780001B88121A9A4200F2A980002B00F0A68042
:10279000484B1A88002A3FF4BFAE474B47481B6896
:1027A0000088A342B8BF2346994241F36681444B57
:1027B0001960DFF8208188F80020344FFDF78EFF84
:1027C00038687F2840F371853E4B7F3883FB0032A9
:1027D000C317C3EB620303EB4303A0EB8300733027
:1027E000394B01931B883860002B40F0CA86234B7D
:1027F00000931B78002B00F0C683344C2378002B09
:1028000000F0C183DFF8D090DFF8B8A04FF0000BE4
:102810000CE003F17300C0B298F8001006F0BCF8A9
:1028200023780BF1010B5B4540F3AD833B6859F80E
:10283000040F1844A0F17F038AFB0321DA17C2EBCF
:10284000610202EB42027F28A3EB8203E1DCFDF789
:1028500003FFE0E71A9CFF1F449DFF1F289DFF1FF9
:102860000C9EFF1F0D9EFF1F0E9EFF1F0F9EFF1F42
:102870009E9BFF1F2A9CFF1F809DFF1FD09DFF1F57
:102880007D9BFF1FAC9BFF1F909DFF1F009EFF1FA6
:10289000EC9BFF1FE89DFF1FA49BFF1FD19DFF1F07
:1028A000849BFF1F289CFF1FF89EFF1FF09BFF1FAC
:1028B000189CFF1F9C9BFF1F489DFF1FE49DFF1F4F
:1028C000809BFF1FABAAAA2AD09BFF1F5489FF1F22
:1028D000299DFF1F0E9CFF1F2C89FF1F554B564A39
:1028E0001B681088554AA342B8BF2346994200F39B
:1028F0007A82534C12888342A8BF03462360002A81
:102900007FF457AF9942C8BF134640F37382401A11
:10291000B0F5804FAABF9B03C3EB8333013093FB19
:10292000F0F0FDF7C1FEC0F3C6100DF0EBF9454B1A
:10293000044618880DF0E6F94349074620460DF095
:1029400035FA014638460DF031FA21460DF026F9E8
:102950004FF07E5104460DF0C7FB002841F0718016
:102960003A4920460DF0DEFB002840F069862046FB
:102970000DF008FCC0B2DFF8F48088F800001CE716
:10298000334B34681988A14274DD324B1B78002B1D
:1029900070D1DFF8DC9099F800007F2840F338868A
:1029A000A3F155337F3803F1004383FB0032C31793
:1029B000C3EB620303EB4303A0EB83007330264BAE
:1029C00001931B88C0B289F80000002B41F03580CC
:1029D000224B00931B78002B00F0A484204C23781A
:1029E000002B00F09F841F4FDFF87C804FF0000A1F
:1029F0000AE003F17300C0B205F0F6FF23780AF194
:102A0000010A534540F38E8457F8043F99F80000BB
:102A10001844A0F17F0388FB0321DA17C2EB61029F
:102A200002EB42027F28A3EB8203E2DCFDF714FEF7
:102A3000E1E700BF489DFF1FE49DFF1F9C9BFF1F18
:102A4000809BFF1FF09DFF1FCDCCCC3D0000FE42C0
:102A5000289CFF1FAC9BFF1FD09BFF1FD09DFF1F1B
:102A60005489FF1F2C89FF1FABAAAA2A0E9CFF1FA7
:102A7000749DFF1FB34F38687F2800F3C281FDF7B4
:102A8000EBFDDFF8249399F800A0824500F0218245
:102A9000AD4B1B88002B43D1AC4AAD48126800886F
:102AA000914205DC8242D4BFC1EB0203C1EB0003BB
:102AB000411AB1F5804FA6BF9B030131C3EB8333AD
:102AC00093FBF1F0FDF7F0FDC0F3C6100DF01AF91D
:102AD000A04B044618880DF015F99F498046204602
:102AE0000DF064F9014640460DF060F921460DF005
:102AF00055F84FF07E5104460DF0F6FA002840F0EC
:102B00008F87964920460DF00DFB002840F09585F3
:102B100020460DF037FBC0B2DFF8908288F8000045
:102B2000BAF17F0F40F3BD838D48AAF17F0A80FB85
:102B30000A304FEAEA73C3EB600000EB4000AAEBF7
:102B400080007330874B00931B78C0B289F8000077
:102B5000002B40F01A83844B03931B78002B40F02A
:102B60004B85824B02931B78002B40F07E87804B75
:102B70000193029B1B78FBB17E4B1B88012B00F05D
:102B8000C385022B01F05380032B01F09281042BAB
:102B900001F09D83052B01F03E84062B01F00D868C
:102BA000072B01F0C187082B02F07880092B02F077
:102BB0008C810A2B02F0C283009B1B78002B00F053
:102BC0007684019B6A4C1988002900F0FD843868DE
:102BD0007F2840F36383624B7F3883FB0032C31747
:102BE000C3EB620303EB4303A0EB83007330386055
:102BF000002940F0AC84009B1B78002B00F075810D
:102C00005D4C2378002B00F07081DFF8A4A1DFF881
:102C10009C814FF0000B0CE003F17300C0B298F8F8
:102C2000001005F0B9FE23780BF1010B5B4540F372
:102C30005C813B685AF8040F494A1844A0F17F03AD
:102C400082FB0321DA17C2EB610202EB42027F280A
:102C5000A3EB8203E0DCFDF7FFFCDFE7474B1960E5
:102C6000474B1B68A92202FB03F3002BBCBF03F5F3
:102C70007F533F339B13543B194481F30C012820AD
:102C80000AF0C6F8FFF70EBB384C3E483549364AC5
:102C9000237003700B70137034E493424FF0000BF9
:102CA00080F2BC800123CDF800B0CDF814B00493BD
:102CB000FFF76FBB344B1B78002B7FF4C2AB039B39
:102CC000324A243B83F34703D9B25B20136005F0FB
:102CD0003BFE99F80040032C30D1DFF8D88098F8FB
:102CE0000030002B42F0BD81294F3B78002B42F091
:102CF000AB81254C2378002B42F09981254B1B7822
:102D0000002B42F08781244A1380244B1B78002B30
:102D100042F04D820C4B7F221A8098F800306BB93C
:102D20003B785BB923784BB91D4A7F21072013807C
:102D300005F00AFE7F210B2005F006FE194B1F68E7
:102D4000FFF77FBB009EFF1F9C9BFF1F809BFF1F09
:102D5000E49DFF1FF09DFF1FCDCCCC3D0000FE4247
:102D6000ABAAAA2AD09DFF1F7D9BFF1F2A9CFF1F95
:102D7000D09BFF1F3E9DFF1F5489FF1FA49BFF1F79
:102D80008C89FF1F809DFF1F0F9EFF1FBC9BFF1F95
:102D90000E9EFF1F0D9EFF1F1E9CFF1F109EFF1FFC
:102DA000729DFF1F909BFF1F749DFF1F0E9CFF1FB6
:102DB0002C89FF1F0C9EFF1FBA4A1078002840F094
:102DC0005983B94A1268D2F17F0248BF033203EB3C
:102DD000A202531CB54A23609942B8BF1160FFF6A6
:102DE0003FAF19463CE7B24B12881960002A7FF4C6
:102DF000E0AC0B469842D4BFC1EB0003C1EB030328
:102E000085E5AC4B7F3883FB0032C317C3EB62030D
:102E100003EB4303A0EB8300733032E60123CDF8CC
:102E200010B0CDF800B00593FFF7B3BA01232B60C3
:102E3000A14EA24CFFF7F1B9029B1B78FBB1A04B4E
:102E40001B88012B00F0E284022B00F06F86032B1D
:102E500001F0A580042B01F05F82052B01F0528365
:102E6000062B01F0A284072B01F00685082B01F048
:102E70004C87092B02F04A800A2B02F02882019B22
:102E80001B88002B00F06C83009B1B783BB9039BD5
:102E90001B7823B9029B1B78002B01F00080894B23
:102EA0001B78002B00F0288187490B78082B00F253
:102EB000238186483A680068854C0133DBB25F1E87
:102EC000101A44F827000B70824B3468198889F86F
:102ED0000020A142784EBFF61FAB32687E4B0892AD
:102EE000089A764C1A60FFF798B9039B1B78002B61
:102EF000A2D03B68A3F10C007F2840F36C836D489F
:102F00008B3B80FB0320DA17C2EB600000EB400034
:102F1000A3EB800303F17300DFF8D081C0B298F80F
:102F2000001005F039FD009B1B78002B84D0664C07
:102F30002378002B80D0DFF8B8A14FF0000B0CE015
:102F400003F17300C0B298F8001005F025FD237856
:102F50000BF1010B5B457FF76FAF3B685AF8040F2D
:102F6000544A1844A0F18B0382FB0321DA17C2EB09
:102F700061020C3802EB42027F28A3EB8203DFDC04
:102F8000FDF76AFBDEE74F4B1B78002B40F0EE822B
:102F90003B68524A1278002A45D0A3F10C007F28E2
:102FA00040F33383434A8B3B82FB0321DA17C2EBA6
:102FB000610202EB4202A3EB820303F17300C0B291
:102FC00098F8001005F0E8FC009B1B7853B33E4CCA
:102FD00023783BB3DFF81891DFF8D8A04FF0000B4F
:102FE0000BE003F17300C0B298F8001005F0D4FCB8
:102FF00023780BF1010B5B4514DD3B6859F8040F96
:103000001844A0F18B038AFB0321DA17C2EB61029B
:103010000C3802EB42027F28A3EB8203E1DCFDF7D0
:103020001BFBE0E73B682E4A1278FAB1244A12886B
:10303000012A00F07284022A00F07786032A01F048
:103040002F80042A01F08C81052A01F0CE82062A05
:1030500001F0D883072A01F0B484082A01F0CD8654
:10306000092A01F098870A2A02F0F980019A128849
:10307000002A00F08D821B4A104C137003232B6032
:10308000FFF7CBB8DFF86C8098F80030002B40F0E9
:103090001081154F3B78002B40F0F984074C3B70B2
:1030A000FFF7BBB8D19DFF1F849BFF1FA49BFF1F91
:1030B000809BFF1FABAAAA2AF89EFF1F4C9DFF1FF3
:1030C0003E9DFF1F809DFF1F5489FF1FA09BFF1F78
:1030D0003089FF1F289CFF1FA49EFF1F7D9BFF1FA1
:1030E0002A9CFF1F749DFF1F9A9BFF1F0E9CFF1FB2
:1030F0002C89FF1F709DFF1F3A68E5E6DBB218467A
:10310000137005F0FFFBAC4BAC491A46AC4B1846AC
:1031100000230B703B7013700370FFF70BB9DFF8DF
:10312000BC8298F80030002B40F0CF81A54F3B784F
:10313000002BB3D0A44BA54C1988A22005F088FD24
:1031400098F800303B70FFF768B80123FFF734B9F7
:1031500080249F499F4BA04A09881B8812680B4412
:10316000B2EB630FBFF66DA99C4B1B78002B40F0B0
:103170001C82B8F800309A4AA3423FF462A9994BE6
:10318000148001221A70FFF75CB9974B01931B88DA
:10319000002B42F08A818A4B0393944B0293944C08
:1031A00023786BB3DFF85C82DFF848A24FF0000BA6
:1031B00009E003F17300C0B205F016FC23780BF1AF
:1031C000010B5B451CDD58F8043F99F800001844DA
:1031D000A0F17F038AFB0321DA17C2EB610202EB45
:1031E00042027F28A3EB8203E3DCFDF735FAE2E736
:1031F0007E4B029305F0F8FB009B1B78002BCED191
:10320000039B1B78002B3FF4B4AC99F80030A3F17A
:103210000C007F2840F3ED8176488B3B80FB032038
:10322000DA17C2EB600000EB4000A3EB800303F170
:103230007300C0B205F0D8FB009B1B78002B00F098
:10324000CD816B4C2378002B01F0C082DFF8B48174
:10325000DFF8A0A14FF0000B0AE003F17300C0B249
:1032600005F0C2FB23780BF1010B5B457FF781ACC6
:1032700058F8043F99F800001844A0F18B038AFB2A
:103280000321DA17C2EB61020C3802EB42027F28FD
:10329000A3EB8203E1DCFDF7DFF9E0E7FDF7DCF902
:1032A000A5E45046FDF7D8F94CE4FDF7D5F9FFF752
:1032B00097BA514A1278002A40F0D581414F434CC9
:1032C0003B70FEF7AABF002008704C49087840B157
:1032D000394900910978002900F0B581009F00214B
:1032E00039704749097800297FF4F0A8002C40F094
:1032F000CE80002840F0CB80384C2F4F94F800E06F
:103300002F4C0394394C02942D4C2C492070374C8F
:103310000097087038702070BEF1000F7FF4E8A8A5
:10332000FFF7EFB8264B1B78002B6DD099F80030D3
:10333000A3F10C007F2840F3CC832E4A8B3B82FB09
:103340000321DA17C2EB610202EB4202A3EB820314
:1033500003F17300C0B205F047FB009B1B78002B04
:1033600052D0234C2378002B4ED0264FDFF8848098
:103370004FF0000A09E003F17300C0B205F034FB1E
:1033800023780AF1010A53453EDD57F8043F99F8C6
:1033900000001844A0F18B0388FB0321DA17C2EB6D
:1033A00061020C3802EB42027F28A3EB8203E2DCCD
:1033B000FDF752F9E1E700BFD09DFF1F809DFF1F81
:1033C0007D9BFF1F9A9BFF1FC29DFF1F4C9DFF1FF0
:1033D000349DFF1F309DFF1FCC9BFF1F709DFF1F63
:1033E000C09DFF1F9E9BFF1FD09BFF1F2A9CFF1F9E
:1033F0005489FF1FABAAAA2AC69DFF1F109EFF1F5C
:103400000C9EFF1F2C89FF1FA84B1B78FBB1A84BFC
:103410001B88012B00F0D486022B00F0CF87032BF2
:1034200001F04A81042B01F0E481052B01F01B849B
:10343000062B01F0DA84072B01F01F86082B01F020
:10344000DD86092B01F0C9870A2B01F0A687019BB5
:103450001B88002B00F0EC82964B1B78002B40F071
:10346000E282954B954A1988346800200123106048
:103470002B602EE50130C0B2022886BF00211170FA
:1034800010701946FFF7ECBB0398002101708C49BE
:10349000097800293FF435A8844902910978002968
:1034A00000F0B287029800210170FFF72AB8039B51
:1034B0001B78002B7FF485AB029B1B78002B7FF4DD
:1034C00080AB019B1988FFF782BB7E4A1278002AE5
:1034D0003FF4F4AE7C4F387802F028FD7B4B1B782C
:1034E000002B00F0BB8439887E2900F2B784784C29
:1034F000DFF80C922368D9F800209B1A0F2B40F2BA
:103500009680744B01311B8889B239802BB1052B11
:1035100003D0C9B2052005F017FA6F4F226898F85A
:103520000030C9F800203B70FEF777BE243B002B2B
:10353000B8F8000040F3788498423EF45AAF9BB24A
:103540006648A8F8003001230370FEF752BFDFF889
:103550009081C0B298F8001005F01EFAFFF74BBB3F
:103560005F4B3878197805F017FA8DE47F214020F9
:1035700005F0EAF95B495C4A3B680B600021117079
:1035800007E5C0B298F8001005F006FAFFF72FB96A
:10359000D8B298F8001005F0FFF93B686BE5534B83
:1035A000DFF860E11978FEF724BF4B2C40F34C8222
:1035B0001834802CB8F800304D4AA8BF8024A342AC
:1035C0007FF4DDADFEF73DBF99F8000005F00CFA81
:1035D0002188FFF7FCBAFDF73FF89DE4029B1B78BA
:1035E000002B7FF4C9AA039B1B78002B7FF4E9AA68
:1035F00067E7FDF731F81CE63E4B01931B88002B73
:103600007FF4F6AD294B0293FFE5FDF725F8D6E4EC
:10361000FDF722F8FFF7D3B90132D2B2022A40F205
:103620005E82002202701946FFF71ABB284C2A4F0F
:1036300098F800303B70FEF7F0BD7F20FFF76CBAC2
:103640007F20FFF798B9194F1A4902974FF0000CE5
:1036500081F800C0009F02994FF0010E87F800E04A
:1036600081F800C03DE6244F387802F05FFC174B2C
:103670001B78002B00F03A8239887E2900F23682CE
:10368000134CDFF87C902368D9F800209B1A0F2B8D
:10369000CDD91A4B0131188889B23980002800F041
:1036A0004182C9B2C0B205F04FF936E72A9CFF1F2C
:1036B0003E9DFF1F809DFF1F289CFF1F809BFF1FBB
:1036C000709DFF1FC69DFF1FC29DFF1F119EFF1F04
:1036D0004C9DFF1F2E9CFF1F9A9BFF1F9E9BFF1F51
:1036E0000E9CFF1FA09BFF1F5489FF1FEF9DFF1F14
:1036F000C09DFF1FD09BFF1FCA9BFF1F049CFF1F85
:10370000FC9DFF1FE19BFF1FDFF8B4A399F80000A9
:10371000BAF80030E34AE44CC31A82FB031ED917FF
:10372000C1EB6E0101EB4101A3EB810303EB43030A
:1037300054F8233018447F2840F3AE847F3882FB4E
:103740000032C317C3EB620303EB4303A0EB830018
:103750007330DFF870B3C0B205F046F9BBF8003043
:10376000022B7FF629AA99F80010BAF80030CD4A4A
:10377000CB1A82FB030ED817C0EB6E0000EB4000A3
:10378000A3EB800303EB430304EB83035868084473
:103790007F2840F320877F3882FB0032C317C3EBBA
:1037A000620202EB4202A0EB82007330C0B205F06D
:1037B0001BF9BBF80030032B7FF6FEA999F8001027
:1037C000BAF80030B74ACB1A82FB030ED817C0EB09
:1037D0006E0000EB4000A3EB800303EB430304EB1C
:1037E0008304A06808447F2840F370817F3882FBFF
:1037F0000032C317C3EB620202EB4202A0EB82006D
:103800007330C0B205F0F0F8FFF7D6B9DFF8B0A218
:103810003868BAF80030A34AA34CC31A82FB031ECF
:10382000D917C1EB6E0101EB4101A3EB810303EB5F
:10383000430354F8233018447F2840F329847F3809
:1038400082FB0032C317C3EB620303EB4303A0EB1D
:1038500083007330DFF87082DFF868B298F80010E8
:10386000C0B205F099F8BBF80030022B7FF607AB29
:103870003968BAF800308B4ACB1A82FB030ED8178E
:10388000C0EB6E0000EB4000A3EB800303EB4303AF
:1038900004EB8303586808447F2840F398867F38F8
:1038A00082FB0032C317C3EB620202EB4202A0EBC1
:1038B00082007330C0B298F8001005F06DF8BBF8C4
:1038C0000030032B7FF6DBAA3968BAF80030754A5E
:1038D000CB1A82FB030ED817C0EB6E0000EB400042
:1038E000A3EB800303EB430304EB8304A0680844C9
:1038F0007F2840F3F8807F3882FB0032C317C3EB88
:10390000620202EB4202A0EB8200733098F80010D2
:10391000C0B205F041F8FFF7B2BADFF8A4A16149DF
:10392000BAF80020604C9A1A81FB020ED017C0EB47
:103930006E0000EB4000A2EB800202EB420254F862
:10394000220018447F2840F32284A0F17F0381FBEA
:103950000321DA17C2EB610000EB4000A3EB80000B
:103960007330DFF860B198F80010C0B205F014F8B9
:10397000BBF80030022B50D93968BAF80030494AF8
:10398000CB1A82FB030ED817C0EB6E0000EB400091
:10399000A3EB800303EB430304EB83035868084461
:1039A0007F2840F385867F3882FB0032C317C3EB44
:1039B000620202EB4202A0EB82007330C0B298F8C0
:1039C000001004F0E9FFBBF80030032B25D938685C
:1039D000BAF80030334AC31A82FB031ED917C1EB71
:1039E0006E0101EB4101A3EB810303EB430304EB05
:1039F0008304A36818447F286EDD7F3882FB003281
:103A0000C317C3EB620202EB4202A0EB82007330E9
:103A1000C0B298F8001004F0BFFF3B68FFF726BB68
:103A20000120FFF779B80021402004F08DFF18E550
:103A300099F8000004F0D8FF0EE504F0D5FFFEF77A
:103A4000C7BF0120FEF797BF243C002CB8F8003018
:103A500040F3C585A3423EF4F4ACA4B2134BA8F8DE
:103A6000004001221A70FEF7ECBC114B01931B8839
:103A7000002B7FF4BFABFFF77CB80E498342A8BF91
:103A800003460B60FEF795BE1446FFF76DBB0A4B6D
:103A90000A4C19886A2005F0DBF898F800303B7072
:103AA000FEF7BBBBABAAAA2A701601009E9BFF1FA4
:103AB000D09BFF1F809BFF1FCA9BFF1F4C9DFF1FBA
:103AC0007C9DFF1FB09BFF1F0E9CFF1FFCF7C4FDDA
:103AD00097E6FCF7C1FD3DE4FCF7BEFD98E70270F8
:103AE0001946FFF7BDB8FCF7B7FD0FE7D14B1B78C0
:103AF000002B3FF49BAD3B88CF4F002B3FF496AD9E
:103B0000CE4CDFF848932268D9F80010521A0F2AD9
:103B10007FF68DADCA4A013B108899B239800028E2
:103B20007FF4BFADC8B204F083FFF6E4DFF820A352
:103B30003868BAF80030C34AC34CC31A82FB031E6C
:103B4000D917C1EB6E0101EB4101A3EB810303EB3C
:103B5000430354F8233018447F2840F325847F38EA
:103B600082FB0032C317C3EB620303EB4303A0EBFA
:103B700083007330DFF8DC82DFF8DCB298F80010E5
:103B8000C0B204F009FFBBF80030022B7FF677A922
:103B90003968BAF80030AB4ACB1A82FB030ED8174B
:103BA000C0EB6E0000EB4000A3EB800303EB43038C
:103BB00004EB8303586808447F2840F30E867F385F
:103BC00082FB0032C317C3EB620303EB4303A0EB9A
:103BD00083007330C0B298F8001004F0DDFEBBF82B
:103BE0000030032B7FF64BA93868BAF80030954AAD
:103BF000C31A82FB031ED917C1EB6E0101EB410111
:103C0000A3EB810303EB430304EB8304A368184491
:103C10007F287FF768AF7F3882FB0032C317C3EB82
:103C2000620303EB4303A0EB830073306EE6DFF81F
:103C300020A299F80000BAF80030824A824CC31AD8
:103C400082FB031ED917C1EB6E0101EB4101A3EB0F
:103C5000810303EB430354F8233018447F2840F3D7
:103C6000A7837F3882FB0032C317C3EB620303EBE9
:103C70004303A0EB83007330DFF8DCB1C0B204F083
:103C8000B3FEBBF80030022B7EF696AF99F8001019
:103C9000BAF800306B4ACB1A82FB030ED817C0EB80
:103CA0006E0000EB4000A3EB800303EB430304EB47
:103CB0008303586808447F2840F393857F3882FB4C
:103CC0000032C317C3EB620303EB4303A0EB830093
:103CD0007330C0B204F088FEBBF80030032B7EF6D0
:103CE0006BAF99F80010BAF80030564ACB1A82FB35
:103CF000030ED817C0EB6E0000EB4000A3EB80036F
:103D000003EB430304EB8304A06808447F287FF798
:103D1000DDAE7F3882FB0032C317C3EB620303EBD7
:103D20004303A0EB830073306BE5DFF824A1454922
:103D3000BAF80020444C9A1A81FB020ED017C0EB4F
:103D40006E0000EB4000A2EB800202EB420254F84E
:103D5000220018447F2840F32E83A0F17F0381FBCB
:103D60000321DA17C2EB610000EB4000A3EB8000F7
:103D70007330DFF8E4B098F80010C0B204F00CFE25
:103D8000BBF80030022B7FF648AE3968BAF8003035
:103D90002C4ACB1A82FB030ED817C0EB6E0000EB47
:103DA0004000A3EB800303EB430304EB8303586859
:103DB00008447F2840F319857F3882FB0032C317FF
:103DC000C3EB620303EB4303A0EB83007330C0B289
:103DD00098F8001004F0E0FDBBF80030032B7FF6EC
:103DE0001CAE3868BAF80030164AC31A82FB031EAC
:103DF000D917C1EB6E0101EB4101A3EB810303EB8A
:103E0000430304EB8304A36818447F287FF764AE60
:103E10007F3882FB0032C317C3EB620303EB43031B
:103E2000A0EB83007330F3E501283EF4E2AA0123FE
:103E3000FFF786BB109EFF1FCA9BFF1F4C9DFF1FF5
:103E4000049CFF1FABAAAA2A6C170100FC9DFF1F50
:103E50007C9DFF1F0E9CFF1FB09BFF1FCE4B1B784E
:103E6000002B3FF4E3AB3B88CC48002B3FF4DEABA8
:103E7000CB4CDFF83C932268D9F80010521A0F2A75
:103E80007FF6D5ABC74A013B128899B20180002A60
:103E90003FF443AB052A7FF43CABFFF73EBB4FF446
:103EA0007A43013BFDD199F8000004F09DFDFEF737
:103EB000F6BFDFF800A399F80000BAF80030BA4A5C
:103EC000BA4CC31A82FB031ED917C1EB6E0101EB7A
:103ED0004101A3EB810303EB430354F8233018445F
:103EE0007F2840F3E8817F3882FB0032C317C3EBA1
:103EF000620202EB4202A0EB82007330DFF8B8B23C
:103F0000C0B204F071FDBBF80030022B7EF654AE57
:103F100099F80000BAF80030A34AC31A82FB0321C3
:103F2000DA17C2EB610202EB4202A3EB820303EB5E
:103F3000430304EB83035B6818447F2840F31F842A
:103F40007F380C2290FBF2F302FB13007330C0B2F7
:103F500004F04AFDBBF80030032B7EF62DAE99F835
:103F60000000BAF80030904AC31A82FB0321DA1726
:103F7000C2EB610202EB4202A3EB820303EB4303B9
:103F800004EB8304A36818447F287FF79FAD7F3834
:103F90000C2290FBF2F302FB1300733031E4DFF8E4
:103FA00014A23868BAF800307F4A804CC31A82FBEA
:103FB000031ED917C1EB6E0101EB4101A3EB810395
:103FC00003EB430354F8233018447F2840F37081F7
:103FD0007F3882FB0032C317C3EB620202EB42025E
:103FE000A0EB82007330DFF8D481DFF8CCB198F811
:103FF0000010C0B204F0D0FCBBF80030022B7EF6FB
:104000003EAF3868BAF80030674AC31A82FB032112
:10401000DA17C2EB610202EB4202A3EB820303EB6D
:10402000430304EB83035B6818447F2840F3AB83AE
:104030007F380C2290FBF2F302FB13007330C0B206
:1040400098F8001004F0A8FCBBF80030032B7EF6B3
:1040500016AF3868BAF80030534AC31A82FB0321FE
:10406000DA17C2EB610202EB4202A3EB820303EB1D
:10407000430304EB8304A36818447F287FF733AD20
:104080007F380C2290FBF2F302FB130073303DE407
:10409000FCF7E2FAFFF7DEBBFCF7DEFAFFF759BBED
:1040A000DFF810A14049BAF80020404C9A1A81FB71
:1040B000020ED017C0EB6E0000EB4000A2EB8002B6
:1040C00002EB420254F8220018447F2840F3F680A5
:1040D000A0F17F0381FB0321DA17C2EB610101EB41
:1040E0004101A3EB81007330DFF8CCB098F80010E9
:1040F000C0B204F051FCBBF80030022B7FF68DAC4F
:104100003868BAF80030284AC31A82FB0321DA174C
:10411000C2EB610202EB4202A3EB820303EB430317
:1041200004EB83035B6818447F2840F338837F38AF
:104130000C2290FBF2F302FB13007330C0B298F82C
:10414000001004F029FCBBF80030032B7FF665ACAF
:104150003868BAF80030144AC31A82FB0321DA1710
:10416000C2EB610202EB4202A3EB820303EB4303C7
:1041700004EB8304A36818447F287FF7ADAC7F3835
:104180000C2290FBF2F302FB1300733040E4FCF7C7
:1041900063FAFFF7E6BB00BF109EFF1FC29DFF1F23
:1041A0004C9DFF1F2E9CFF1FABAAAA2AFC170100E3
:1041B000FC9DFF1F7C9DFF1FB09BFF1F0E9CFF1FE0
:1041C000DFF838A399F80000BAF80030C34AC44CAD
:1041D000C31A82FB0317D917C1EB670101EB410139
:1041E000A3EB810303EB430354F8233018447F28E7
:1041F0006ADD7F3882FB0032C317C3EB620202EB39
:104200004202A0EB82007330DFF8F4B2C0B204F0D7
:10421000EBFBBBF80030022B7FF619A999F80000E0
:10422000BAF80030AD4AC31A82FB0321DA17C2EB99
:10423000610202EB4202A3EB820303EB430304EBB4
:1042400083035B6818447F2840F3AC827F380C22DC
:1042500090FBF2F302FB13007330C0B204F0C4FB16
:10426000BBF80030032B7FF6F2A899F80000BAF8EB
:1042700000309A4AC31A82FB0321DA17C2EB6102AB
:1042800002EB4202A3EB820303EB430304EB830440
:10429000A36818447F2814DD7F380C2290FBF2F3CA
:1042A00002FB13007330C0B204F09EFBFFF7CFB8DF
:1042B000FCF7D2F997E6FCF7CFF91FE6FCF7CCF94B
:1042C00012E7FCF7C9F9EEE7FCF7C6F99CE7DFF85F
:1042D0002CA299F80000BAF80030804A814CC31A29
:1042E00082FB031ED917C1EB6E0101EB4101A3EB69
:1042F000810303EB430354F8233018447F28DADDAD
:104300007F3882FB0032C317C3EB620303EB430326
:10431000A0EB83007330F1E5DFF8E0A13868BAF86C
:1043200000306E4A6F4CC31A82FB031ED917C1EBD3
:104330006E0101EB4101A3EB810303EB430354F84E
:10434000233018447F28B3DD7F3882FB0032C31747
:10435000C3EB620303EB4303A0EB8300733042E63D
:10436000DFF898A15D49BAF800205E4C9A1A81FBEB
:10437000020ED017C0EB6E0000EB4000A2EB8002F3
:1043800002EB420254F8220018447F2896DDA0F187
:104390007F0381FB0321DA17C2EB610000EB4000D1
:1043A000A3EB800073309FE6FCF756F9FFF7E2BB02
:1043B000FCF752F960E4FCF74FF9DAE4DFF83CA1CE
:1043C00099F80000BAF80030444A474CC31A82FBFF
:1043D0000317D917C1EB670101EB4101A3EB81037F
:1043E00003EB430354F8233018447F287FF76CAF66
:1043F0007F3882FB0032C317C3EB620303EB430336
:10440000A0EB83007330FFE6384800903848394904
:104410000390FEF76DB8DFF8E4A099F80000BAF851
:1044200000302E4A344CC31A82FB0321DA17C2EB48
:10443000610202EB4202A3EB820303EB430354F855
:10444000233018447F2840F3A7817F380C2290FB4B
:10445000F2F302FB13007330DFF8A4B0C0B204F033
:10446000C3FABBF80030022B19D999F80000BAF84A
:1044700000300C22C11A91FBF2F302FB131302FB72
:1044800003435B6818447F2840F385847F3890FBA2
:10449000F2F302FB13007330C0B204F0A5FABBF8CC
:1044A0000030032B7EF688ABBAF8003099F8000094
:1044B0000C22C11A91FBF2F302FB131302FB03441B
:1044C000A36818447F287FF701AB7F3890FBF2F395
:1044D00002FB13007330FFF794B900BFABAAAA2AFE
:1044E00070160100DC1901006C170100D09DFF1F40
:1044F0007D9BFF1F809DFF1F341B01007C9DFF1FC4
:10450000B09BFF1FDFF864A33868BAF80030CE4ACA
:10451000CE4CC31A82FB0321DA17C2EB610202EB15
:104520004202A3EB820303EB430354F82330184405
:104530007F2840F32E817F380C2290FBF2F302FBA0
:1045400013007330DFF82883DFF828B398F80010E1
:10455000C0B204F021FABBF80030022B1AD9386837
:10456000BAF800300C22C11A91FBF2F302FB1313CC
:1045700002FB03435B6818447F2840F3C3837F3802
:1045800090FBF2F302FB13007330C0B298F80010F6
:1045900004F002FABBF80030032B7EF670ACBAF8D8
:1045A000003038680C22C11A91FBF2F302FB13139E
:1045B00002FB0344A36818447F287FF794AA7F383E
:1045C00090FBF2F302FB13007330FFF79FB9FCF787
:1045D00043F8FFF76FB9FCF73FF8FFF7E7B8012B97
:1045E0003DF42FAF0124FFF739BADFF880A29649D6
:1045F000BAF80020954C9A1A81FB0210D117C1EB32
:10460000600101EB4101A2EB810202EB420254F88E
:10461000220018447F2840F3B980A0F17F030C20CA
:1046200093FBF0F200FB12307330DFF848B298F8D9
:104630000010C0B204F0B0F9BBF80030022B1AD958
:104640003868BAF800300C22C11A91FBF2F302FB71
:10465000131302FB03435B6818447F2840F34F8326
:104660007F3890FBF2F302FB13007330C0B298F86E
:10467000001004F091F9BBF80030032B7FF6CDA9B0
:10468000BAF8003038680C22C11A91FBF2F302FB31
:10469000131302FB0344A36818447F287FF71CAA66
:1046A0007F3890FBF2F302FB13007330FFF7B0B9D1
:1046B000FBF7D2FFFFF782B9DFF8B0A199F800004D
:1046C000BAF80030604A624CC31A82FB0321DA1741
:1046D000C2EB610202EB4202A3EB820303EB430352
:1046E00054F8233018447F2846DD7F380C2290FB95
:1046F000F2F302FB13007330DFF878B1C0B204F0BC
:1047000073F9BBF80030022B19D999F80000BAF8F8
:1047100000300C22C11A91FBF2F302FB131302FBCF
:1047200003435B6818447F2840F38B807F3890FBFD
:10473000F2F302FB13007330C0B204F055F9BBF87A
:104740000030032B7EF683AEBAF8003099F80000F3
:104750000C22C11A91FBF2F302FB131302FB034478
:10476000A36818447F287FF7ACAD7F3890FBF2F345
:1047700002FB1300733096E5FBF76EFFBCE7FBF717
:104780006BFFFFF7E4BBFBF767FF58E4FBF764FF41
:104790004BE7FBF761FFD5E6FBF75EFF5CE6FBF757
:1047A0005BFFCBE4FBF758FF57E5DFF8C0A03868A4
:1047B000BAF80030244A274CABE6DFF8B0A099F8ED
:1047C0000000BAF80030204A224C2CE6029B1B78ED
:1047D000002B7EF4D1A9FEF7F4B9FBF73DFFFFF7FC
:1047E000F9B9FBF739FFFFF774BAFBF735FFFFF7AD
:1047F000EEBADFF878A099F80000BAF80030124A53
:10480000154C61E7DFF864A00F49BAF80020114C9D
:10481000F1E6124B1B78002B00F0C182104B1B7885
:10482000002B7DF40EAE0F4B1B78002B3DF409AE30
:10483000B8F800300C490A33A8F800300A70FDF7C8
:1048400000BEFBF709FF77E7ABAAAA2A341B0100D9
:10485000FC1701004C190100DC1901000D9EFF1F1F
:104860000E9EFF1F0F9EFF1F9E9BFF1F7C9DFF1F25
:104870000E9CFF1FB09BFF1FA44C2388002B40F011
:10488000BE83DFF8A0B2A249A24A0988D7F8008007
:10489000B2F800E0A048C1EB080C0C229CFBF2F13E
:1048A00002FB11C14FF0900C0CFB0EFE02FB01E16C
:1048B0006FF00B0E405880440EFB03807F2840F3BE
:1048C0000285A0F17F0393FBF2F002FB10307330FE
:1048D000924BC0B2197804F05FF8BBF8002023882F
:1048E0001344022B23DD8A4A8A4B11883868B3F8B7
:1048F00000C0DFF824E2411A0C2291FBF2F302FB24
:104900001311902303FB0CF302FB013373445B6828
:1049100018447F2840F3AD857F3890FBF2F302FB0B
:10492000130073307D4BC0B2197804F035F8BBF832
:10493000002023881344032B23DD754A754B11880F
:104940003868B3F800C0DFF8D0E1411A0C2291FBBF
:10495000F2F302FB1311902303FB0CF302FB013370
:1049600073449B6818447F2840F35D857F3890FB33
:10497000F2F302FB13007330684BC0B2197804F0F5
:104980000BF8BBF8002023881344042B7EF777AA8A
:10499000634B1B88012B7EF472AA3A68A2F10C00CB
:1049A0007F2840F38F828B3A0C2092FBF0F300FBC0
:1049B00013207330594BC0B2197803F0EDFFFEF7A6
:1049C0005EBA524C2288002A00F0D7825449DFF8A0
:1049D00054B10988BBF800000331884227DD4C48F8
:1049E0004C490088B1F800E0DFF82CC1181A0C21FE
:1049F00090FBF1F901FB19004FF0900909FB0EFE45
:104A000001FB00E06FF00B0E5CF8000003440EFBAE
:104A100002307F2840F3B7847F3890FBF1F301FB2D
:104A200013007330C0B298F8001003F0B5FFBBF864
:104A3000002023881344022B23DD354B354A386888
:104A40001B88B2F800C0DFF8D0E0C31A0C2193FB3A
:104A5000F1F201FB1232902303FB0CF301FB023352
:104A600073445B6818447F2840F3E4847F3890FBEC
:104A7000F1F301FB13007330C0B298F8001003F09B
:104A80008BFFBBF8002023881344032B23DD204B2E
:104A9000204A38681B88B2F800C0DFF87CE0C31AEF
:104AA0000C2193FBF1F201FB1232902303FB0CF378
:104AB00001FB023373449B6818447F2840F3C18490
:104AC0007F3890FBF1F301FB13007330C0B298F80C
:104AD000001003F061FFBBF8002023881344042B6F
:104AE0007EF79BAF0E4B1B88012B7EF496AF3A6886
:104AF000A2F10C007F287EF7EFAF8B3A0C2092FBDF
:104B0000F0F300FB13207330FEF782BF109CFF1FF1
:104B10007C9DFF1F2A9DFF1FE01201000E9CFF1FBE
:104B2000EA9BFF1FB09BFF1FCE4C2388002B40F059
:104B30002782DFF864B3CC49CC4A098899F8000091
:104B4000B2F800E0DFF85483C1EB000C0C229CFBB0
:104B5000F2F102FB11C14FF0900C0CFB0EFE02FBB8
:104B600001E16FF00B0E58F8011008440EFB030032
:104B70007F2840F30484A0F17F0393FBF2F002FB53
:104B800010307330C0B203F02FFFBBF80020238831
:104B90001344022B22DDB44AB44B118899F800006B
:104BA000B3F800C0DFF8F4E2411A0C2291FBF2F3F3
:104BB00002FB1311902303FB0CF302FB013373443C
:104BC0005B6818447F2840F3E5837F3890FBF2F35D
:104BD00002FB13007330C0B203F006FFBBF80020E5
:104BE00023881344032B22DD9F4AA04B118899F898
:104BF0000000B3F800C0DFF8A4E2411A0C2291FBD8
:104C0000F2F302FB1311902303FB0CF302FB0133BD
:104C100073449B6818447F2840F302847F3890FBDC
:104C2000F2F302FB13007330C0B203F0DDFEBBF8F9
:104C3000002023881344042B7DF7BEAF8C4B1B88C8
:104C4000012B7DF4B9AF99F80020A2F10C007F2868
:104C50007EF73CAF8B3A0C2092FBF0F300FB132065
:104C60007330FEF7CEBDDFF800A299F80000BAF865
:104C70000030804CC11A0C2291FBF2F302FB13139B
:104C800002FB03F3E35818447F287FF775AD7F38A4
:104C900090FBF2F302FB130073302DE5764B1B887B
:104CA000182B12D099F800201344A3F118007F2884
:104CB00040F3DC830C20973B93FBF0F200FB1233B4
:104CC00003F17300C0B203F08FFE6C4A6C4B127894
:104CD00033F81230182B3DF46FAF99F800201344CD
:104CE000A3F118007F287EF7F1AE0C20973B93FBD1
:104CF000F0F200FB123303F17300FEF782BDFBF705
:104D0000ABFCB3E4FBF7A8FC3FE45B4B1A88182A22
:104D100013D03B681344A3F118007F2840F37D8330
:104D20000C20973B93FBF0F200FB123303F173006E
:104D3000544BC0B2197803F02FFE504B50491A78EB
:104D4000022A94BF013200221A701A7831F8120038
:104D5000182810D10424022A02F10100C2B288BF2F
:104D6000002231F81200182804D1013CF3D11A7046
:104D7000FEF785B81A703B680344A3F118007F283A
:104D800040F3A0800C20973B93FBF0F200FB123322
:104D900003F173000EE6FBF75FFCFFF77DBB3A4BB8
:104DA0001B78002B7DF486AF384B1B78002B3DF42D
:104DB00048ABB8F8003036490133A8F800300A7023
:104DC000FDF73FBB304B1B78002B7DF43AAB2F4BEC
:104DD0001B78002B3DF435ABB8F800302C49013B73
:104DE000A8F800300A70FDF72CBBDFF87CA099F81A
:104DF0000000BAF80030274C3CE71F4A1288182AF6
:104E000012D01344A3F118007F2840F3C0820C2075
:104E1000973B93FBF0F200FB123303F17300C0B237
:104E200098F8001003F0B8FD144B15491A78022ABF
:104E300094BF013200221A701A7831F81200182833
:104E40002FD10424022A02F10100C2B288BF00223D
:104E500031F81200182823D1013CF3D11A703B68B5
:104E6000FEF704B9109CFF1F7C9DFF1F2A9DFF1FAA
:104E7000EA9BFF1F341B0100BA9BFF1F0F9CFF1F03
:104E8000989DFF1F0E9CFF1F0E9EFF1F0F9EFF1F72
:104E90009E9BFF1F4C190100B09BFF1FE0120100F9
:104EA0001A703B680344A3F118007F287EF714AE04
:104EB0000C20973B93FBF0F200FB123303F17300DD
:104EC000FEF7A6BDFBF7C8FB74E5BF4B1B88182B8C
:104ED00012D099F800201344A3F118007F2840F362
:104EE000AD820C20973B93FBF0F200FB123303F1F1
:104EF0007300C0B203F078FDB44AB54B127833F8B2
:104F00001230182B7FF4E9AEFDF756BEAE4B1A886F
:104F1000182A13D03B681344A3F118007F2840F3EC
:104F200086820C20973B93FBF0F200FB123303F1D7
:104F30007300A84BC0B2197803F02EFDA34BA4490F
:104F40001A78022A94BF013200221A701A7831F8B6
:104F5000120018287FF40FAF0424022A02F1010284
:104F600094BFD2B2002231F8120018287FF402AFA9
:104F7000013CF2D11A70FDF782BFDFF87CB22EE55A
:104F8000954ADFF874B21288BBF8001003329142E0
:104F90007FF7FBADCFE58C4A1288182A12D0134454
:104FA000A3F118007F2840F35E820C20973B93FB0F
:104FB000F0F200FB123303F17300C0B298F8001056
:104FC00003F0EAFC814B82491A78022A94BF01322D
:104FD00000221A701A7831F8120018287FF461AF95
:104FE0000424022A02F1010294BFD2B2002231F855
:104FF000120018287FF454AF013CF2D12EE7764A14
:10500000DFF8F4B11288BBF80010033291427FF749
:1050100064AC38E4714B01227F2107201A8003F031
:1050200093FC7F210B2003F08FFCFDF76EBE6C4BD1
:1050300004227F2107201A8003F086FC00210B2028
:1050400003F082FCFDF75ABE654B02227F21072048
:105050001A8003F079FC7F210B2003F075FCFDF72B
:1050600048BE5F4B002107201C8003F06DFC7F21B0
:105070000B2003F069FCFDF737BE5A4C2388002B48
:1050800040F0E681DFF870B1574999F80000574ABF
:1050900009881788DFF858E1411A0C2291FBF2FCCD
:1050A00002FB1C114FF0900C0CFB07F702FB017187
:1050B0006FF00B075EF80110014407FB03107F2817
:1050C00040F3C3817F3890FBF2F302FB130073308F
:1050D000C0B203F089FCBBF8002023881344022BE4
:1050E00021DD414B414A99F800001B88B2F800E0ED
:1050F0003F4FC31A0C2193FBF1F201FB12329023B4
:1051000003FB0EF301FB02333B445B6818447F282A
:1051100040F3C8817F3890FBF1F301FB130073303B
:10512000C0B203F061FCBBF8002023881344032BBA
:1051300021DD2D4B2D4A99F800001B88B2F800E0C4
:105140002B4FC31A0C2193FBF1F201FB1232902377
:1051500003FB0EF301FB02333B449B6818447F289A
:1051600040F39D817F3890FBF1F301FB1300733016
:10517000C0B203F039FCBBF8002023881344042B91
:105180007EF765A9144B1B88012B7EF460A999F862
:105190000020A2F10C007F287FF793A88B3A0C2007
:1051A00092FBF0F300FB13207330FFF77CB8114B38
:1051B00000227F2107201A8003F0C6FB7F210B20ED
:1051C00003F0C2FBFDF7A9BDC29BFF1F0F9CFF1F91
:1051D000109DFF1F0E9CFF1FEA9BFF1F1E9CFF1FC1
:1051E000729DFF1F109CFF1F7C9DFF1F2A9DFF1FAC
:1051F000E01201009C9BFF1FB09BFF1FB04B1B8860
:10520000182B12D099F800201344A3F118007F281E
:1052100040F33C810C20973B93FBF0F200FB1233F0
:1052200003F17300C0B203F0DFFBA64AA64B12786D
:1052300033F81230182B3EF40AA999F800201344D1
:10524000A3F118007F287FF73CA80C20973B93FB25
:10525000F0F200FB123303F17300FFF724B89B4A0E
:105260001288182A12D01344A3F118007F2840F3A3
:1052700007810C20973B93FBF0F200FB123303F104
:105280007300C0B298F8001003F086FB8D4B904974
:105290001A78022A94BF013200221A701A7831F863
:1052A000120018287FF4FDAD0424022A02F1010245
:1052B00094BFD2B2002231F8120018287FF4F0AD6A
:1052C000013CF2D1CAE5FBF7C7F9FFF701BB7F4B01
:1052D0001A88182A13D03B681344A3F118007F28BA
:1052E00040F3DA800C20973B93FBF0F200FB123383
:1052F00003F17300774BC0B2197803F04DFB714B8B
:1053000073491A78022A94BF013200221A701A785F
:1053100031F8120018287FF42EAD0424022A02F17D
:10532000010294BFD2B2002231F8120018287FF493
:1053300021AD013CF2D11A70FDF7A1BD634B1B8872
:10534000182B12D099F800201344A3F118007F28DD
:1053500040F393800C20973B93FBF0F200FB123359
:1053600003F17300C0B203F03FFB564A584B12786A
:1053700033F81230182B7FF4B0ACFDF71DBCFBF7EF
:105380006BF9FFF7FFBBFBF767F9FFF74BBBFBF7C9
:1053900063F944E5FBF760F91DE44C4B1B88182BBF
:1053A00011D099F800201344A3F118007F286ADD7A
:1053B0000C20973B93FBF0F200FB123303F17300D8
:1053C000C0B203F011FB3F4A414B127833F8123060
:1053D000182B7FF432AFFEF73AB83F4B1B88182BDF
:1053E00011D099F800201344A3F118007F2850DD54
:1053F0000C20973B93FBF0F200FB123303F1730098
:10540000C0B203F0F1FA2F4A344B127833F812305D
:10541000182B7FF412AFFEF71AB8FBF71DF987E4DB
:10542000FBF71AF900E4FBF717F9FFF7A5BAFBF74A
:1054300013F97EE5FBF710F9FFF71EBBFBF70CF93C
:1054400057E5FBF709F9FFF741BBFBF705F93FE625
:10545000234ADFF898B01288BBF80010033291425B
:105460007FF739AE10E6FBF7F7F8A6E5FBF7F4F89F
:1054700028E4FBF7F1F8FFF755BAFBF7EDF871E711
:10548000FBF7EAF8FDE6FBF7E7F899E7FBF7E4F846
:10549000C8E6FBF7E1F8B3E7FBF7DEF82AE7FBF72E
:1054A000DBF865E6FBF7D8F83AE60E4B03930E4BB4
:1054B0000293FDF79FBE23601946FDF7D1BB00BFE5
:1054C000BA9BFF1F0F9CFF1F989DFF1FC49BFF1FD0
:1054D000189DFF1F0E9CFF1FC29BFF1F109DFF1FEB
:1054E000EA9BFF1F7D9BFF1F2A9CFF1FB09BFF1F96
:1054F00038B507F0A3F90B4805F0DAF800234FF0B0
:105500007E5201210848FAF7B1FF084B084A0949C1
:10551000802400251C7118461D60BDE838400AF043
:1055200051BE00BF1C9CFF1F509DFF1FD49DFF1F3D
:105530001C89FF1FFD05000010B50446A420636808
:10554000198803F085FBE368A6201988BDE81040A0
:1055500003F07EBB43682A20198803F079BB00BFA3
:1055600010B5044622206368198803F071FBE368D4
:1055700024201988BDE8104003F06ABB10B504462A
:105580000A206368198803F063FBE3680C2019881C
:10559000BDE8104003F05CBB10B50446062063680C
:1055A000198803F055FBE36808201988BDE810400E
:1055B00003F04EBB10B5044602206368198803F05F
:1055C00047FBE36804201988BDE8104003F040BBA6
:1055D00070B50E4C84B012250422012306460390B8
:1055E000029320468DE824001423102106F064FA6B
:1055F0000622092302930396019520460092142364
:10560000102106F059FA04B070BD00BF409EFF1F84
:105610002DE9F041224D82B0012602B284B20092FF
:10562000284601967823192106F08CF904F10C0222
:1056300012B28DE844002846A7197823192104F1F5
:10564000020806F07FF93FB20FFA88F819233A46AC
:10565000284619460196CDF8008006F073F97823A4
:105660003A4628461946CDF80080019604F10A070B
:105670000B3406F067F93FB224B278233A46284645
:1056800019468DE8500006F05DF9192300943A465A
:1056900001962846194606F055F902B0BDE8F0819A
:1056A000409EFF1F2DE9F0411E4682B01446002A9D
:1056B0006AD0099B4D4A00EBC305012C6F892989EB
:1056C0006868A7EB010382FB03E21A444FEAE37325
:1056D000C3EBA21302887BD0042C38D112FA83F3D7
:1056E000994203DC9F423946A8BF1946089A0180B7
:1056F000B6F90030BDF920803D48971D4FF0000EEF
:105700003FB2194642460097CDF804E006F01AF978
:1057100029896A896B68521A1B885C2AA3EB0103EA
:1057200059DD03EB43030132C3EB431393FBF2F365
:1057300003F11B0213B20120328019464246019048
:1057400000972B4806F0FEF82A4B00221A702A4BCD
:10575000022CB3F9001045D0082C31D100221A8058
:1057600091422DD0089AB6F9003021480632012422
:1057700012B2009219460194BDF9202006F0E2F819
:10578000204602B0BDE8F0811C4D1D4A2B6812680E
:10579000CB1A93420F4617D9164A3388117814480A
:1057A000012918BF01241470089A06321BB212B2E4
:1057B0008DE814001946BDF9202006F0C3F82F60CB
:1057C000012002B0BDE8F081204602B0BDE8F081C2
:1057D0009BB2D31A84E75C2101FB03F393FBF2F243
:1057E0001B32A7E74A1C12B21A80B9E7C94216B2A7
:1057F000409EFF1FB99EFF1F1E9EFF1FA49EFF1FFE
:10580000082B010030B583B000230C4605B200938D
:1058100026225B231C210C4805F0E4FD29460123C8
:105820002622094805F0EEF8002C24B205DB2146BB
:1058300001232622044805F0E5F8044A044B1580AC
:105840001C8003B030BD00BF409EFF1FAA89FF1F10
:10585000AC89FF1F70B59F4C237882B01BB19E4B63
:105860004FF6FF721A809D4BB3F90030C3B99C4AC2
:10587000994B1068B3F9002080F30C005B2303FB05
:1058800000F000131C30824243D04FF0FF31FFF78D
:10589000B9FF944805F00AFE0023237002B070BDE2
:1058A000012B1BD0022B53D0032B38D0042B00F03C
:1058B0008D80052BF0D10F2007F068FEC0F53B600E
:1058C0000830B0F5AF6F41DBB0F5FA6FA8BF4FF409
:1058D000FA60A0F5AF625B2383482EE0834B1A6821
:1058E000B2F52F7F32DB41F25C239342A8BF13460F
:1058F000A3F52F735B227E4802FB03F380FB03209A
:10590000DB17C3EBA0201C30734BB3F9003083428C
:10591000BBD1784BB3F900300133B6D1BCE7764B3D
:105920001B68B3F5FA7F11DBB3F57A6FA8BF4FF4AC
:105930007A637248A3F5FA725B2303FB02F380FBE0
:105940000320DB17C3EB20201C30DDE71C20DBE746
:105950006B4B1B68B3F5FA7F2EDBB3F57A6FA8BFEC
:105960004FF47A63A3F5FA7264485B2303FB02F3F6
:1059700080FB0320DB17C3EB20201C30614B1B682E
:10598000B3F5FA7F1ADBB3F57A6FA8BF4FF47A63E9
:10599000A3F5FA7259495B2303FB02F381FB032150
:1059A000DB17C3EB21211C314B4BB3F90030834291
:1059B00006D0FFF727FF6CE71C20DFE71C21F3E789
:1059C0004C4BB3F900308B42F3D165E72722002519
:1059D0008DE8240076231C2142484B4E05F0B2FF8F
:1059E00016E0B0F5AF7FA8BF4FF4AF70323803FBBD
:1059F00000F386FB0321DB17C3EB61111C3109B2F5
:105A000001231D442722374804F0FCFF0C2D09D048
:105A1000E9B23E4804F0B4FE31284FF05B03E0DC0D
:105A20001C21EDE7012007F0B1FD6FF495733238CA
:105A3000374A03FB00F082FB0023C017C0EB63234F
:105A400003F5AF73312B42DDB3F5AF7FA8BF4FF441
:105A5000AF735B22323B2C4D02FB03F385FB032526
:105A6000DB17C3EB65151C35002007F08FFD6FF4C5
:105A700095733238264A03FB00F082FB0023C017DF
:105A8000C0EB632303F5AF73312B1EDDB3F5AF7F9E
:105A9000A8BF4FF4AF735B22323B1B4902FB03F3F9
:105AA00081FB0321DB17C3EB61111C310A4BB3F9F6
:105AB0000030AB4201D028467BE70E4BB3F90030F3
:105AC0008B423FF4E6AE284673E71C21EEE71C2527
:105AD000CAE700BF149EFF1FAA89FF1F1A9EFF1F5F
:105AE0008C9DFF1F409EFF1F37800B6D8C9BFF1FFF
:105AF000D3058541AC89FF1FCC9BFF1F011FB81246
:105B0000D49BFF1F049EFF1F4B48371B1C9CFF1F8D
:105B100067BBCF462DE9F04FDFF8EC82B74CB8F900
:105B200000604D7854F8264087B08246039305B153
:105B30000D78DFF8FCB2002A34D19BF800308BBB23
:105B4000AF4EB6F90000002800F0CE80012800F02A
:105B50002481012032232A46019000935146A94B0B
:105B60002046FFF79FFD00250746B6F90030022BBF
:105B700040F3F48000233380B8F90030A24A002BB0
:105B8000C0F2F880052BC4BF00231380039B002BB9
:105B900040F0F680002D0CBF38464FF0FF3007B0C4
:105BA000BDE8F08F964EE36822689848049300277A
:105BB000059237808BF8007005F06CFB1120FFF721
:105BC00027FD4FF0010919232821CDF804900091F9
:105BD000242219468D4805F0B5FE78232821242279
:105BE000CDF8049000918948194605F0ABFE49466E
:105BF000864806F03DFA02221921844806F034FA5C
:105C0000DDF8149048460BF0BBF8494602467F4841
:105C100006F0C4FB7D4806F0D7FB394614227B48CA
:105C200006F022FA03227A49784806F0B7FB774853
:105C300006F0CAFB39462322744806F015FA0322FF
:105C40007449724806F0AAFB704806F0BDFB049B3D
:105C5000002B72D10123704A18461370FFF7B8FC6D
:105C6000208963896768191A5C293A885BDC131AF2
:105C70005C2202FB03F292FBF1F31B33674A634899
:105C8000138001271BB21A2219468DE884001422C2
:105C900005F058FE049BDBB1218A638AE768581A35
:105CA0005C283A886FDD521A02EB4202C2EB4212C4
:105CB000431C92FBF3F31B33524A544813800127D1
:105CC00038221BB28DE884001946322205F03AFED4
:105CD000534A544BB6F90000012111704FF6FF7280
:105CE0001A8000287FF432AFDFF848914E4AD9F885
:105CF00000301268C3EB0A0393424CD9464B1A7822
:105D0000012A18BF012018700127FFF761FCC9F8AC
:105D100000A0012D4ED0042D59D0022D60D0082DA9
:105D200064D0002521E7121A02EB4202C2EB4212B4
:105D30004B1C92FBF3F31B33A0E72F20FFF768FC0B
:105D400039463222314806F08FF9032237492F486D
:105D500006F024FB2D4806F037FB7BE77FF40CAF01
:105D6000E368002B3FF406AFB8F90030264A002B59
:105D7000BFF608AF05231380039B002B3FF40AAF47
:105D8000FFF768FD06E7511A5C2202FB01F292FB65
:105D9000F0F31B3390E70746BBE7002714238DE899
:105DA00088002A4651461D4B2046FFF77BFC3D46A6
:105DB0000746DAE6B8F800308BF800500133A8F84F
:105DC0000030636983B1002520469847CDE6B8F8D6
:105DD00000300122013BA8F800308BF80020F0E7EA
:105DE000012333800025C7E61D46BEE66369002215
:105DF00032804FF0FF35002BE6D1BDE6B089FF1FA2
:105E00001E9EFF1F189EFF1F1A9EFF1F409EFF1F12
:105E10000C1C0100101C0100B99EFF1F169EFF1FE5
:105E2000149EFF1FAA89FF1F082B0100141C0100EC
:105E30001C9EFF1FA49EFF1F01210D2007F078B9B3
:105E400000210D2007F074B901460D2007F070B94C
:105E500008B50D2007F072F9B0FA80F149090D205C
:105E6000BDE8084007F064B910B5002144080D20D2
:105E700007F05EF9204607F097F90D20012107F0A1
:105E800057F92046BDE8104007F08EB9214A224B51
:105E900010881B68984210B535DA204A1288141A07
:105EA0009A42A8BF1A46B4F5157F22DA121A40F2B8
:105EB000532303FB02F393FBF4F105310A2006F0B0
:105EC000A7FF174B197801B3164B17491B6840F20F
:105ED000271283F3070302FB03F381FB0321194419
:105EE000DB17C3EBA11105310920BDE8104006F016
:105EF0008FBF131A4FF41572611C02FB03F393FB5F
:105F0000F1F10531DAE70021D8E70920BDE81040BA
:105F100006F07EBF289CFF1F809BFF1FE49DFF1F94
:105F2000EC9BFF1F849BFF1F090402817F2838B56B
:105F3000A8BF7F200F4C4FF4167202FB00F284FBC7
:105F400002311144D2170546C2EBA1110A2006F016
:105F50005FFF7F3D4FF4967303FB05F384FB032142
:105F60001944DB17A3EBA1110920BDE8384006F066
:105F70004FBF00BF09040281C368B3F9003030B5D8
:105F800083EAE374A4EBE374002BA0B218DB0123D3
:105F900000E0134603EB830252009442F9DA0A4D03
:105FA00090FBF3F285FB03E403FB1200DB173032B6
:105FB000D3EBA40380B201F8012BF1D10B7030BDFB
:105FC0002D230B700131E2E76766666638B5094D2F
:105FD0008224204602F056FE35F8021B00B28842A9
:105FE000204601D002F034FE0234A4B28A2CF0D153
:105FF00038BD00BF189DFF1F024B8020198802F09A
:1060000027BE00BFC49BFF1F38B5094D782420462A
:1060100002F038FE35F8021B00B28842204601D05B
:1060200002F016FE0234A4B2802CF0D138BD00BFBD
:10603000109DFF1F024B7620198802F009BE00BF99
:10604000C29BFF1F38B5094D4624204602F01AFEB8
:1060500035F8021B00B28842204601D002F0F8FD5C
:106060000234A4B24E2CF0D138BD00BF989DFF1F62
:10607000024B4420198802F0EBBD00BFBA9BFF1F02
:10608000024B4E20198802F0E3BD00BFD09BFF1FDA
:10609000024B9A20198802F0DBBD00BF109CFF1F45
:1060A000024B9820198802F0D3BD00BFEA9BFF1F66
:1060B000024B8C20198802F0CBBD00BF2A9DFF1F28
:1060C000024B9C20198802F0C3BD00BFB09BFF1F8C
:1060D000024BA020198802F0BBBD00BFA09DFF1F8E
:1060E000024B9620198802F0B3BD00BF7C9DFF1FB4
:1060F000024B8A20198802F0ABBD00BF3E9DFF1FF6
:1061000008B5034B1020198802F0A2FD012008BD3C
:106110003C9DFF1F024B1020198802F099BD00BF63
:106120003C9DFF1F024B2C20198802F091BD00BF3F
:10613000AE9BFF1F024B1E20198802F089BD00BFD5
:10614000C89BFF1FC3680E20198802F081BD00BFE5
:10615000024B2820198802F07BBD00BF949DFF1FD1
:10616000024B6220198802F073BD00BFDA9BFF1F4B
:10617000024B6420198802F06BBD00BF909DFF1F89
:10618000024B5A20198802F063BD00BF949BFF1F89
:10619000024B1620198802F05BBD00BF9C9BFF1FBD
:1061A000024B2E20198802F053BD00BF189CFF1F20
:1061B000024B3020198802F04BBD00BFF09DFF1F3D
:1061C000024B9E20198802F043BD00BF9089FF1F3B
:1061D000024B1820198802F03BBD00BF2E9CFF1F08
:1061E000024BA220198802F033BD00BFC29DFF1FE1
:1061F000024B1A20198802F02BBD00BFD89BFF1F4D
:10620000024B1C20198802F023BD00BFD29BFF1F48
:10621000024B6620198802F01BBD00BFCE9DFF1FF8
:10622000024B7220198802F013BD00BFEC9DFF1FC6
:10623000024B2020198802F00BBD00BFCC9DFF1F30
:10624000024B3220198802F003BD00BFBE9DFF1F24
:10625000024B6820198802F0FBBC00BF049CFF1FA2
:10626000024B6C20198802F0F3BC00BF889BFF1F13
:10627000024B5220198802F0EBBC00BF2E89FF1F91
:10628000024B5020198802F0E3BC00BF2089FF1F99
:10629000024B5420198802F0DBBC00BFA489FF1F09
:1062A000024B5C20198802F0D3BC00BFA889FF1FF5
:1062B000024B5E20198802F0CBBC00BF2C89FF1F67
:1062C000024B6020198802F0C3BC00BF2C9DFF1F49
:1062D000024B5620198802F0BBBC00BF0C9CFF1F6C
:1062E000244B1B880B2B43D8DFE803F00B10151A47
:1062F0001F24292E33383D06084604221E490AF081
:10630000FDBD084604221D490AF0F8BD08460422D6
:106310001B490AF0F3BD084604221A490AF0EEBDF3
:106320000846042218490AF0E9BD08460422174924
:106330000AF0E4BD0846042215490AF0DFBD08460C
:10634000042214490AF0DABD0846042212490AF070
:10635000D5BD0846042211490AF0D0BD08460422E2
:106360000F490AF0CBBD084604220E490AF0C6BD0B
:10637000704700BF7C9DFF1FA4230100682101001E
:106380001C200100582401002020010040240100AD
:106390002420010028200100882201002C20010077
:1063A000B023010030200100064B074A10B41C88BE
:1063B000064B0846002C14BF11461946042210BC97
:1063C0000AF09CBDE89BFF1F34200100382001002B
:1063D000064B074A10B41C88064B0846002C14BF15
:1063E00011461946042210BC0AF088BD1A9CFF1FF2
:1063F0003420010038200100064B074A10B41C88E5
:10640000064B0846002C14BF11461946042210BC46
:106410000AF074BD2E9DFF1F3420010038200100BA
:10642000064B074A10B41C88064B0846002C14BFC4
:1064300011461946042210BC0AF060BD449DFF1F9E
:106440003420010038200100064B074A10B41C8894
:10645000064B0846002C14BF11461946042210BCF6
:106460000AF04CBD7E9DFF1F342001003820010042
:10647000064B074A10B41C88064B0846002C14BF74
:1064800011461946042210BC0AF038BD1E9CFF1F9D
:1064900034200100382001001B4B1B880A2B0AD82E
:1064A000DFE803F00A0E12161A1E22262A2E060014
:1064B000164B186808607047154B186808607047DD
:1064C000144B186808607047134B186808607047D1
:1064D000124B186808607047114B186808607047C5
:1064E000104B1868086070470F4B186808607047B9
:1064F0000E4B1868086070470D4B186808607047AD
:106500000C4B1868086070473E9DFF1F602001001B
:10651000382001003C2001004020010044200100FF
:10652000482001004C2001005020010054200100AF
:10653000582001005C200100F0B52B4E2B4FDFF8F6
:10654000C4E005460FCE87B06C460FC496E8030042
:106550003B68274A274F44F8040B40F6CC3083426F
:10656000C8BF3A46BEF800602180012E118892789B
:10657000ADF80D108DF80F202AD032D340F6CA02A4
:10658000022E18BF00229A4226DAA3F698031A496F
:106590001A4AC3EB031381FB03011944DB17C3EB56
:1065A0006123243382FB0321DA17C2EBA10202EB41
:1065B0008201A3EB4103303330328DF813308DF874
:1065C00011206946284616220AF098FC07B0F0BD53
:1065D00040F698029A42D8DB094B1868CDF81100B2
:1065E000EFE740F6FC02CEE774200100849DFF1F18
:1065F00068200100642001003B773B98676666666F
:106600006C200100209DFF1FF8B5174C174E227813
:10661000174D33782F888E46003218BF012201466D
:106620007046FFF777FA002398423370237015DB2A
:1066300014BF012000202B889F420ED040F23A72F6
:10664000A3F5AF730B490C4C02FB03F381FB031260
:10665000DB17A3EB621332332360F8BD0749012235
:1066600018460A702270E6E7A08AFF1F319EFF1FBE
:10667000DC9DFF1FB5814E1B9489FF1FB89EFF1F35
:10668000014B187802F07CBAA09EFF1F014B1878CE
:1066900002F090BA4C90FF1F134BB3F9003030B5A5
:1066A00083EAE374A4EBE374002BA0B218DB0123AC
:1066B00000E0134603EB830252009442F9DA0B4DDB
:1066C00090FBF3F285FB03E403FB1200DB1730328F
:1066D000D3EBA40380B201F8012BF1D10B7030BDD4
:1066E0002D230B700131E2E74C90FF1F6766666651
:1066F000144BB3F9003070B583EAE375A5EBE3758D
:10670000002BACB21ADB012300E0034603EB83004D
:1067100040008542F9DA0C4E94FBF3F086FB03E56A
:1067200003FB1044DB173030D3EBA503A4B201F810
:10673000010BF1D105480B70106070BD2D230B705B
:106740000131E0E7949BFF1F676666668C200100BD
:10675000134BB3F9003030B583EAE374A4EBE37470
:10676000002BA0B218DB012300E0134603EB8302E9
:1067700052009442F9DA0B4D90FBF3F285FB03E4EF
:1067800003FB1200DB173032D3EBA40380B201F815
:10679000012BF1D10B7030BD2D230B700131E2E7DD
:1067A0009089FF1F67666666134BB3F9003030B5FA
:1067B00083EAE374A4EBE374002BA0B218DB01239B
:1067C00000E0134603EB830252009442F9DA0B4DCA
:1067D00090FBF3F285FB03E403FB1200DB1730327E
:1067E000D3EBA40380B201F8012BF1D10B7030BDC3
:1067F0002D230B700131E2E7C29DFF1F67666666BD
:10680000134BB3F9003030B583EAE374A4EBE374BF
:10681000002BA0B218DB012300E0134603EB830238
:1068200052009442F9DA0B4D90FBF3F285FB03E43E
:1068300003FB1200DB173032D3EBA40380B201F864
:10684000012BF1D10B7030BD2D230B700131E2E72C
:106850002E89FF1F67666666134BB3F9003030B5AB
:1068600083EAE374A4EBE374002BA0B218DB0123EA
:1068700000E0134603EB830252009442F9DA0B4D19
:1068800090FBF3F285FB03E403FB1200DB173032CD
:10689000D3EBA40380B201F8012BF1D10B7030BD12
:1068A0002D230B700131E2E72089FF1F67666666C2
:1068B000134BB3F9003030B583EAE374A4EBE3740F
:1068C000002BA0B218DB012300E0134603EB830288
:1068D00052009442F9DA0B4D90FBF3F285FB03E48E
:1068E00003FB1200DB173032D3EBA40380B201F8B4
:1068F000012BF1D10B7030BD2D230B700131E2E77C
:10690000A489FF1F67666666134BB3F9003030B584
:1069100083EAE374A4EBE374002BA0B218DB012339
:1069200000E0134603EB830252009442F9DA0B4D68
:1069300090FBF3F285FB03E403FB1200DB1730321C
:10694000D3EBA40380B201F8012BF1D10B7030BD61
:106950002D230B700131E2E7A889FF1F6766666689
:10696000134BB3F9003030B583EAE374A4EBE3745E
:10697000002BA0B218DB012300E0134603EB8302D7
:1069800052009442F9DA0B4D90FBF3F285FB03E4DD
:1069900003FB1200DB173032D3EBA40380B201F803
:1069A000012BF1D10B7030BD2D230B700131E2E7CB
:1069B0002C89FF1F6766666608B5702002F062F9D1
:1069C000044B1988884204D07020BDE8084002F0CA
:1069D0003FB908BD209DFF1F08B5742002F052F991
:1069E000044B1988884204D07420BDE8084002F0A6
:1069F0002FB908BDB49DFF1F054B1B880846042214
:106A000013B904490AF07ABA03490AF077BA00BF09
:106A1000D09BFF1F94200100902001000E4B1B888B
:106A2000032B17D8DFE803F0110C070208460422F5
:106A30000A490AF063BA0846042209490AF05EBA14
:106A40000846042207490AF059BA084604220649B2
:106A50000AF054BA704700BF2A9DFF1FA42001000E
:106A6000A02001009C2001009820010010B40A4BD6
:106A70000A4C0A4693E8030083B0238802AC04E979
:106A8000030004EB8303104653F8081C052203B0EF
:106A900010BC0AF033BA00BFA81C0100909DFF1F74
:106AA00030B40A4B0A4D0C4693E8070084B02B889B
:106AB00004AD05E9070005EB8303204653F80C1CE1
:106AC000042204B030BC0AF019BA00BFB01C0100A7
:106AD000209DFF1FF0B40C4D0C4F0E460FCD8CB017
:106AE00001AC0FC40FCD0FC495E807003B8884E8C4
:106AF00007000CAA02EB8303304653F82C1C042237
:106B00000CB0F0BC0AF0FAB9BC1C0100729DFF1F6A
:106B1000F0B40B4D0B4F0E460FCD86B06C460FC434
:106B200095E803003B8884E8030006AA02EB830390
:106B3000304653F8181C042206B0F0BC0AF0DEB947
:106B4000E81C01002E9CFF1FF0B40A4D0A4F0E46B0
:106B50000FCD86B001AC0FC42A683B88226006AA1C
:106B600002EB8303304653F8141C0C2206B0F0BC31
:106B70000AF0C4B9001D0100D29BFF1FF0B40A4DFA
:106B80000A4F0E460FCD86B001AC0FC42A683B8871
:106B9000226006AA02EB8303304653F8141C042239
:106BA00006B0F0BC0AF0AAB9141D0100B49DFF1F85
:106BB000164B1B880BB31BB283EAE370A0EBE370A8
:106BC000002B30B584B21DDB012300E0134603EB3C
:106BD000830252009042F9DA0D4894FBF3F280FBF5
:106BE00003E503FB1244DB173032D3EBA503A4B259
:106BF00001F8012BF1D10B7030BD08460422054984
:106C00000AF07CB92D230B700131DDE7049CFF1FD6
:106C100067666666A820010030B40A4B0A4D0C4630
:106C200093E8070084B02B8804AD05E9070005EB65
:106C30008303204653F80C1C042204B030BC0AF035
:106C40005DB900BF281D0100889BFF1F054B1B88F5
:106C50001BB9054B186808607047084604220349B1
:106C60000AF04CB9A09DFF1F38200100342001001C
:106C7000164B1B880BB31BB230B583EAE374A4EB4D
:106C8000E374002BA0B21CDB012300E0134603EBEE
:106C9000830252009442F9DA0D4D90FBF3F285FB2A
:106CA00003E403FB1200DB173032D3EBA40380B202
:106CB00001F8012BF1D10B7030BD064B186808604C
:106CC00070472D230B700131DEE700BFC89BFF1F0B
:106CD0006766666638200100164B1B880BB31BB233
:106CE00030B583EAE374A4EBE374002BA0B21CDBA1
:106CF000012300E0134603EB830252009442F9DAC9
:106D00000D4D90FBF3F285FB03E403FB1200DB1750
:106D10003032D3EBA40380B201F8012BF1D10B7018
:106D200030BD064B1868086070472D230B70013189
:106D3000DEE700BFC49DFF1F67666666382001005E
:106D4000164B1B880BB31BB230B583EAE374A4EB7C
:106D5000E374002BA0B21CDB012300E0134603EB1D
:106D6000830252009442F9DA0D4D90FBF3F285FB59
:106D700003E403FB1200DB173032D3EBA40380B231
:106D800001F8012BF1D10B7030BD064B186808607B
:106D900070472D230B700131DEE700BF9C9BFF1F66
:106DA00067666666AC200100174B1B881BB31BB2DD
:106DB00070B583EAE375A5EBE375002BACB21EDB7F
:106DC000012300E0034603EB830040008542F9DA2B
:106DD0000E4E94FBF3F086FB03E503FB1044DB1738
:106DE0003030D3EBA503A4B201F8010BF1D1084870
:106DF0000B70106070BD074B1868086070472D233A
:106E00000B700131DCE700BF189CFF1F67666666E8
:106E1000B020010038200100164B1B880BB31BB2B9
:106E200030B583EAE374A4EBE374002BA0B21CDB5F
:106E3000012300E0134603EB830252009442F9DA87
:106E40000D4D90FBF3F285FB03E403FB1200DB170F
:106E50003032D3EBA40380B201F8012BF1D10B70D7
:106E600030BD064B1868086070472D230B70013148
:106E7000DEE700BFF09DFF1F6766666638200100F1
:106E8000164B1B880BB31BB230B583EAE374A4EB3B
:106E9000E374002BA0B21CDB012300E0134603EBDC
:106EA000830252009442F9DA0D4D90FBF3F285FB18
:106EB00003E403FB1200DB173032D3EBA40380B2F0
:106EC00001F8012BF1D10B7030BD064B186808603A
:106ED00070472D230B700131DEE700BFCE9DFF1FF1
:106EE0006766666638200100164B1B880BB31BB221
:106EF00030B583EAE374A4EBE374002BA0B21CDB8F
:106F0000012300E0134603EB830252009442F9DAB6
:106F10000D4D90FBF3F285FB03E403FB1200DB173E
:106F20003032D3EBA40380B201F8012BF1D10B7006
:106F300030BD064B1868086070472D230B70013177
:106F4000DEE700BFEC9DFF1F676666663820010024
:106F5000174B1B881BB31BB270B583EAE375A5EB17
:106F6000E375002BACB21EDB012300E0034603EB0C
:106F7000830040008542F9DA0E4E94FBF3F086FB65
:106F800003E503FB1044DB173030D3EBA503A4B2B9
:106F900001F8010BF1D108480B70106070BD074B70
:106FA0001868086070472D230B700131DCE700BFC3
:106FB000CC9DFF1F67666666B02001003820010087
:106FC000074B1B88022B06D0012B0CBF054B064B31
:106FD000186808607047054B18680860704700BF64
:106FE0002C9DFF1FB8200100BC200100B42001002F
:106FF000054B1B881BB1054B186808607047044B94
:1070000018680860704700BF0C9CFF1FC420010077
:10701000C0200100184B1A8852B3184A128830B5A4
:107020000A80B3F90030002B83EAE374A4EBE37425
:10703000BCBF2D238B70A0B2ACBF02310331012342
:1070400000E0134603EB830252009442F9DA0C4D40
:1070500090FBF3F285FB03E403FB1200DB173032F5
:10706000D3EBA40380B201F8012BF1D10B7030BD3A
:10707000044B186808607047D89BFF1FC8200100A8
:10708000676666663820010070B53C4D2B78064671
:10709000002B35D11C4673780BB9204670BDFAF72A
:1070A00055FE374A374B3848127831781B780078CC
:1070B00002EB43034A1E03EB80030E2AEDD801A026
:1070C00050F822F02D7100004F7100009B700000FD
:1070D0002D7100009B7000009B7000009B700000F1
:1070E0001B7100009B7000009B7000009B700000F3
:1070F0009B7000009B7000009B70000017710000E7
:10710000AE21224803F076FE204804F0C3F80023A5
:107110002B700124BFE706F059FBAF211B4803F099
:1071200069FE1B4A012313702B70B6E783B9194817
:10713000038804294FF6FF7103F1FF320CBF0123CE
:107140000B46134403F07F03013303800FE073B158
:10715000013B114A32F813304BB10E4E0F48104923
:10716000104A33800123002606700B701370084A02
:107170000221012311702B70204670BDA08AFF1FD1
:10718000109EFF1F119EFF1FC69DFF1F409EFF1FE9
:10719000B89EFF1FC09DFF1F009DFF1FFC9BFF1F90
:1071A0009E9BFF1FBB9EFF1F10B5064B064C1A8807
:1071B0002046012101F03AFD21884220BDE810401F
:1071C00001F046BDE89BFF1FB89BFF1F10B5064BA3
:1071D000064C1A882046022101F028FD2188422011
:1071E000BDE8104001F034BD1A9CFF1FB89BFF1F83
:1071F00010B5064B064C1A882046042101F016FDF6
:1072000021884220BDE8104001F022BD2E9DFF1FC5
:10721000B89BFF1F10B5064B064C1A882046062166
:1072200001F004FD21884220BDE8104001F010BDAE
:10723000449DFF1FB89BFF1F10B5064B064C1A88D4
:107240002046002101F0F2FC21884220BDE81040D8
:1072500001F0FEBC7E9DFF1FB89BFF1F08B51220EA
:1072600001F010FD054B1988884206D0122001F06C
:10727000EFFCBDE8084001F003BC08BD729DFF1F94
:1072800008B5582001F0FEFC054B1988884206D04D
:10729000582001F0DDFCBDE8084001F0F1BB08BD5D
:1072A000C49DFF1F08B5142001F0ECFC054B1988A4
:1072B000884206D0142001F0CBFCBDE8084001F064
:1072C000DFBB08BD1E9CFF1FF0B480EAE075A5EB94
:1072D000E0750028ACB21FDB1DBF2B230B704E1CCA
:1072E0000E46012300E0134603EB83025200954251
:1072F000F9DA0B4F94FBF3F287FB030503FB12440F
:10730000DB173032D3EBA503A4B206F8012BF1D181
:1073100033700846F0BC70472D230B704E1CE0E71D
:1073200067666666174B18880C2813D0192815D085
:107330001A2817D01B2819D01C281BD01D281DD097
:107340001E2803D00C3800B2FFF7BEBF0E4A1068EB
:10735000086070470D4A1068086070470C4A106852
:10736000086070470B4A1068086070470A4A106846
:1073700008607047094A106808607047084A10683A
:1073800008607047BE9DFF1FE8200100D02001006B
:10739000D4200100D8200100DC200100E020010001
:1073A000E4200100034B1888A0EB8000400000B2ED
:1073B000FFF78ABFA09EFF1F024BB3F90000FFF743
:1073C00083BF00BFDA9BFF1F024B1888033800B24F
:1073D000FFF77ABF949DFF1F024B18880C3800B24C
:1073E000FFF772BF989BFF1F024B1888183800B236
:1073F000FFF76ABFC49BFF1F024B1888183800B202
:10740000FFF762BFC29BFF1F024B1888183800B2FB
:10741000FFF75ABFBA9BFF1FC3681888183800B21D
:10742000FFF752BF054B1B881BB9054B1868086056
:10743000704708460422034909F060BDEA9BFF1F1C
:107440003820010034200100054B1B881BB9054B77
:1074500018680860704708460422034909F04EBDC9
:10746000109CFF1F382001003420010030B5134C60
:1074700085B001252B463C2202212046009503F0D1
:107480002FFD204603F006FF0022402180232046E6
:107490000191009311460A4B029504F0A9FB204686
:1074A00004F004F807480849084A00230360838071
:1074B0000B608B801360938005B030BD409EFF1F32
:1074C000E4260100209EFF1F389EFF1FA89EFF1F7D
:1074D00010B500EBC00000F10F02D2B293B284B03D
:1074E0009C1E981C3D2303918DE819003921024808
:1074F00004F0E2FA04B010BD409EFF1F014B0122D0
:107500001A707047319EFF1FF0B56B4B6B4C6C4F80
:107510006C4E6D4D85B004228DE80C000293204620
:107520006A4B4022802103F0E3FA2046684A694909
:10753000694C08F047FE6949694A8F61694FCF611C
:10754000694F9761694B6A4FD7616A4F9F616A4F74
:10755000DF616A4FB7616A4FF7616A4FAF616A4F87
:10756000EF616A4FA7616A486A4FE7616A4F8761B6
:107570006A496B4FC7616B4F8F616B4A6B4FCF612D
:107580006B4F97616B4B6C4FD7616C4F6C4E9F612B
:107590006C4FDF616C4F6D4DB7616D4FF7616D4F93
:1075A0006D4CAF616D4FEF616D4F6E48A7616E4FCF
:1075B000E7616E4F6E4987616E4FC7616E4F6F4ACC
:1075C0008F616F4FCF616F4F6F4B97616F4FD76177
:1075D0006F4F9F616F4E704FDF61704FB761704D9D
:1075E000704FF761704FAF61704C714FEF61714F29
:1075F000A7617148714FE761714F87617149724F9F
:10760000C761724F8F61724A724FCF61724F97613B
:10761000724B734FD761734F9F61734E734FDF612E
:10762000734FB761734D744FF761744FAF61744C12
:10763000744FEF61744F7548A761754FE761754FDF
:1076400075498761754FC761754F764A8F61764F6F
:10765000CF61764F764B9761764FD761764F774EF5
:107660009F61774FDF61774F774DB761774FF76154
:10767000774F784CAF61784FEF6178487849794F10
:10768000794DA761E561794F794D7A4CDFF808E2D1
:10769000794A7A4B8761C5618C61794E794F7A4D11
:1076A0007A4CC1F81CE07A487A499761D5619C61AF
:1076B000D861B16005B0F0BD40420F00409EFF1F91
:1076C000D9730000088CFF1FCC8EFF1F6890FF1F2E
:1076D0001C89FF1F49AB0000108AFF1FEC89FF1FA8
:1076E000A88EFF1F45610000C9730000188EFF1FA0
:1076F00051610000A9630000A9710000D16300007E
:10770000CD710000F9630000F1710000B973000051
:10771000988CFF1F6161000021640000288DFF1F0D
:10772000157200006D6A0000748CFF1F716100000B
:1077300049640000048DFF1F39720000A57300002A
:10774000E08CFF1F8166000099660000848EFF1F99
:107750008D660000A16A00009C8BFF1FB9690000C4
:10776000D56A0000388FFF1F5D720000D96C0000E1
:10777000508CFF1F81720000F1660000588BFF1FC4
:107780008161000071640000A48FFF1FA5720000DA
:10779000416D00002C8CFF1F91610000A96D00005D
:1077A0004C8DFF1FA1610000196E0000E48BFF1FCC
:1077B000B161000051670000C88AFF1FC16100006D
:1077C000116B0000348AFF1FD1610000A96700001F
:1077D000BC8CFF1FE161000015700000608EFF1F70
:1077E000F1610000496B00002890FF1F016200005A
:1077F000816E0000F48DFF1F11620000E96E000031
:10780000EC8AFF1F216200007D6B00005C8FFF1F70
:10781000D9690000516F00003C8EFF1F31620000EB
:1078200025730000108BFF1F41620000B16B000048
:10783000A48AFF1F51620000196C0000F88FFF1F1F
:107840006162000001680000C08BFF1F71620000D0
:10785000596800007C8AFF1F81620000348BFF1F83
:10786000F08EFF1FB16800009162000009690000FE
:10787000A162000061690000588AFF1FC889FF1FCC
:107880001C90FF1FC16F0000C1620000F16F00007B
:10789000D1620000217E0000B1620000F0B5461CFC
:1078A00083B00D460127032336B22AB2044631467F
:1078B0008DE888002448ADB204F094F80C23AA1C8B
:1078C00012B200930197052321B21F4804F08AF8F1
:1078D0001E4A1F4B12881B68BA422AD023D3022AA1
:1078E00010D11C4CA3F6CA0384FB03241C44DB17F1
:1078F000C3EB24140A2CA8BF0A2424EAE474A2B21D
:1079000023B202E000231A461C460D35AA1A0120B4
:107910000093019012B2314603230B4803F0E0FFBD
:10792000204603B0F0BD0C4CA3F6FC0384FB0324FB
:10793000DDE7084CA3F6980384FB03241C44DB1703
:10794000C3EBE404D6E700BF409EFF1F209DFF1F4E
:10795000849DFF1F898888881F85EB512DE9F0439E
:107960008FB283B0DFF84C80BD1D461D2DB204B22E
:1079700036B24FF001090AB223463146404600951F
:10798000CDF8049003F0DEFF2A46334621464046F8
:107990008DE8200203F0D6FF07F10C020095334674
:1079A00012B22146CDF80490404603F0CBFF03B05D
:1079B000BDE8F083409EFF1F2DE9F043804685B06F
:1079C000002956D10121304804F052FB2F4998F884
:1079D000062098F8083011F80290994522DA4FEA0B
:1079E00089064D460C24D8F80C3027489B595F680F
:1079F00022B2002104F038FB384609F0C1F93946BB
:107A00000246214804F0CAFC1F4804F0DDFC98F847
:107A1000083001350934AB42A4B206F1040601DD99
:107A2000422CE0D1B9F1000F13D109F106099945B3
:107A30000CDA3C2301213B22039102930093019233
:107A400039233F223A21104804F036F805B0BDE84A
:107A5000F0830F2301213B220391029300930192B3
:107A600039230C223A21084804F026F898F8083007
:107A7000DBE700213423009301913F230C220248CD
:107A800003F02EFF9EE700BF409EFF1F389EFF1FA2
:107A900010B5104C0121204604F0F0FA20460121D7
:107AA00004F0E6FA20463422552104F0DDFA20469F
:107AB0000222094904F072FC20460522074904F01D
:107AC0006DFC204604F080FC2046BDE8104003F029
:107AD000EDBC00BF409EFF1FEC200100F020010024
:107AE00070B50D46064609F04BF900EB40008400E6
:107AF000002D36D0284609F043F900EB4000400045
:107B000023185B1003F16001091A282209B21748F3
:107B1000C3F1600404F0A8FA0121144804F0A8FAA3
:107B2000284609F02DF929460246104804F036FC93
:107B30000E4804F049FC02210C4804F099FA21B2E5
:107B400021220A4804F090FA304609F019F931462A
:107B50000246064804F022FC0448BDE8704004F0E8
:107B600033BC6410C4F16004E5E700BF409EFF1F12
:107B7000184B70B5B3F9003083EAE374A4EBE374F7
:107B8000002B82B0A1B21EDB68466D46012300E0E7
:107B9000134603EB830252009442F9DA0E4E91FB36
:107BA000F3F286FB03E403FB1211DB173032D3EB55
:107BB000A40389B205F8012BF1D119462B70FFF708
:107BC0008FFF02B070BD2D238DF800300DF101053F
:107BD0006846DBE73C9DFF1F6766666610B50D4B88
:107BE0001B5C51F82340237884B013B1012004B00A
:107BF00010BD04AA01A942F8103D2046A369984788
:107C0000A38A9B07F2D401A80099FFF769FF01201E
:107C100004B010BD209EFF1F2DE9F04F2F4DDFF85F
:107C2000CCB0DFF8C4A0DFF8C8900FCD91B003ACA2
:107C30000FC40FCD0FC40FCD0FC42B6823600025D8
:107C4000A8462F462E4600E09846BAF80030244950
:107C50005BF8232028461123F8F710FD00EBC00441
:107C600000EB840089FB00340444C017C0EB64348B
:107C7000C4F13C00C6F13C0207F14101012600B20B
:107C800008F1410300901BB2019612B209B21548E7
:107C900003F058FE08EB060305F211153C2B2646AF
:107CA000ADB24746D0D134226B210E4804F0DCF946
:107CB00000210C4804F0DCF90B4B1B8810AA02EBE6
:107CC000830353F8344C204609F05AF8024605481D
:107CD000214611B0BDE8F04F04F060BB341D010037
:107CE00024170100409EFF1FAE9BFF1F20150100BF
:107CF0000900028010B5424C424882B003F0CAFA33
:107D00002378C3B906213F4804F0B2F92378012B48
:107D100037D90A22022B11463A486BD004F0A4F955
:107D200039490322374804F039FB364802B0BDE830
:107D3000104004F049BB354B1A7801210523002A75
:107D400035D10191009311462E4803F04BFE304B84
:107D50001A78002A36D005230122019200930022CE
:107D60000A21284803F0BCFD2A4B1A78002A35D195
:107D700001210523019100931421224803F032FED2
:107D8000C0E7254C2388092B32D9632B8CBF0A21ED
:107D90001F210A221B4804F067F92188194804F0C2
:107DA00063FB184802B0BDE8104004F00DBB002290
:107DB000019100931146134803F092FD144B1A7879
:107DC000002AC8D105230121019100930A210D4801
:107DD00003F008FE0F4B1A78002AC9D001220523B0
:107DE0000192009300221421064803F079FD89E7EF
:107DF0003021CEE704F038F90322084992E700BFAA
:107E0000BB9EFF1F409EFF1FFC200100109EFF1F16
:107E1000119EFF1FC69DFF1FC09DFF1FF820010080
:107E2000F8B56D4D287840B96C4B1B6899425CD30E
:107E30006B4A012313702B70F8BD0C46002669486D
:107E4000664F03F027FA04F6AC53324665483B60B0
:107E500031212E7004F008F901216248624D04F0CE
:107E60000DF931465F4804F003F905225F495D488A
:107E700004F094FA5B4804F0A7FA0C221021594848
:107E800004F0F2F80B225A49564804F087FA05220A
:107E90005849544804F082FA524804F095FA564B77
:107EA00050481C68A4F69803C3EB031385FB032515
:107EB0001D441021DB172022C3EB652504F0D4F804
:107EC00040F6CC339C4205F124054FF022014FF0DF
:107ED00004000BDCFFF7E2FC484B1C88064674B339
:107EE000012C46D0022C41D00120F8BDFFF736FD11
:107EF000092243493B4804F051FA2A22102139480B
:107F000004F0B2F83F4C374884FB0534EB17C3EB61
:107F1000A404214604F0A8FA01223B49314804F0A8
:107F20003DFA04EB8401A5EB41012E4804F09CFAD4
:107F3000012236492B4804F031FA0120F8BD3449BA
:107F40001022284804F02AFA264804F03DFA2A2292
:107F50001021244804F088F83146224804F084FABD
:107F600007222C491F4804F019FACBE70C222A49B2
:107F7000E7E70C2229491B4804F010FA194804F0DD
:107F800023FA2A221021174804F06EF831461548CA
:107F90001C4E04F069FA07221E49124804F0FEF94B
:107FA00086FB0536EB17C3EBA60631460D4804F0F9
:107FB0005BFA224614490B4804F0F0F906EB8601FF
:107FC000A5EB4101074804F04FFA22460F49054846
:107FD00004F0E4F92046F8BDA08AFF1F289EFF1F89
:107FE000B89EFF1F409EFF1F3B773B98002101007A
:107FF00008210100F0200100849DFF1F209DFF1F2C
:108000001421010067666666982C0100102C01009F
:1080100020210100342101004C2101003C210100FC
:108020002DE9F041754C2278002A05460F4614BF11
:108030004FF001084FF000084ED1714E3368CB1A53
:10804000B3F5FA6F04D86B78A3B94046BDE8F08168
:108050006C4B6D486D49DFF8D0E11A700123037055
:108060000988237026208EF8002000F0F1FD6B783F
:10807000002BEAD03760F9F769FE654A654B66491F
:10808000127828781B78097802EB4303421E03EB31
:1080900081030E2AD9D801A151F822F08D81000068
:1080A000598100004B8000008D8100004B80000052
:1080B0004B8000004B800000418100004B8000009D
:1080C000F38000004B8000004B8000004B800000DC
:1080D0004B800000EF800000AF215048484E02F076
:1080E00089FEFFF707FE002337602370ABE705F03A
:1080F0006DFB4A4803F0CEF80221484803F0B8FF70
:108100000F222321454803F0AFFF0522444943488D
:1081100004F044F9414804F057F91E2223213F4856
:1081200003F0A2FF05223F493C4804F037F93B48E1
:1081300004F04AF9394803F0B9F900F0ADFC84E7DE
:10814000394D2B78012B50D9304B2620198800F05F
:108150007FFD00232B7078E7002B3FF476AF013BC7
:10816000324A32F81330002B3FF46FAF274C3048BF
:1081700025492D4A23804FF001080023037081F820
:10818000008082F80080FFF7B5FD5EE793B1013B08
:10819000264A32F8131019B31C4B254D1A4C224AAB
:1081A00019800026012326202E702370137000F002
:1081B0004FFD15E0154C1E4922880B7004284FF620
:1081C000FF7002F1FF310CBF012202460A440E4E3D
:1081D000154D02F07F0201320121228031702B7097
:1081E000FFF788FD4FF001082FE70649064A0123F3
:1081F0000020087013702370A6E700BFA08AFF1F3D
:10820000B49EFF1FB89EFF1F9E9BFF1FC09DFF1FB8
:10821000109EFF1F119EFF1FC69DFF1F409EFF1F48
:108220005C21010064210100BB9EFF1F009DFF1F18
:10823000FC9BFF1F2DE9F04F05468BB00F46AD4864
:108240000121164603F01AFFAA8812F0010440F03B
:10825000B080DFF8CC8298F80030002B7DD1AB796C
:10826000A54AD15CA1B9DFF8BCA279781AF80390CD
:1082700041B339780139072900F2B780DFE811F0FE
:10828000F1005401B5006C01B500B500B500E9007E
:108290007C78002C00F0CA800139EC68387854F8FA
:1082A0002170FC68411EB4F80080072900F2A78005
:1082B000DFE811F074015901A5006C01A500A500CB
:1082C000A5009F00DFF854A2DAF80020B21AB2F538
:1082D000967F75D9894A107801281ABF012010703D
:1082E0001170874A18BF0146D05CC0EB0900C0B2CC
:1082F000FFF7EEF80124CAF80060AB889B0770D541
:108300007B78002B6DD0F9F721FD7E4B7E4A7F48AC
:108310001B78127839780078022515FB02330A2978
:1083200003EB800300F04E810C295AD1002B58D06A
:1083300003F11900764E774A013B0021400080B2DC
:1083400026F813100123157088F8003000F080FC27
:10835000714B032220461A702FE0664802F09AFF04
:108360000121644803F084FE62482246214603F05E
:108370007BFEAB88580725D42C68204608F000FD0A
:10838000214602465B4804F009F85A4804F01CF8FC
:10839000092201238DE80C0000217F23554803F0BA
:1083A000D1FA00212846FFF707FB002388F80030A8
:1083B00055E7AB683146384698470BB0BDE8F08FBB
:1083C0000846FAE72B6804A8984704A808F0D8FCE8
:1083D00004A90246474803F0E1FF464803F0F4FFD2
:1083E000D6E720460BB0BDE8F08F00240AF80390D2
:1083F00083E70021D1543846FB699847FC68A4F80C
:108400000080002725223C238DE88400412118228A
:10841000384803F065FAE968A879FFF7DFFB374AC7
:108420003E4B17701E600BB0BDE8F08F3B490A68E9
:10843000B21AB2F5967FD4D9304F0E603E78012E35
:1084400000F0B480E968184601233B70FFF7C6FBD3
:10845000B3E7304AE9791170012288F8002000243E
:10846000C4E72A7A013A4A45BFDD09F10104E4B2C2
:10847000A145BAD0224E16F803B0CBEB0900C0B22A
:108480000021FFF725F82B7A052BD9461BD9CBEB1A
:108490000402042A40F3AE80A4F1040BBBF1000FE8
:1084A000C0F2B080063B5B45A8BF5B465FFA83F92C
:1084B000AA791348B15C994205D000F802900121D5
:1084C0002846FFF779FAC9EB0400C0B201210B4E30
:1084D000FEF7FEFF0021342301910093054831701F
:1084E00040230B223F21A14603F0FAF90124AB7986
:1084F0007CE700BF409EFF1FA89EFF1FB99EFF1F85
:10850000389EFF1F109EFF1F119EFF1FC69DFF1F5D
:10851000009DFF1FB89EFF1FBB9EFF1FA49EFF1F55
:10852000A08AFF1F209EFF1F0FFA89F1E868604CA8
:1085300050F821602168049134785E4904980860FD
:10854000002C71D0012C7FF450AF5B4A317A88F84F
:1085500000401170002449E7B9F1000F50D009F133
:10856000FF34E4B284E7B98A01F0040189B200293A
:108570003FF440AF3B6A03929847039A00283FF4C8
:108580003DAFAB79FC680021D15438E77B8A434585
:108590003CD908F101081FFA88F830E73B8A4345C7
:1085A0003BD208F1FF381FFA88F828E725238DE829
:1085B000180042483C703C231822412103F090F9F6
:1085C0003046FAE6002B3FF40CAF3D4A3D4E118891
:1085D000394A03F11900013B400080B226F813101C
:1085E000012388F80030157000F032FB364B20462E
:1085F0001D70E2E6002A3FF755AF04F1FF3B4DE75F
:108600004C46F3E64FF000094B4651E7BB8ADA07C8
:108610007FF5F5AEB7F81080F1E6BB8AD9077FF594
:10862000EEAEB7F81280EAE62849C85CC0EB090054
:1086300009F1010EC0B201214FF0340B02F803E042
:10864000FEF746FFB6681D48019440230B223F21E8
:108650000124CDF800B003F043F940230B223F2161
:108660001648CDF800B0019403F0BCF92146134838
:1086700003F0FEFC304608F083FBA0EB800000F125
:108680005F0109B20F220D4803F0EEFC304608F0FE
:1086900077FB31460246094803F080FE074803F0A5
:1086A00093FEE968A879FFF799FAAB799EE600BFD7
:1086B000F89EFF1FA49EFF1FB89EFF1F409EFF1F36
:1086C000C09DFF1F009DFF1FBB9EFF1F389EFF1F09
:1086D0002DE9F047DFF808926D4B99F800601B68B0
:1086E000DFF800A282B0003601934FF0030018BFFC
:1086F0000126019F9AF8008004F020FD0546042021
:1087000004F01CFD0446052004F018FD800040EA3A
:108710004404062004F012FD2C4364B25D4944EA8F
:10872000C0000A7880F00F03DBB29A425A4A3CD06C
:108730001760002259480B7003788DF800808DF87F
:10874000012053B3564A12684EF66021BA1A8A4283
:1087500019D8022B59D0012B5FD0062B48D0032B00
:1087600063D0042B69D0052B77D0072B7DD0082B45
:1087700000F08380092B68D016B14A4802F096FEBB
:1087800002B0BDE8F087484A484C0023012123701D
:1087900003701360938089F800103A466946444894
:1087A000FFF748FD3043C6B2E6E71268BA1A1E2A40
:1087B0006BD99AF80020934222D0394C3D488AF870
:1087C0000030012B276082EA030207609846B1D08F
:1087D000042BAFD137480068381AB0F5C87FA9D943
:1087E000354C2068381A3228A4D927601A46A1E7E8
:1087F0003A4669463148FFF71DFD3043C6B2BBE734
:10880000012B4FF00002E3D1E4E73A4669462C48D9
:10881000FFF710FD3043C6B2AEE73A466946294835
:10882000FFF708FD3043C6B2A6E73A466946264838
:10883000FFF700FD3043C6B29EE73A46694623483B
:10884000FFF7F8FC3043C6B296E73A46694620483F
:10885000FFF7F0FC3043C6B28EE73A4669461D4842
:10886000FFF7E8FC3043C6B286E73A4669461A4845
:10887000FFF7E0FC3043C6B27EE73A466946174848
:10888000FFF7D8FC3043C6B276E7002252E700BFBC
:10889000F89EFF1FBC9EFF1F2C9EFF1FB89EFF1F50
:1088A000B09EFF1F409EFF1FA89EFF1FBA9EFF1F86
:1088B000701F0100C09EFF1F349EFF1FA01F0100FC
:1088C000C81E0100CC1D0100642B0100542B0100C7
:1088D000BC1D0100241E0100AC1E01001C90FF1FE6
:1088E000A08AFF1F309EFF1F28B11028044BA8BF8D
:1088F000102018607047024B01201860704700BFBD
:10890000C49EFF1F38B50F4D2B78013B01381B0269
:10891000C4B203F47063200443F4404343F00C03F7
:1089200000F4FE00184305F071FD2868013860F07E
:108930003F00C0B204F098FD2046BDE8384004F086
:1089400093BD00BFC49EFF1F70B5124D2B78013B35
:108950001B0203F47063064643F4304308063204F6
:1089600000F0FE4043F00B03034302F4FE00184303
:108970000C4605F04BFD2868013860F04F00C0B28E
:1089800004F072FD304604F06FFD2046BDE87040F3
:1089900004F06ABDC49EFF1F70B5124D2B78013BD9
:1089A0001B0203F47063064643F4104308063204C6
:1089B00000F0FE4043F00903034302F4FE001843B5
:1089C0000C4605F023FD2868013860F06F00C0B246
:1089D00004F04AFD304604F047FD2046BDE87040F3
:1089E00004F042BDC49EFF1F38B5104D2B78013BEB
:1089F0001B0203F47063044643F41043000443F085
:108A0000090300F4FE00184305F000FD2868013852
:108A100060F06F00C0B204F027FD204604F024FD92
:108A20000020BDE8384004F01FBD00BFC49EFF1FFA
:108A300038B50E4D2B78013B1B0203F470630446DE
:108A400043F45043000443F00D0300F4FE001843C8
:108A500005F0DCFC2868013860F02F00C0B204F09B
:108A600003FD2046BDE8384004F0FEBCC49EFF1F55
:108A700008B5002005F094FD0028FAD108BD00BF1C
:108A800008B564210720FFF75FFF7F210B20BDE8B9
:108A90000840FFF759BF00BF10B500217B20FFF74A
:108AA00053FF0024E0B2FFF79FFF0134022004F0DF
:108AB0007BFB802CF6D110BD10B504464FF440600E
:108AC00004F082FC04F0DAFC2CB1102C044BA8BF9B
:108AD00010241C6010BD024B01241C6010BD00BF9F
:108AE000C49EFF1F10B5044641F0E00004F0BCFC3A
:108AF00004F07F0004F0B8FCC4F3C610BDE81040D9
:108B000004F0B2BC38B5134D2B78044641F6FF7221
:108B1000A0F50050824203F1FF33A8BF02461B02BA
:108B200002F5005203F47063100443F4604343F011
:108B30000E0300F4FE005204184302F0FE421043FC
:108B400005F064FC296801392046C9B2BDE8384007
:108B5000FFF7C8BFC49EFF1F38B504460D46F0207E
:108B600004F082FC35B1254414F8010B04F07CFCC0
:108B7000AC42F9D1F720BDE8384004F075BC00BF25
:108B800000B50B4B83B00246998818680090032A01
:108B9000ADF8041002D903B05DF804FB6846062165
:108BA0008DF80520FFF7D8FF03B05DF804FB00BF88
:108BB000D02B010000B50B4B024683B01868998892
:108BC0000090131F4C2BADF8041002D903B05DF8D0
:108BD00004FB684606218DF80520FFF7BDFF03B0B2
:108BE0005DF804FBD82B0100030203F4FE43C0F33D
:108BF000C6101843704700BF03784078DB0103F4C8
:108C00007E5300F07F001843704700BF82B002AA75
:108C1000114642F8040D002012F8013B03F07F03D7
:108C2000914243EA0020F7D102B07047003210B4FD
:108C300003884FF0010404FA01F418BF012202FA7C
:108C400001F123EA04020A43028010BC704700BF0E
:108C500070B5CEB20C46054603F038FE864203D00E
:108C60003146284603F04CFE0135284603F02EFE1F
:108C7000240A844205D021462846BDE8704003F00E
:108C80003FBE70BD38B5054603F020FE4FF000042E
:108C900060F30704681C03F019FE60F30F24A0B210
:108CA00038BD00BFF8B504460020FFF7EBFF002CED
:108CB00000F05F814FF4AF610220FFF7C9FF04208D
:108CC0004FF47A61FFF7C4FF0B2004F037FA002855
:108CD00040F09B864FF496610620FFF7B9FF4FF4F2
:108CE000FA610820FFF7B4FF4FF4FA610A20FFF79A
:108CF000AFFF40F6B8310C20FFF7AAFF4FF42F6109
:108D00002220FFF7A5FF40F6AC512420FFF7A0FF7B
:108D10007D212A20FFF79CFF0C210E20FFF798FFF2
:108D200001211020FFF794FF02211220FFF790FF8E
:108D300000211420FFF78CFF00211620FFF788FF89
:108D400002211820FFF784FF01211A20FFF780FF7E
:108D500001211C20FFF77CFF04211E20FFF778FF74
:108D600014212020FFF774FF01212620FFF770FF58
:108D700003212820FFF76CFF04212C20FFF768FF58
:108D800014212E20FFF764FF00213020FFF760FF41
:108D90000C213220FFF75CFF00213420FFF758FF41
:108DA00000213620FFF754FF00213820FFF750FF45
:108DB00000213A20FFF74CFF00213C20FFF748FF3D
:108DC00000213E20FFF744FF00214020FFF740FF35
:108DD00000214220FFF73CFF1F214420FFF738FF0E
:108DE00013214620FFF734FF0E214820FFF730FF04
:108DF00011214A20FFF72CFF0A214C20FFF728FF02
:108E000000214E20FFF724FF06215020FFF720FF0E
:108E100002215220FFF71CFF0C215420FFF718FFFE
:108E200000215620FFF714FF00215820FFF710FF04
:108E300001215A20FFF70CFF08215C20FFF708FFF3
:108E40000A215E20FFF704FF00216020FFF700FFEA
:108E500004216220FFF7FCFE01216420FFF7F8FEE9
:108E600000216620FFF7F4FE0B216820FFF7F0FEDB
:108E70007F216A20FFF7ECFE00216C20FFF7E8FE5F
:108E800000216E20FFF7E4FE00217020FFF7E0FED6
:108E900000217220FFF7DCFE00217420FFF7D8FECE
:108EA0001F217620FFF7D4FE13217820FFF7D0FE94
:108EB0000E217A20FFF7CCFE11217C20FFF7C8FE9F
:108EC0000A217E20FFF7C4FE1F218020FFF7C0FE8D
:108ED00013218220FFF7BCFE0E218420FFF7B8FE8D
:108EE00011218620FFF7B4FE0A218820FFF7B0FE8B
:108EF00000218A20FFF7ACFE00218C20FFF7A8FE9E
:108F000000219620FFF7A4FE00219820FFF7A0FE85
:108F100000219A20FFF79CFE05219C20FFF798FE78
:108F200006219E20FFF794FE0021A020FFF790FE6F
:108F30007F21A220FFF78CFE40F2A461A420FFF75E
:108F400087FE4FF4E161A620FFF782FE2821002072
:108F5000FFF77EFE0220FFF795FEB0F5805F034627
:108F600016D34FF4AF610220FFF772FE4FF4AF63E8
:108F70000EE04FF6FF7398423FF49CAE282840F075
:108F800050850220FFF77EFEB0F5805F0346E8D2F1
:108F9000D24A04201380FFF775FEB0F5805F0346C8
:108FA00080F07984CE4A06201380FFF76BFEA0F58F
:108FB0002F739BB2B3F57A6F024606D940F628218B
:108FC0000620FFF745FE40F62822C64B08201A80EF
:108FD000FFF758FEA0F52F739BB2B3F57A6F0246E8
:108FE00006D940F6E4410820FFF732FE40F6E4429D
:108FF000BD4B0A201A80FFF745FEA0F5FA739BB21D
:1090000040F6AC518B42024606D94FF4FA610A2071
:10901000FFF71EFE4FF4FA62B44B0C201A80FFF7E4
:1090200031FEA0F5FA739BB240F6AC518B4202467A
:1090300006D940F6B8310C20FFF70AFE40F6B832E8
:10904000AB4B0E201A80FFF71DFE1828034600F2D6
:109050003F84A84A10201380FFF714FE431E9BB2E2
:109060000F2B024604D901211020FFF7F1FD012248
:10907000A14B12201A80FFF705FE0A28034600F2D2
:1090800020849E4A14201380FFF7FCFD012803462C
:1090900004D900211420FFF7DBFD0023984A162095
:1090A0001380FFF7EFFD7F28034600F20384954A03
:1090B00018201380FFF7E6FD0528034600F2F4832D
:1090C000914A1A201380FFF7DDFD0C28034600F2B9
:1090D00033848E4A1C201380FFF7D4FD04280346F6
:1090E00000F223848A4A1E201380FFF7CBFD092853
:1090F000034600F21384874A20201380FFF7C2FD45
:109100004628034600F20384834A22201380FFF797
:10911000B9FDA0F5FA739BB240F6AC518B42024602
:1091200006D94FF42F612220FFF792FD4FF42F62F2
:109130007A4B24201A80FFF7A5FDA0F5FA739BB2A5
:1091400040F6AC54A342024604D921462420FFF73E
:109150007FFD2246724B26201A80FFF793FD7F2861
:10916000034600F2CE836F4A28201380FFF78AFD62
:109170000628034600F2BF836B4A2A201380FFF7BC
:1091800081FDA0F132039BB2B3F5967F024604D96C
:109190007D212A20FFF75CFD7D22644B2C201A8064
:1091A000FFF770FD0C28034600F29F83604A2E20D3
:1091B0001380FFF767FD1E28034600F290835D4A87
:1091C00030201380FFF75EFD0928034600F2168465
:1091D000594A32201380FFF755FD1E28034600F23E
:1091E0000684564A34201380FFF74CFD7F2803463F
:1091F00000F2F783524C36202380FFF743FD7F288F
:10920000034600F2E88338206380FFF73BFD7F28A8
:10921000034600F2DA833A20A380FFF733FD7F286C
:10922000034600F2CC833C20E380FFF72BFD7F2830
:10923000034600F2BE833E202381FFF723FD7F28F3
:10924000034600F2B08340206381FFF71BFD7F28B7
:10925000034600F2A2834220A381FFF713FD394D9C
:1092600028804420FFF70EFD3028034600F28F834C
:10927000354A46201380FFF705FD3028034600F2EB
:109280008083324C48202380FFF7FCFC30280346C3
:1092900000F271834A206380FFF7F4FC3028034614
:1092A00000F263834C20A380FFF7ECFC30280346D8
:1092B00000F255834E20E380FFF7E4FC01280346CB
:1092C00004D900214E20FFF7C3FC0023204A502080
:1092D0001380FFF7D7FC431E3CE000BF289CFF1F14
:1092E000E49DFF1FA89DFF1FBC9DFF1F889DFF1FC2
:1092F000C09BFF1F989BFF1F3C9DFF1F729DFF1F80
:109300001E9CFF1F9C9BFF1F2E9CFF1FD89BFF1FB7
:10931000D29BFF1FC89BFF1FCC9DFF1F349DFF1FCB
:10932000309DFF1FC09DFF1F949DFF1FDC9DFF1FF1
:10933000AE9BFF1F189CFF1FF09DFF1FBE9DFF1FD0
:10934000009DFF1FB89BFF1FBA9BFF1F989DFF1F2B
:10935000D09BFF1F9BB20B2B024604D90621502045
:10936000FFF776FC0622CF4B52201A80FFF78AFCCB
:109370000428034600F2ED82CB4A54201380FFF705
:1093800081FC431E9BB21D2B024604D90C215420A4
:10939000FFF75EFC0C22C54B56201A80FFF772FCCB
:1093A0000128034604D900215620FFF751FC002371
:1093B000BF4A58201380FFF765FC7F28034600F260
:1093C000C282BC4A5A201380FFF75CFC431E9BB24A
:1093D000092B024604D901215A20FFF739FC01224A
:1093E000B54B5C201A80FFF74DFC431E9BB2102B3F
:1093F000024604D908215C20FFF72AFC0822AF4B63
:109400005E201A80FFF73EFC431E9BB21D2B0246D6
:1094100004D90A215E20FFF71BFC0A22A84B60201A
:109420001A80FFF72FFC0228034600F22282A54A89
:1094300064201380FFF726FC0128034604D901218C
:109440006420FFF705FC01239F4A62201380FFF789
:1094500019FCC31E9BB2012B024604D904216220D1
:10946000FFF7F6FB0422994B66201A80FFF70AFCEF
:109470007F28034600F2F781954A68201380FFF7A2
:1094800001FC7F28034600F2E881924A6A2013809B
:10949000FFF7F8FB7F28034600F2D9818E4A6C2043
:1094A0001380FFF7EFFB0228034600F2CA818B4AC4
:1094B0006E201380FFF7E6FB1928034600F2BB81FC
:1094C000874A70201380FFF7DDFB0228034600F275
:1094D000AC81844A72201380FFF7D4FB0628034630
:1094E00000F29D81804A74201380FFF7CBFB042893
:1094F000034600F28E817D4A8A201380FFF7C2FB6B
:109500000A28034600F27F81794A8C201380FFF7F6
:10951000B9FB0428034600F27081764A9820138034
:10952000FFF7B0FB0128034604D900219820FFF77C
:109530008FFB0023704A9A201380FFF7A3FB0128BA
:10954000034604D900219A20FFF782FB00236B4ACF
:1095500096201380FFF796FB0B28034600F2478105
:10956000674A9C201380FFF78DFB831E9BB2032B61
:10957000024604D905219C20FFF76AFB0522614BB6
:1095800076201A80FFF77EFB3028034600F22981FF
:109590005D4A78201380FFF775FB3028034600F200
:1095A0001A815A4C7A202380FFF76CFB302803463F
:1095B00000F20B817C206380FFF764FB30280346B8
:1095C00000F2FD807E20A380FFF75CFB302803467D
:1095D00000F2EF808020E380FFF754FB3028034641
:1095E00000F2E1804A4A82201380FFF74BFB3028CB
:1095F000034600F2D280474C84202380FFF742FBD1
:109600003028034600F2C38086206380FFF73AFBD0
:109610003028034600F239818820A380FFF732FB0F
:109620003028034600F22B81A020E380FFF72AFBBD
:109630000128034604D90021A020FFF709FB0023DD
:10964000354A9E201380FFF71DFBC31E9BB20C2BD7
:10965000024604D906219E20FFF7FAFA06222F4B74
:10966000A2201A80FFF70EFB431E9BB27E2B024600
:1096700004D97F21A220FFF7EBFA7F22284BA420F8
:109680001A80FFF7FFFAA0F5AF639BB2B3F5167F20
:10969000024647D940F2A461A420FFF7D9FA40F26C
:1096A000A4623FE02089FF1F2E89FF1FA489FF1FAE
:1096B0000C9CFF1FC49DFF1F949BFF1FA889FF1FC9
:1096C0002C89FF1F2C9DFF1F909DFF1FDA9BFF1F02
:1096D000CE9DFF1F049CFF1FCA9BFF1F889BFF1F7F
:1096E000129EFF1F209DFF1FEC9DFF1FB49DFF1FBB
:1096F0003E9DFF1F2A9DFF1FEA9BFF1F109CFF1F1F
:109700007C9DFF1FB09BFF1FC29BFF1F109DFF1F73
:10971000C49BFF1F189DFF1FA09DFF1F9089FF1F67
:10972000C29DFF1FD54BA6201A80FFF7ABFAA0F50C
:10973000AF639BB2B3F5167F06D9A6204FF4E16163
:10974000FFF786FA4FF4E1602B88DFF850E3CC4F47
:10975000CC4ACD4DCD4ECE4CCE4903F0010CAEF8E7
:1097600000C0C3F3400EA7F800E0C3F380071780E2
:10977000C3F3C007C84A2F70C3F30017C3F34015E3
:10978000C3F38013378025800B801080F8BD0E2135
:109790008420FFF75DFA0E2336E713218220FFF7BE
:1097A00057FA132327E71F218020FFF751FA1F23C1
:1097B00018E70A217E20FFF74BFA0A230AE7112156
:1097C0007C20FFF745FA1123FCE60E217A20FFF7F3
:1097D0003FFA0E23EEE613217820FFF739FA132320
:1097E000DFE61F217620FFF733FA1F23D0E60021A2
:1097F0009620FFF72DFA0023B2E600218C20FFF718
:1098000027FA002389E600218A20FFF721FA0023A6
:109810007AE600217420FFF71BFA00236BE6002193
:109820007220FFF715FA00235CE600217020FFF795
:109830000FFA00234DE600216E20FFF709FA0023FE
:109840003EE600216C20FFF703FA00232FE67F217C
:109850006A20FFF7FDF97F2320E60B216820FFF740
:10986000F7F90B2311E600216620FFF7F1F9002339
:1098700002E600216020FFF7EBF90023D7E50A217B
:109880008820FFF7E5F90A23CEE611218620FFF7AD
:10989000DFF91123C0E64FF47A610420FFF7D8F90D
:1098A0004FF47A63FFF77EBB02211820FFF7D0F94F
:1098B000022305E400211620FFF7CAF90023FFF771
:1098C000F6BB02211220FFF7C3F90223FFF7D9BB31
:1098D0000C210E20FFF7BCF90C23FFF7BABB1421B3
:1098E0002E20FFF7B5F9142369E404212C20FFF79B
:1098F000AFF904235AE403212820FFF7A9F9032331
:109900003AE401212620FFF7A3F901232BE41421D7
:109910002020FFF79DF91423FFF7F6BB04211E203A
:10992000FFF796F90423FFF7E6BB01211C20FFF7A0
:109930008FF90123FFF7D6BB01211A20FFF788F921
:109940000123FFF7C6BB00215820FFF781F9002350
:1099500037E502215220FFF77BF902230CE50A21AB
:109960004C20FFF775F90A23A4E411214A20FFF7E0
:109970006FF9112396E40E214820FFF769F90E23B1
:1099800088E413214620FFF763F9132379E41F21AC
:109990004420FFF75DF91F236AE400214020FFF710
:1099A00057F9002357E400213E20FFF751F9002327
:1099B00049E400213C20FFF74BF900233BE4002160
:1099C0003A20FFF745F900232DE400213820FFF766
:1099D0003FF900231FE400213620FFF739F9002367
:1099E00011E400213420FFF733F9002302E40C21B5
:1099F0003220FFF72DF90C23FFF7F3BB00213020B5
:109A0000FFF726F90023FFF7E3BB40F628210620E5
:109A1000FFF71EF940F6E4410820FFF719F9FFF7B8
:109A200063B917287FF646A919287FF6B5A91B2820
:109A30007FF6D2A91C283FF4E7A91E287FF6ECA9DF
:109A40001F283FF4F1A920283FF40AAA21283FF457
:109A500013AA22283FF418AA23283FF421AA242875
:109A60003FF452AA25283FF457AA26283FF458AAC3
:109A700027287FF46BAAFFF75BBA00BF2C9CFF1F5F
:109A8000E89BFF1F1A9CFF1F239DFF1F2E9DFF1F9A
:109A9000929DFF1F449DFF1FAA9DFF1F7E9DFF1FDC
:109AA000F8B5B92006F0C8FB204B214A054603CB88
:109AB0001368C5F803001A0CA820C5F807102B80FE
:109AC000AA70FFF791F82E46002426F80B0FA0B2DB
:109AD000FFF7D8F8FFF788F80234A82C26F8020F11
:109AE000F5D16C1E05F1B4064FF0FF3014F8013FBC
:109AF000082758400F4B40F300017A1E0B4012F02C
:109B0000FF0783EA5000F5D1B442EFD1C043FFF71D
:109B10007DF83A46C5F8B500B921284604F0C4FCE2
:109B20002846BDE8F84006F08FBB00BFE42B0100DB
:109B3000E02B01002083B8EDF0B50E4B0E4C05462E
:109B400093E8070085B024682E88AD7801AB83E8E0
:109B50000700270C184600220B21ADF804408DF8B1
:109B60000670ADF80C608DF80E5004F09DFC05B049
:109B7000F0BD00BFF02B0100E02B0100F0B5124B4F
:109B8000124D1E68124F0FCD87B06C460FC495E87A
:109B9000030044F8040B38683B79CDF80D00320C13
:109BA000282021808DF802208DF81130ADF800605A
:109BB000FFF71AF80022ADF80B001221684604F0F6
:109BC00073FC07B0F0BD00BFE02B0100FC2B0100CF
:109BD000F0200100002004F0E3BC00BF02F02EBE24
:109BE00070B5124C82B00025402306462946204617
:109BF000009301958023202201F072FE2022294645
:109C0000204602F031FA2046012102F037FA3046B0
:109C100007F0B6F831460246204602F0BFFB204668
:109C200002B0BDE8704001F041BC00BF409EFF1F84
:109C3000F0B5B82983B075D90546441E00F1B406C5
:109C40004FF0FF3014F8012F08275040404A40F3EE
:109C500000017B1E0A4013F0FF0782EA5000F5D195
:109C6000B442EFD1C043FEF7D1FF0146D5F8B500AD
:109C70000190019A914202D0B2F17F2F0BD105F1F0
:109C80000B00FEF7B9FFA8280BD03248FFF7A8FF5A
:109C9000002003B0F0BD3048FFF7A2FF384603B004
:109CA000F0BD05F10D00FEF7A7FF282840D10024E4
:109CB00040F6AC5613E004281AD0062821D0082814
:109CC0001FD00A2828D00C2822D1A1F5FA7292B20E
:109CD000B24201D8FEF7BCFF0234A82C0ED004F12A
:109CE0000D002844FEF788FF022C0146A0B2E2D105
:109CF000B1F5805FEED30234A82CF0D1012003B07F
:109D0000F0BDA1F52F7292B2B2F57A6FE4D8E1E717
:109D1000222801D0242811D1A1F5FA7292B2B242C0
:109D2000DAD8D7E70D48FFF75BFF002003B0F0BD9E
:109D30000B48FFF755FF002003B0F0BD2A28C9D11A
:109D4000A1F1320292B2B2F5967FC5D8C2E700BF48
:109D50002083B8ED402C01002C2C0100142C0100B4
:109D6000542C010003290CD970B5461C82B005465D
:109D70000C46304603222A4907F070F810B102B0B1
:109D800070BD70470B2C05D905222649281D07F008
:109D900065F840B12448FFF723FF244802B0BDE82E
:109DA0007040FFF7C9BE05F10901032201A807F0C1
:109DB000A5F801A803221E4907F050F8D8B10322E4
:109DC0001C4901A807F04AF808B301A803221A4960
:109DD00007F044F8B0B91948FFF702FFA11E89B295
:109DE0003046FFF725FF0028C9D0154802B0BDE86E
:109DF0007040FFF7F5BE1348FFF7F2FEFFF750FE85
:109E00001148F3E71148FFF7EBFE1148C6E7114888
:109E1000FFF7E6FE02B0BDE87040FFF7AFBE00BF3F
:109E2000E02B0100002101006C2C0100802C0100BE
:109E3000842C0100AC2C0100C42C0100C82C0100B2
:109E4000DC2C0100882C01009C2C0100F02C01006E
:109E5000042D0100B02C01002DE9F043174D2B68B3
:109E600083B081460F469046F3B1154E34880A19E7
:109E700092B218461146328006F05CFD28603A46E0
:109E80004946204402F06CFDB8F1000F09D031883A
:109E90002868FFF767FF286806F0D6F900232B60D3
:109EA000338003B0BDE8F083054E0193084631804E
:109EB00006F0C2F9019B28601C46E0E7CC9EFF1F1C
:109EC000C89EFF1F10B51F4C4FF4FA70FBF7CCFF74
:109ED000204601F0DFF900221146204602F0C4F8C6
:109EE0002046012102F0CAF82046002102F0C0F805
:109EF0000B221549204602F051FA204602F064FA7E
:109F00000F221249204602F049FA204602F05CFA7C
:109F10000F490722204602F041FA204602F054FA87
:109F2000204601F0C3FA0B4B0B4A1A604FF4FA704B
:109F3000FBF79AFFFFF722FE0848BDE81040FFF745
:109F40004FBE00BF409EFF1F082D0100142D0100D1
:109F5000242D010084A0FF1F599E00002C2D01001C
:109F60000020704790F8392090F83800101A704798
:109F700090F8383090F839209A4205D95A1C034499
:109F800080F83820187E70474FF0FF30704700BFD0
:109F900090F8383090F839209A4286BF1B18187E06
:109FA0004FF0FF30704700BF704700BF38B505461F
:109FB000B0F85E0090B195F85D301446C3F121020F
:109FC00094420CD805F13B001844224602F0C8FC2C
:109FD00095F85D30234485F85D30204638BD01207A
:109FE00014462871EEE700BFB0F85E306BB190F810
:109FF0005D30202B07D8C218013380F85D30012076
:10A0000082F83B107047012303710020704700BFA6
:10A010000023426980F8383080F8393080F85C30AD
:10A0200080F85D3080F85E3080F85F3006CA30B46A
:10A030000D68046943662A4383660A60A370426917
:10A0400090F861301649146813441D7A5B7B01EB6C
:10A05000C5051B026D6803F4E06343F064032B60E5
:10A0600090F8623013449D7CDB7D01EBC5011B023F
:10A07000496803F4E06343F064030B6021685368AC
:10A08000194205D0036927225A70036904229A7184
:10A09000036920225A71036980229A7030BC70478C
:10A0A0006038010043690CCB12681A420CD0094B8E
:10A0B00099420AD9084B9942036994BF1A220D228A
:10A0C0005A70036904229A717047036927225A70F3
:10A0D000F7E700BF7F1A06003F420F0010B5026984
:10A0E000D378DBB2D90604463DD510215806D1708D
:10A0F00038D503F0040303F0FF02002B51D03D4993
:10A10000626E00230B7084F85D30002A5BD09047AC
:10A1100094F85D30002B56D02369D0229A702369C1
:10A1200094F83B201A712369012284F85C200222F2
:10A13000DA7010BD304B84F860009C424AD02F4B3F
:10A140009C4252D094F8391013791F29DBB207D8FA
:10A150002848007820B16018013184F8391003765E
:10A160000223D37010BD5906C3D4917801F01001B9
:10A1700001F0FF000029DDD013F001031ED194F897
:10A180005C1094F85D00884281BF4B1C091984F86B
:10A190005C3091F83B3013712369D0229A702269A8
:10A1A000DEE7236984F83920C0229A702369114AB6
:10A1B0001979012111700222DA7010BDC023937049
:10A1C00022691379CCE70122002384F85D2084F80A
:10A1D0003B30A1E7626994F86130094913440322D6
:10A1E000187A02F043FD2269ACE7626994F86130A5
:10A1F0000449F3E7D09EFF1F6890FF1FD490FF1F14
:10A2000065A2000071A200000369DB7803F020035F
:10A2100073B190F860300133DBB2012B80F860300D
:10A220001AD9426990F861301344187A02F09ABD45
:10A2300070B5426903F0FF0590F86130134404469D
:10A24000187A02F08FFDA36E5BB184F8385094F851
:10A250003900BDE87040184790F85F30002BE0D01F
:10A26000704770BD0148FFF7CFBF00BF6890FF1F68
:10A270000148FFF7C9BF00BFD490FF1F2DE9F04789
:10A28000374FDFF8E0903B68026982B006460093E2
:10A29000DDF800800021A025D3789B065BD53B68C4
:10A2A0000193019BC8EB03030F2BF5D949B1102B88
:10A2B000F2D000209070336980229A7002B0BDE81D
:10A2C000F087726996F8613013440521187A02F01C
:10A2D00043FF726996F861301344012193F812A08C
:10A2E000504602F039FF09240021504602F020FFB9
:10A2F0002B46013BFDD10121504602F019FF2B46B0
:10A30000013BFDD1013CEFD1706996F86110014429
:10A310004FF4A0720C7A4B7B09EBC4011B02496815
:10A3200003F4E06343F064030B6096F86230034487
:10A33000997CDB7D09EBC1011B02496803F4E063F2
:10A3400043F064030B60013AFDD13269D3789B0678
:10A350004FF00101A3D4012002B0BDE8F08700BF97
:10A36000F89EFF1F60380100F0B503691222DA7011
:10A370000269937803F0200385B004460D46002B54
:10A380005ED0B42393703C4922690B680093009E11
:10A3900005E00B680193019B9B1B042B42D8D378EB
:10A3A00003F0200303F0FF00002BF2D094F85D309F
:10A3B000002B31D04FF0000E4FF0020C04EB0E03D7
:10A3C00093F83B3013710B680393039F206907E0F8
:10A3D0009B060DD50B680293029BDB1B052B28D82F
:10A3E000C378DBB203F0020202F0FF06002AEFD0CE
:10A3F00080F803C02669F378DBB2DF0632462DD43D
:10A400009F062BD5DB0731D40EF1010E94F85D3099
:10A410005FFA8EFE7345D1D800201DBB002384F85F
:10A420005E3004E09070236980229A70042005B0A9
:10A43000F0BD86702369802204209A7005B0F0BDBB
:10A4400003F0FF06FFF71AFF10B9042005B0F0BDB6
:10A45000236984F85F60B0229A7094E78023B37018
:10A460000420DAE726698023B370D7E7BEF1000F36
:10A470000CBF02200320F6E7F89EFF1F2DE9F041F4
:10A4800006690025122780F8385080F83950F77097
:10A49000D0F810C09CF802E00EF0200E88B0044600
:10A4A000884615461E46BEF1000F49D0B4238CF8ED
:10A4B0000230784B21691A680092DDF800E006E06E
:10A4C0001A6801920198CEEB0000042830D8C878B1
:10A4D00000F0200000F0FF070028F1D04FEA48020A
:10A4E00042F00102D2B20A711A680292DDF808E065
:10A4F000206906E01A6803920399CEEB0101052951
:10A500002AD8C17801F0020101F0FF070029F1D03B
:10A510004FF0020C80F803C02269D17811F01107C6
:10A5200022D12DBB002E0CBFA0238023937003E00B
:10A530008F70236980229A70384608B0BDE8F08198
:10A540000EF0FF07FFF79AFE0028F5D0236984F884
:10A550005F70B0229A70ACE787702369802238461A
:10A560009A7008B0BDE8F081802393700027E3E77C
:10A57000012D75D0A021917021690A79BE466746E8
:10A580004FF0A80C1A680492049805E01A68059226
:10A59000059A121A052A4AD8CA7802F0020202F075
:10A5A000FF08002AF2D0CF702169CA78D2B212F027
:10A5B000100F08465AD1920658D5013DEDB2012D33
:10A5C00049D0BEF11F0F3BD90A79012DDAD11A68A3
:10A5D0000692069D05E01A680792079A521B052A03
:10A5E00046D8C27802F0020202F0FF01002AF2D03F
:10A5F0000223C3702269D378DBB2D9063AD49B0612
:10A6000034D5B023BEF11F0F93703FD8226904EBFD
:10A610000E0312791A760EF1010E5FFA8EFE16B154
:10A62000236980229A7084F839E0774684E781F8BC
:10A630000280236980229A70774684F839E07BE7AC
:10A6400004EB0E0291F8048082F818800EF1010EDE
:10A650005FFA8EFEB9E781F802C021690846B0E7CB
:10A66000A82191702069BE460279B0E7774663E77A
:10A670008170DEE71021A023D170013BFDD122695A
:10A68000937803F0F7037746937055E723691B79B6
:10A69000C5E700BFF89EFF1F0148FFF71FBD00BFC1
:10A6A0006890FF1F0148FFF719BD00BFD490FF1F3E
:10A6B000704700BF38B5144C037801225B00054693
:10A6C000204684F83B3084F85E2084F85D20FFF754
:10A6D0008BFC20460021FFF747FE0B4C2978012315
:10A6E00020461A46FFF7CAFE0128F6D194F8383002
:10A6F00094F839209A4205D9E218013384F83830A9
:10A70000107E38BDFF2038BD6890FF1F38B51B4C48
:10A71000037801225B000546204684F83B3084F82C
:10A720005E2084F85D20FFF75FFC20460021FFF7E4
:10A730001BFE124C2978204601230222FFF79EFEC1
:10A740000228F6D194F8382094F839108A420FD2B2
:10A75000531CDBB2A018994284F83830007E0AD925
:10A76000234402321B7E84F8382040EA032038BD9F
:10A770004FF6FF7038BD40F47F4038BD6890FF1F32
:10A780000C2901D9002070470231490001F0FE0177
:10A79000FFF7BCBF70B50C4C0378164601255B0073
:10A7A000204684F83B3084F85E5084F85D50FFF713
:10A7B0001BFC31462046FFF717FC29462046BDE822
:10A7C0007040FFF7D1BD00BF6890FF1FF8B5054688
:10A7D0000F461646412421463A462846FFF7DAFF3F
:10A7E000611C0234C9B232462846E4B2FFF7D2FFF8
:10A7F000592CF0D1F8BD00BF38B504460D46354898
:10A80000FFF706FC6322802120462570FFF7C2FF78
:10A81000012002F0C9FC204600225E21FFF7BAFFAA
:10A8200020465D21FFF746FF242801D0002038BDD7
:10A83000204606220C21FFF7C9FF204601222B21CA
:10A84000FFF7A8FF204601222C21FFF7A3FF204697
:10A850000E222D21FFF79EFF204600222E21FFF71A
:10A8600099FF204601222F21FFF794FF2046052261
:10A870003021FFF78FFF204601223121FFF78AFFA9
:10A88000204600223221FFF785FF20460022332197
:10A89000FFF780FF204600223421FFF77BFF204690
:10A8A00000223521FFF776FF204600225B21FFF7CB
:10A8B00071FF204610225C21FFF76CFF204620220A
:10A8C0005D21FFF767FF20468F225E21FFF762FFC1
:10A8D000012038BD6890FF1F10B4047F4160022C36
:10A8E000C26002D010BC01F0D7BB836810BC18470F
:10A8F00090E80C00F0B41C6859682568164F174E94
:10A9000029432160164D17491760D6601561116003
:10A91000417A154A5C180A3194F8244053F82150C2
:10A9200002EBC40149680D60017A5C1803EB8101F8
:10A93000247ECD6902EBC40149680D60817A581804
:10A9400003EB810390F83000596B02EBC002F0BCBE
:10A9500053681960704700BF01401F0001100038A4
:10A960000110007800001F8060380100704700BFB0
:10A97000F0B50C1EBDF8146034DBB0F9067019197F
:10A98000B942C4BF3B1B1BB2002BA6461CDD002AEC
:10A990001146B8BFD11D02F00705CC10826A012014
:10A9A00007FB04E1A840012E0A44C0B21ED00CD31C
:10A9B000022E09D1013B12FA83F3013A12F8011F6A
:10A9C00041409A421170F9D1F0BDC043013B12FAE7
:10A9D00083F3C0B2013A12F8011F01409342117093
:10A9E000F9D1F0BD23441BB20024C6E7013B12FAA3
:10A9F00083F3013A12F8011F01439A421170F9D111
:10AA0000F0BD00BFF8B50D1E0EDB14461F4606460E
:10AA100001F03AFBA84207DD002C05DB304601F0CF
:10AA200037FBA04201DCF8BDF8BD304601F02AFB3F
:10AA3000022853D003284BD0012806D16540F38863
:10AA40006C406540013B5D1B2DB2012F03D02AD322
:10AA5000022F14D0F8BD002C2246B6F90630B06A99
:10AA6000B8BFE21D42F3CF0202FB035504F0070416
:10AA7000435D012101FA04F41C434455F8BD002C48
:10AA80002246B6F90630B06AB8BFE21D42F3CF02E3
:10AA900002FB035504F00704435D012101FA04F4AD
:10AAA0005C404455F8BD002C2246B6F90630B06A29
:10AAB000B8BFE21D42F3CF0202FB035504F00704C6
:10AAC000435D012101FA04F423EA04044455F8BD6E
:10AAD0003389013B591B25460CB2B6E7F188328910
:10AAE0000139013A4D1B141B2DB224B2ADE700BF52
:10AAF0002DE9F041079E9DF91880089D04461F46E8
:10AB000000F0C0FF0D4B0E480E4984F83380FF2241
:10AB1000002F08BF1F4684F82F20002384F8302020
:10AB200084F8312084F832202060A665E5656762EC
:10AB300061652362A3622046BDE8F0816890FF1F33
:10AB4000B82D01000110013810B50446806A034B8E
:10AB5000236008B105F078FB204610BDB82D010038
:10AB6000F8B5436ADBB190F82C200125AA4083F8A0
:10AB70003B2083F85E5083F85D500446406A0368CA
:10AB80000E461B6800219847606A036831461B68BF
:10AB900098472946606ABDE8F840FFF7E5BBC26BFD
:10ABA000C56C1368046A23EA050313604CB122687C
:10ABB0004FF00043D3625163D36A002BFCDA936BEE
:10ABC000F8BD836B466B0825802410E03768426C23
:10ABD0003A4332601F68826C3A431A601A68876C85
:10ABE000013D22EA07024FEA54041A6007D02142CD
:10ABF000ECD13268476C22EA07023260EAE7F8BD1E
:10AC000070B50446406A0D4600282BD0A16DFFF7B1
:10AC100049FA002D20460CBFA621A721FFF7A0FF6F
:10AC2000606A20B1E16DBDE87040FFF73BBA216C6E
:10AC3000226D0868236A02430A6093B1DA7A82B10E
:10AC4000D00703D5224A99691160DA7A910703D5B2
:10AC5000204AD9691160DA7A520702D51E4A1B6A66
:10AC6000136070BD236A002B2BD0D97A626DE1B1DD
:10AC700072B6D97ACE0706D51848D9680668314029
:10AC800099610160D97A880706D51548196906685F
:10AC90003140D9610160D97A4E0705D5114859690B
:10ACA000066831401962016062B61B68D96891423A
:10ACB00007D00D4818600D49DA6042F080401861F5
:10ACC0001960226C216D136823EA01031360A0E769
:10ACD00000E100E004E100E008E100E080E100E0E4
:10ACE00084E100E088E100E001403F0000003F8097
:10ACF000436A2DE9F04105460E469046002B3ED0B2
:10AD000090F82C100124A14083F83B1083F85E409A
:10AD100083F85D40406A036800211B6808F1FF3733
:10AD20009847FFB2B8F1000F23D03744A046013E48
:10AD3000686A16F8011F03681B6898470134B74218
:10AD4000E4B216D0202CF3D10121686AFFF70CFB86
:10AD500095F82C206B6A520083F83B2083F85E80C4
:10AD600083F85D80686A036800211B6898470124A6
:10AD7000DEE7686A0121BDE8F041FFF7F5BAC26B72
:10AD8000C16C136823EA010306EB080413604FF05B
:10AD90000048A6420ED02B6A16F801EB63B11A6880
:10ADA000C2F82C80C2F834E0D36A002BFCDAA64249
:10ADB000936BF0D1BDE8F081AB6BD5F834C00820BF
:10ADC0008021DCF800206F6C1EEA010F14BF3A43AB
:10ADD000BA43CCF800201A68AF6C3A431A601A687C
:10ADE000AF6C013822EA07024FEA51011A60E8D13C
:10ADF000CFE700BF70B50446406A0D46002828D052
:10AE0000A16DFFF74FF920462946FFF7A9FE606ABA
:10AE100020B1E16DBDE87040FFF744B9216C226DAF
:10AE20000868236A02430A6093B1DA7A82B1D007D4
:10AE300003D5234A99691160DA7A910703D5214A2B
:10AE4000D9691160DA7A520702D51F4A1B6A13606A
:10AE500070BD236A002B2BD0D97A626DE1B172B636
:10AE6000D97ACE0706D51948D96806683140996164
:10AE70000160D97A880706D51548196906683140F6
:10AE8000D9610160D97A4E0705D51248596906681B
:10AE900031401962016062B61B68D968914207D0DF
:10AEA0000D4818600D49DA6042F080401861196061
:10AEB000226C216D136823EA01031360A3E700BF2E
:10AEC00000E100E004E100E008E100E080E100E0F2
:10AED00084E100E088E100E001403F0000003F80A5
:10AEE0002DE9F041044686B0806A9DF830801E4608
:10AEF0000F461546B4F90830002800F04281DA1DEB
:10AF000048BF03F10E02B4F90630D21003FB02F27F
:10AF1000002105F0BDFCB4F90820202A00F392803E
:10AF2000B4F90610A34B0120203A733902EBD27218
:10AF300001EBD1714FF0200E029073208DE801409B
:10AF400042F34F0241F34F01204600F051FE606A88
:10AF500084F82D70002800F04D81002D40F08A808B
:10AF6000B4F90830202B14BF3D253C2584F82C5023
:10AF7000B8F1000F40F0858006B394F93300002843
:10AF800018DBC0B2012102F0E7F8012194F8330088
:10AF900002F0CEF8012002F007F9002194F8330006
:10AFA00002F0C6F80A2002F0FFF8012194F83300FD
:10AFB00002F0BEF8606A002800F08280A16DFFF701
:10AFC00071F804227C492046FFF792FE217A01396C
:10AFD000C9B22046FFF7C4FD784904222046FFF796
:10AFE00087FE94F92D30012B14BF14211021204627
:10AFF000FFF7B6FD042272492046FFF779FEB4F947
:10B000000630802B00F09280602B00F0A680D921C2
:10B010002046FFF7A5FD94F92D30012B14BFF12137
:10B0200022212046FFF79CFD204606226549FFF7B6
:10B030005FFE606A50B3E16DFFF734F8012006B09F
:10B04000BDE8F081B4F906105F4B0120403A523957
:10B050004FF0400E029002EBD272522001EBD17100
:10B060008DE8014042F34F0241F34F01204600F0CA
:10B07000BFFD6CE76DB284F82C50B8F1000F3FF4BF
:10B080007BAFFEF7C5FF002E94D076E7216C226DD2
:10B090000868236A02430A6073B1DA7A62B1D007A2
:10B0A00003D54A4A99691160DA7A91077CD452072C
:10B0B00002D5474A1B6A1360012006B0BDE8F08143
:10B0C000236A002B2BD0D97A626DE1B172B6D97A9E
:10B0D000CF0706D53F48D9680568294099610160C6
:10B0E000D97A8E0706D53C48196905682940D96187
:10B0F0000160D97A4D0705D5384859690568294056
:10B100001962016062B61B68D968914207D0344861
:10B1100018603449DA6042F0804018611960226C8E
:10B12000216D136823EA010313604AE7B4F908307C
:10B13000202B00F08680402B7FF469AF2A492046FF
:10B140000322FFF7D5FD94F92D30012B14BFCF2139
:10B150009F212046FFF704FD59E7B4F90830102B72
:10B160007FF455AF214920460322FFF7C1FD94F932
:10B170002D30012B14BFAF2110212046FFF7F0FC2A
:10B1800045E7DA1D48BF03F10E02B4F90630D210CC
:10B1900003FB02F21046059205F04EF8A06200286B
:10B1A0003FF44DAF059AB3E6114AD9691160DA7AD6
:10B1B0007DE700BF102E0100F02F0100F42F0100E9
:10B1C000F82F0100FC2F01000430010000E100E035
:10B1D00008E100E080E100E084E100E088E100E0D7
:10B1E00001403F0000003F800C2E0100C4320100EE
:10B1F00004E100E0012194F83100244F01F0ACFF9C
:10B2000094F83200012101F0A7FF94F9312094F95C
:10B21000323057F83220E26357F83330206A236423
:10B220000125E56425651A682A431A6078B1B8F1EA
:10B23000000F3FF428AFFFF75BFB002E3FF4BAAEE0
:10B240009BE6042212492046FFF752FDDFE629461D
:10B2500094F82F0001F080FF294694F8300001F0A7
:10B260007BFF94F92F2094F9303057F83220626335
:10B2700057F833306564A5641A68A36322F00102AD
:10B280001A60002E3FF496AE77E600BF60380100EA
:10B29000082E0100B0F90820D31D48BF02F10E03AB
:10B2A000B0F90620806ADB1002FB03F2002105F0F2
:10B2B000EFBA00BFF0B50029BDF814502EDBB0F98D
:10B2C0000660B1422ADA002A59DBB0F90870144648
:10B2D0001C44BC42C4BFBB1A1BB2002B1EDDD2B241
:10B2E000D408D0F828E016FB041112F00702DBB2F4
:10B2F0000EEB010421D0C2F10807FAB2374F934296
:10B30000BF5C0CD2C3EB020CFF2646FA0CF6012DF3
:10B3100007EA06073FD005D3022D36D0F0BD012D38
:10B3200039D030D21EF8016026EA07070EF8017006
:10B330009342F3D3B0F906100C449A1AD2B2072AFA
:10B3400010D9022D36D0002D14BFFF26002613463B
:10B350002670083BB0F90610DBB2072B0C44F7D877
:10B3600002F00702002AD9D01D4B012D9B5C1DD095
:10B3700017D3022DD2D1227853402370F0BD13444D
:10B380001BB20022A1E7022D25D11EF801607740F3
:10B390000EF80170CCE71EF8016037430EF801701B
:10B3A000C6E7227822EA03032370F0BD2278134314
:10B3B0002370F0BD11462378DB4323700839B0F9C0
:10B3C0000630C9B207291C44F5D812F00702A5D0EF
:10B3D000034B9B5CCFE73444AFE700BFA82D0100CF
:10B3E000982D010070B4C47DBDF80C50022C18D00B
:10B3F000032C1FD0012C0BD0002A03DBB0F908402E
:10B40000944201DC70BC7047039570BCFFF7B0BA82
:10B41000C4880395013CA41A0A4621B270BCFFF708
:10B4200049BF0689C488013E641AB21AE41A12B2EE
:10B4300021B2E1E704890395E41A641A114622B2A5
:10B4400070BCFFF737BF00BF70B4C57DBDF80C609E
:10B45000022D1AD0032D12D0012D03D0039670BCFB
:10B46000FFF728BFC488E41AA41A0A4621B2002AAA
:10B4700003DBB0F90840944213DC70BC70470489C8
:10B48000013C641A114622B2F1E7C488058903968B
:10B49000013CAD1AED1A621A11B22AB270BCFFF764
:10B4A00009BF039670BCFFF763BA00BF2DE9F843EC
:10B4B0000446406A002863D0A16DFEF7F3FD052223
:10B4C00074492046FFF714FCA1790139C9B220461E
:10B4D000FFF746FBB4F90820E588A66AD31D48BFEC
:10B4E00002F10E03DB10626A15FB03F51FFA85F803
:10B4F000002A7BD094F82C300125AB4082F83B30F9
:10B5000082F85E5082F85D50606A036840211B68D3
:10B5100008F1FF379847BFB2B8F1000F23D0374486
:10B52000A846013E606A16F8011F03681B68984729
:10B530000135B742EDB216D0202DF3D10121606A5A
:10B54000FEF712FF94F82C20636A520083F83B2028
:10B5500083F85E8083F85D80606A036840211B6821
:10B5600098470125DEE70121606AFEF7FDFE606A6B
:10B57000002800F08D80E16DBDE8F843FEF792BD34
:10B58000236A002B2BD0D97A626DE1B172B6D97AD9
:10B59000CE0706D54048D968056829409961016001
:10B5A000D97A8D0706D53D48196905682940D961C2
:10B5B0000160D97A480705D5394859690568294095
:10B5C0001962016062B61B68D968914207D035489C
:10B5D00018603549DA6042F0804018611960226CC9
:10B5E000216D136823EA0103136068E7E26BE36CE3
:10B5F0001168276A0B4306EB080913604FF0004EF1
:10B600004E450DD016F801CB2FB33A68C2F82CE0A6
:10B61000C2F834C0D36A002BFCDA4E45936BF1D1EB
:10B62000226C236D11680B43136097B1FB7A83B1D1
:10B63000D90703D51D4BBA691A60FB7A9A0703D55F
:10B640001B4BFA691A60FB7A5B0702D5194B3A6A01
:10B650001A60BDE8F883A36BD4F8348008208021F9
:10B66000D8F80020656C1CEA010F14BF2A43AA43D6
:10B67000C8F800201A68A56C2A431A601A68A56CDD
:10B68000013822EA05024FEA51011A60E8D1B7E712
:10B69000276AC5E7A02D010080E100E084E100E019
:10B6A00088E100E001403F0000003F8000E100E051
:10B6B00004E100E008E100E02DE9F04F85B0994693
:10B6C000BDF93870BDF83CA0BB1AC1EB090B002BCB
:10B6D000B8BF5B42BBF1000FB8BFCBF1000B5B45BD
:10B6E0000D4616460093804648DC4D453A463346A3
:10B6F0004CDC194613460A46C5EB09019B1A89B270
:10B70000002B0CB2B8BF5B4204EBD474BE42ACBF9A
:10B710004FF0FF3201224D45039102924FEA64043B
:10B7200029DC9BB201930DE0D8F80070BF69B847DF
:10B73000019BE41AA3B21CB20135002C2DB211DB1F
:10B74000A94518DB009B5B452A46534631464046D7
:10B75000EADCD8F80020534697692946324640462D
:10B76000B847E5E7029A1644039AA94502EB030499
:10B7700036B224B2E6DA05B0BDE8F08F4A462B4671
:10B78000B94635464D4517461E46B2DD3046294678
:10B790003E464D4607468946AEE700BF10B40468F2
:10B7A0002469A44610BC604730B40468BDF8085052
:10B7B0000295A46BA44630BC604700BF30B4046857
:10B7C000BDF808500295E46BA44630BC604700BF4A
:10B7D00070B40468BDF90C60BDF810500396049570
:10B7E000246CA44670BC6047704700BF10B582B09F
:10B7F000B0F90C2001910168009200220C6CB0F9A4
:10B800000A301146A04702B010BD00BF704700BF0C
:10B8100001F003010129C17506D0032904D0C288B3
:10B8200003894281838170470289C3884281838171
:10B83000704700BF2DE9F0410568134E6F6986B06F
:10B84000B7420446BDF8308010D1013B13441BB20F
:10B850000093CDF804800B46AD6A2046A8472368C4
:10B86000DB6AB3420AD106B0BDE8F08105930492C9
:10B870000391B84703A925680EC9E6E7204606B03C
:10B88000BDE8F041184700BFE9B700002DE9F041DD
:10B890000568124E6F6986B0B7420446BDF8308025
:10B8A0000FD1013BCDF804800B4400921BB2AD6A6E
:10B8B0002046A8472368DB6AB3420AD106B0BDE838
:10B8C000F081059304920391B84703A925680EC936
:10B8D000E7E7204606B0BDE8F0411847E9B70000A9
:10B8E0002DE9F04F0568DFF858B06F6985B05F4506
:10B8F0000646BDF93890BDF83CA00C46904615D1DF
:10B900001F19BC420CDACDF800A0214601342D6A83
:10B910004B464246304624B2A847BC423568F2DB6B
:10B92000EB6A5B4507D105B0BDE8F08F0393B847DC
:10B930003568039BE4E7304605B0BDE8F04F184793
:10B94000E9B700002DE9F04387B099420546BDF9FB
:10B950003840BDF83C6025D0A24212D00768DFF81D
:10B960008080D7F81490C14532D18DE85000284628
:10B97000BC6AA0472B68DB6A434524D107B0BDE809
:10B98000F083994202DD08461946034628680E9660
:10B99000C46B01335B1A1BB22846A44607B0BDE84E
:10B9A000F0436047A24202DD134622461C46286847
:10B9B0000E96631C846B9B1A1BB22846A44607B0E4
:10B9C000BDE8F0436047284607B0BDE8F04318479C
:10B9D000059304920391C84703A92F680EC9C4E7D1
:10B9E000E9B700002DE9F04FD0F800E0DFF89090C3
:10B9F000DEF814B083B0CB450446BDF93080BDF805
:10BA000034A00D4617461E4631D1CDF800A0DEF811
:10BA100024B0294633463A462046D8472368CDF815
:10BA200000A008F1FF323A44D3F824B0294612B2FC
:10BA300033462046D8472368CDF800A02946D3F8DE
:10BA400020B03A4643462046D8472068CDF800A0AB
:10BA5000711E29444346056A09B23A462046A84762
:10BA60002368DB6A4B4506D103B0BDE8F08FD847A9
:10BA7000D4F800E0C9E7204603B0BDE8F04F18470E
:10BA8000E9B70000F0B4002401264FF6FF75094F16
:10BA900007600471C475C48104824476C4618675EC
:10BAA000067685824582C180028141818281F0BC17
:10BAB000704700BFD03201002DE9F04F85B0066815
:10BAC000BDF84450BDF93880CDF80080044601959A
:10BAD000D6F848B00392BDF93C60BDF94070894684
:10BAE0009A46D84723680195009742465146D3F8B5
:10BAF000488020463346C0472068039B0E930F952D
:10BB0000856C4B463A4631462046AC4605B0BDE80A
:10BB1000F04F60472DE9F04F87B01746BDF9404020
:10BB200000912546E91D059344BF2B4603F10E0104
:10BB30000268BDF8486053690294C91003912B490B
:10BB4000BDF9444001968B42824645D1002C3CDD34
:10BB5000029B3C445E1EB6B24FF0000923B2049330
:10BB600001364D46029B002B28DD059B002403EB8C
:10BB7000090806E0EDB22B0604F1010411D4A64237
:10BB80001CD0A1B211F0070F23B24FEA4505F1D145
:10BB9000002BB8BF0733DB10013418F803502B0615
:10BBA000EDD5009BD2F818B019443A4609B2019B72
:10BBB0005046D847A642DAF80020E2D1039B01376D
:10BBC0009944049B3FB2BB42CCD1D36A074A93420B
:10BBD00006D107B0BDE8F08F9847DAF80020B5E746
:10BBE000504607B0BDE8F04F184700BFE9B7000066
:10BBF00070B4BDF90C60BDF91050BDF81440039647
:10BC00000495059470BCFFF785BF00BF2DE9F04F88
:10BC100093B090460591C1691090BDF870000790EF
:10BC2000BDF874909DF878A00493002900F0CD80B1
:10BC30000A7A0AC9894604998A1AD2B203EBC20366
:10BC4000BAF1010FDA780B9293F905201E8893F868
:10BC500002B00F9293F9064079D913B2099323B237
:10BC60000C93109B1A68A94B1193194653698B4288
:10BC700040F0A6800B9B002B55D01FFA88F30021C3
:10BC80000D93C8462344DDF8409006910E930F466D
:10BC90000C46BBF1000F3FD0BDF818100C9B03976A
:10BCA0001FFA8AF0CB1813FB00F304900E9801449E
:10BCB0000D98034409B21BB20A910893002505E0D0
:10BCC0000135EBB264009B45E4B222D9039B2B44BF
:10BCD000590703D1731C18F806409EB22306EFD50E
:10BCE000099BBDF81000E91811FB00F10598BAF1A5
:10BCF000010F0FFA8AF301441CD0079801900093BA
:10BD0000D26909B217464846089AB847D9F80020C0
:10BD1000D6E7039F5F44FFB2069B0B99013306935E
:10BD2000DBB29942B5D8D36A119A934243D113B08A
:10BD3000BDE8F08F0F9B191893690A9A29441F4692
:10BD400009B2079B4846B847D9F80020B8E7002356
:10BD50000C93099385E70A9A0D9B0132013B52B27D
:10BD600013F0FF030A920D936FD1DDF81890079B33
:10BD7000DDF83C80DDF820A04B4517D0BAF1010F6B
:10BD800000F0C8800B9A109DCDF804900BEB8B014E
:10BD90004FEACB030A4400931146DEF81C40534699
:10BDA000424609B22846A047D5F800E0DEF82C301C
:10BDB000119A9342BBD0109813B0BDE8F04F1847CA
:10BDC000109D284698472A6854E7109A0598B2F9BA
:10BDD0000A308342ABDDB2F90C304345A7DD0623C0
:10BDE00013FB0A03002BA2DD08EBCA03002B9EDD28
:10BDF000537E2BB9049BAF2B02D90133DBB20493E2
:10BE0000109BD3F800E0414B11931A46DEF8143032
:10BE1000934240F08E801FFA88F30E9308339BB252
:10BE2000BDF81420059305230D9300230A93CDF844
:10BE30003C800FFA8AF3DDF84080CDF818900B9221
:10BE40001FFA8AFBCDF820A099460A9ABDF8100087
:10BE50000B9C0E9D0523194611FB00232C4811460F
:10BE6000C75C039702FB0B4214FA81F312B21BB2B8
:10BE700009920C932C462E461CE0089B0999012B35
:10BE80002AB24B4640462DD0079F0197CDF800902F
:10BE9000DEF81CA0D047D8F800E0039B5B08013413
:10BEA0000393059BA4B25D445E44A342ADB2B6B217
:10BEB0003FF451AF039BD807DFD4079B069A934208
:10BEC000EBD0089B012B16D0069B0193CDF8009078
:10BED000DEF81CA009994B4632B24046D047D8F84C
:10BEE00000E0DAE7DEF818A0079B0C9922B2D047F1
:10BEF000D8F800E0D1E7DEF818A00C9913464046C8
:10BF000022B2D047D8F800E0C7E700BFE9B7000089
:10BF1000203301000B99109DCDF800900531DEF81B
:10BF2000204009B2424608232846A047D5F800E041
:10BF30003CE7109C20469847D4F800E06BE700BF30
:10BF4000F0B5C36985B004462BB30A2968D00D2922
:10BF50004AD01A7A914247D3587A884244D35D68CE
:10BF60008A1A05EBC205AA78002A50D0E878002882
:10BF70004DD0207E00283AD095F905E0B4F90E00A6
:10BF8000A67DB4F90A70724406FB0202BA4262DC72
:10BF9000B4F9102030E00A2956D00D2924D0027EB1
:10BFA000002A4BD0B0F90E00A57DB4F90A60062234
:10BFB00012FB0502B2423EDD228AE38102EBC5029A
:10BFC00012B218462282A78A668A02950B468DE82D
:10BFD000C00001462046FFF719FEA37DE28903EB6E
:10BFE000430302EB4303E381012005B0F0BDA67DCE
:10BFF000B4F90E00B4F91020B4F814E0678A029680
:10C000000B468DE8804001462046FFF7FFFD297969
:10C01000E389A27D012001FB0233E38105B0F0BD7D
:10C020000022C2819A7A817D038A01FB0233038256
:10C03000012005B0F0BDB4F91020C4E7857DB4F946
:10C040001020B0F90E00BEE7028A817DC38102EBA9
:10C05000C1030382C8E70020E0819B7A228A03FBA8
:10C06000062212B22282C7E7C1810282704700BF56
:10C07000002908BF01218175704700BF818241827C
:10C08000704700BFC07D7047B0F90A00704700BF1D
:10C09000B0F90C00704700BF10B4EFF3108272B615
:10C0A000437F33B9017F012907D003290FD0012332
:10C0B000437702B962B610BC7047124C2168A1B137
:10C0C000114943610B68836108605861EFE70F4CC9
:10C0D000216881B10E4943610B6883610860586132
:10C0E0000C4B4FF080511960E1E7074B41618161D2
:10C0F00020601860DBE7064B4161816120601860B9
:10C10000EEE700BFE49EFF1FE09EFF1FD49EFF1FCF
:10C11000D89EFF1F04ED00E070B5EFF3108272B6F9
:10C120000C4C206880B10C4E00254369236073B12C
:10C130009D6102B962B6457783689847EFF3108234
:10C1400072B620680028F0D102B962B670BD3360C3
:10C15000EFE700BFD49EFF1FD89EFF1FFFF7DCBF95
:10C16000184A30B41468002C27D0036821688B4229
:10C170000ED2CB1A00218460C1602360E0601060A1
:10C180000223037530BC704711688B42144608D3F4
:10C19000A2685B1A0360002AF6D18260C460A060C6
:10C1A000EEE7D268C2608460E060C568CB1A022204
:10C1B000A8602360027530BC70478460C460106062
:10C1C000DEE700BFDC9EFF1FF8B5224E34682CB3BB
:10C1D0002368002B3AD1204F1D4604E03468ECB1AF
:10C1E0002368002B32D1A36803B1DD60206933607E
:10C1F000036825751B68BB4221D1037F4560022B74
:10C20000C46020D0FFF748FF6368002BE6D02360AE
:10C210002046FFF7A5FF3468002CE1D1EFF310832F
:10C2200072B60E4A00211068116003B962B628B1D7
:10C230008468FFF795FF20460028F9D1F8BD224613
:10C2400000219847E0E783689847DDE7013B2360DA
:10C25000E4E700BFDC9EFF1FD9A80000EC9EFF1F93
:10C26000024A136801331360FFF7AEBFF89EFF1F49
:10C27000704700BF0368F0B4FBB1002501249D6046
:10C28000DC601B4C1A601C44241104F144056A1143
:10C29000032692009E60174F0679174B47F824102B
:10C2A00002F1604202F5614205F01F05012000FA2B
:10C2B00005F5E6541560F0BC7047104C236843F454
:10C2C0000003236000BF0E4B0E4DA4F58734A4F588
:10C2D0009E7401261E60234604609C68002CD0D00A
:10C2E0001033AB420360F8D1002303601846E2E745
:10C2F000008FFCBF4091FF1F44E400E03C800440FD
:10C3000000700340407103400168A9B10B4BF0B4C9
:10C310000B441B110A4E0B4F0B4D46F8237003F1D3
:10C32000440202F01F0401235211A340002445F8E7
:10C3300022308C600460F0BC704700BF008FFCBFEF
:10C340004091FF1F71C2000080E100E0024A034BF0
:10C35000012111601B6818470C7103404091FF1FB9
:10C36000024A034B012111605B6818471C710340AE
:10C370004091FF1F024A034B012111609B6818473F
:10C380002C7103404091FF1F024A034B01211160B1
:10C39000DB6818473C7103404091FF1FF8B50E461B
:10C3A00071B17AB10746144600253B6816F8011BA7
:10C3B0001B6838469847013C0544F6D12846F8BD2D
:10C3C0000846F8BD1046F8BD00B5064A0368128855
:10C3D0005B6883B001A9ADF804200222984703B03E
:10C3E0005DF804FB20380100F0B507468BB0002A49
:10C3F00033D0012A08BF0A2251B3212400E0F4B24D
:10C40000B1FBF2F502FB1511C8B2092900F13001A8
:10C4100098BFC8B20AA988BF3730214488BFC0B2CC
:10C4200001F8240C661E2946002DE8D133B1013CE9
:10C43000E4B20AAB23442D2203F8242C3B6801AA62
:10C4400011195B683846C4F1220298470BB0F0BD61
:10C4500030228DF825202124E8E70368C9B21B6843
:10C4600098470BB0F0BD00BF0029BABF49422D2349
:10C4700000230A22FFF7B8BF374A384913681B0662
:10C48000FCD40B6813F08003F8D172B634490A78F3
:10C49000002A5FD0334A3448F0B4344C1768066839
:10C4A0002568D4680C303E44143200681268304F5E
:10C4B00035442C4420440244C2F34E022D4E2E48F3
:10C4C0002E4D2F4C42F400423A60376806682D68C2
:10C4D0002C4A24680C303E44006812682A4F3544C8
:10C4E0002C4420440244C2F34E02284E2848294DD1
:10C4F000294C42F400423A60376806682D68274AA2
:10C5000024680C303E4400681268254F35442C44A2
:10C5100020440244C2F34E02224E2348234D244CB1
:10C5200042F400423A60376806682D68214A246860
:10C530000C303E440068126835442C4420440244C8
:10C54000C2F34E021C4842F4004202600B7062B615
:10C55000F0BC704762B6704724B0034024B00B4073
:10C56000F19EFF1F38B003403CB0034040B0034091
:10C570002CB0034058B003405CB0034060B00340AF
:10C5800064B003406CB0034030B0034038B00B409F
:10C590003CB00B4040B00B4044B00B404CB00B40A3
:10C5A0002CB00B4058B00B405CB00B4060B00B405F
:10C5B00064B00B406CB00B4030B00B4030B4294835
:10C5C000294A2A4B2A4D6024E121047011701B78FE
:10C5D000284C082B30D00A2B2748284937D00C2B61
:10C5E0000CBF35223D2212232A60236002600B60BB
:10C5F000234B24491B78244ABBB101230B601360F1
:10C60000224B23491B78234A012B26D9042B0FD90F
:10C61000082B1ED9102B94BF862387230B60136031
:10C620001D4B01221A7030BC70470B601360E7E7A6
:10C6300084230B601360F3E700F58E200F49083068
:10C64000012213232A60236002600B60D0E73922A5
:10C65000F7E785230B601360E2E780230B6013602C
:10C66000DEE700BF00400740014007405091FF1F38
:10C6700008B003400CB0034008B00B400CB00B40B6
:10C68000F49EFF1F20B0034020B00B405191FF1FCC
:10C6900024B0034024B00B40F19EFF1F0C2830B49F
:10C6A00017D91023984228BF18461C46104A114D2E
:10C6B0001178181A8C42287018D00F4913700B7813
:10C6C00023B10E490E4A00230B60136030BCFFF704
:10C6D00075BF0A2802D90C231C46E7E7082802D9AF
:10C6E0000A231C46E2E708231C46DFE730BC7047FC
:10C6F0005091FF1FF09EFF1FF19EFF1F24B00340CB
:10C7000024B00B4028282FD8334B2DE9F0411E5C74
:10C71000FF2E2BD0314B1B78002B2AD132062CD484
:10C7200072B62F4D2F4C2F46012326602B7062B618
:10C7300072B623681B060CD43B781BB9F4E72B7840
:10C74000002BF1D062B602F09BF972B6236818068E
:10C75000F5D5254B1B6800222A7062B6234A107853
:10C7600043FA00F0BDE8F081002070470020BDE8EA
:10C77000F081FFF781FE3206D2D572B61C4DDFF88C
:10C780007C801C4C06F04007FFB206F03F06D8F84C
:10C790000030DFB123F01003C8F800300123266019
:10C7A000134A2B7062B672B6236819060CD413783C
:10C7B0001BB9ECE72B78002BE9D062B602F060F9E8
:10C7C00072B623681B06F5D50B4BC3E743F0100385
:10C7D000C8F80030E2E700BF24380100F19EFF1FD7
:10C7E000F39EFF1F00B0034010B00340F09EFF1FF8
:10C7F000F29EFF1F00B00B4010B00B400CB00B407E
:10C800000A4A0B49136843F4805313600B7843B909
:10C81000084BC0221A70084B80F30C0000B218803D
:10C820007047044B80221A70F5E700BF2C8004404B
:10C83000F49EFF1F21C00C4000C00C40F0B51B4B04
:10C840001B4E596818689A68DB6885B06C460FC43F
:10C85000337899071DD5174A174C1378174913F0E9
:10C86000700318BF1370164A164B802717700026E6
:10C870003320032226706D4608701A7072B6043C8D
:10C8800045F001052046A84762B6237813F07003EF
:10C8900009D10D4B064901E0013B02D00A78D207CD
:10C8A000FAD505B0F0BD237005B0F0BD50380100D9
:10C8B0000100024000000240040002400B00024060
:10C8C000070002400A000240410D0300B0F5006F6E
:10C8D0000AD210B5094B1B78DB07044606D504F1D4
:10C8E000A0500078C0B210BD00207047FFF7A6FF2F
:10C8F00004F1A0500078C0B210BD00BF010002409A
:10C90000B0F5006F17D238B50F4B1B78DA070D461C
:10C91000044611D504F1A0500378AB420AD00B4A6B
:10C92000137813F0700318BF1370074A057013785B
:10C93000DB07FCD538BD7047FFF780FF04F1A0503E
:10C940000378AB42EBD1F5E7010002400000024062
:10C9500008B5F5F76BF8F5F739FC02F091F8FAE74E
:10C96000844641EA000313F003036DD1403A41D3FA
:10C9700051F8043B40F8043B51F8043B40F8043BB9
:10C9800051F8043B40F8043B51F8043B40F8043BA9
:10C9900051F8043B40F8043B51F8043B40F8043B99
:10C9A00051F8043B40F8043B51F8043B40F8043B89
:10C9B00051F8043B40F8043B51F8043B40F8043B79
:10C9C00051F8043B40F8043B51F8043B40F8043B69
:10C9D00051F8043B40F8043B51F8043B40F8043B59
:10C9E00051F8043B40F8043B51F8043B40F8043B49
:10C9F000403ABDD2303211D351F8043B40F8043BE9
:10CA000051F8043B40F8043B51F8043B40F8043B28
:10CA100051F8043B40F8043B103AEDD20C3205D3F8
:10CA200051F8043B40F8043B043AF9D2043208D0F0
:10CA3000D2071CBF11F8013B00F8013B01D30B8862
:10CA400003806046704700BF082A13D38B078DD040
:10CA500010F003038AD0C3F10403D21ADB071CBF12
:10CA600011F8013B00F8013B80D331F8023B20F87C
:10CA7000023B7BE7043AD9D3013A11F8013B00F8B5
:10CA8000013BF9D20B7803704B7843708B7883703D
:10CA90006046704708B5104C08E0236859050DD46E
:10CAA00023681A050FD42368DB0411D423685803C4
:10CAB000F3D500F08DFE23685905F1D502F044F856
:10CAC00023681A05EFD502F0D5F82368DB04EDD50D
:10CAD00000F0F0FCEAE700BF3480044008B5FFF73F
:10CAE000D9FF00BF014B10221A807047002005407B
:10CAF000704700BF094908B50B6830B16A46184451
:10CB0000A2F58052904202D20860184608BD03F098
:10CB100065FB0C2303604FF0FF3008BD5491FF1FED
:10CB2000FEE700BFEFF3138070B9EFF310836BB92A
:10CB3000EFF305825AB94FF48070EFF311832BB1F4
:10CB4000984228BF184670474FF0FF3070470F2AB1
:10CB500001D81846F1E7014BD05CEEE7F0E300E0C6
:10CB6000F0B44D1E2E46002400E00134B0FBF2F379
:10CB700002FB1300092800F130078ABF3730F8B2F2
:10CB8000C0B206F8010F1846002BEED10A195370F7
:10CB90004CB1107815F8016F28700133E01A834208
:10CBA00002F80169F5DB0846F0BC7047704700BF2A
:10CBB00010B40F4B53F8302092F880422CB101236F
:10CBC00069B182F8803010BC704703EBC0035B682A
:10CBD0001A6841B922F002021A6010BC704782F84C
:10CBE000003110BC704742F003021A6010BC70475D
:10CBF000603801001C4A02EBC00301295B6811D0B8
:10CC000004291BD052F83000002280F8802229B17C
:10CC1000022920D0032922D01A6070474FF4807275
:10CC20001A60704752F830004FF4A27280F88012F8
:10CC30001A601A6822F020021A60704752F8301009
:10CC40004FF4A272012081F880021A601A6842F043
:10CC500020021A60704740F203121A6070474FF4C6
:10CC600081721A60704700BF60380100212848D8DF
:10CC7000F8B5042A44D8DFE802F0484B4E034500DB
:10CC80004FF410262B4B03EBC0030D465C68216864
:10CC900011F4E06148D0284B284A2949C3F89C2167
:10CCA00004F140422748C3F8A411A2F59221264F6F
:10CCB000C3F8A0017C292548C3F8A871C3F8AC01CA
:10CCC0002CD9A2F594237C2B2AD9A2F596237C2B70
:10CCD00028D9A2F598237C2B29D9A2F59A227C2A5F
:10CCE00027D81B4872B6236823F4702343F0807260
:10CCF000C4F384011643236040F82150266062B6D5
:10CD0000F8BD70474FF43026BCE74FF40026B9E772
:10CD10004FF44026B6E74FF42026B3E70D48E1E78D
:10CD20000D48DFE70D48DDE7FFF764FFB3E70C4888
:10CD3000D8E7F8BD603801000082FF1FF188FF1FAF
:10CD40009988FF1FC588FF1F6D88FF1F4188FF1F3F
:10CD50003092FF1F5891FF1F9091FF1FE091FF1F1E
:10CD60001092FF1F1A4B03EBC00010B4426802F18F
:10CD70004043A3F592217C2923D9A3F594217C2952
:10CD80000DD9A3F596217C291FD9A3F598217C29DB
:10CD900019D9A3F59A237C2B11D80E4C00E00E4C28
:10CDA00072B613680D4823F08773C2F3840123F42D
:10CDB000803343F08073136044F8210062B610BCE6
:10CDC0007047074CECE7074CEAE7074CE8E700BF81
:10CDD000603801003092FF1F9091FF1FADCB000023
:10CDE0005891FF1F1092FF1FE091FF1F30B4054BB9
:10CDF000054D064C002210211A602A60206019603F
:10CE000030BC704714D0034004D0034000D003402E
:10CE1000282838B52ED0002904464FDD5F4B1B78FB
:10CE2000012505FA03F28A4202D8212837D938BDF4
:10CE30000338C2B2012A3AD9202C4AD0192C48D042
:10CE4000574A126802FB011222FA03F31D2800F26E
:10CE50009B80DFE800F0928B847D9999766F999999
:10CE60009999999999999968615A53994C9999996D
:10CE700099999945494B1B780B2B08D90C2B1CBF52
:10CE80000C3B19410846BDE83840FFF7B9BCC3F177
:10CE90000C0399400846BDE83840FFF7B1BC29466D
:10CEA000FFF786FE2946BDE83840FFF7A3BE3D4A9E
:10CEB000126802FB011222FA03F3C7E72128B6D851
:10CEC0000021FFF775FE20460121BDE83840FFF73D
:10CED00091BE354A126802FB011222FA03F3B5E74C
:10CEE0003249334A0B604FF45173136038BD3149F6
:10CEF000314A0B604FF45173136038BD2F49304AEB
:10CF00000B6040F24443136038BD2E492E4A0B603B
:10CF100040F24443136038BD2C492D4A0B6040F267
:10CF20004443136038BD2B492B4A0B6040F2444305
:10CF3000136038BD29492A4A0B6040F2444313600C
:10CF400038BD2849284A0B6040F24443136038BD7D
:10CF50002649274A0B6040F24443136038BD2549F7
:10CF6000254A0B6040F24443136038BD2349244AEC
:10CF70000B604FF45173136038BD2249224A0B6095
:10CF80004FF45173136038BD212C3FF650AF7F2909
:10CF9000D4BF00210121204693E700BF3892FF1F34
:10CFA000088003400890034008800B4010800B402D
:10CFB00048A0044018800B404CA004401880034057
:10CFC00008B004401080034004B004404080034097
:10CFD00018C004403880034014C004402880034037
:10CFE00010B00440208003400CB004403080034067
:10CFF00010C00440488003401CC004401890034007
:10D0000034900440109003403090044038B1102810
:10D0100028BF1020044AC3B2107813707047024A28
:10D0200001231078137070473892FF1F2DE9F843E1
:10D030000E4680463249334D304603F055F847F6E8
:10D04000122300281ABF1D464FF002094FF00109B4
:10D05000002425FA04F002F051FE4FF05E5107461D
:10D0600002F0A4FE0146304603F052F830B9013414
:10D07000072CEED1E80902F041FE0746314638465A
:10D0800002F048FF4FF07C5102F086FD03F07AF881
:10D090004FF6FF729042A8F1030328BF1046012B00
:10D0A00029D9B8F1170F17D8174B23FA08F303F053
:10D0B000010383F0010223B9B8F1190F0FD0BDE8C5
:10D0C000F883124B124D13491A6044EAC9042A60CE
:10D0D00008601C60BDE8F883B8F1200FECD10E4B5E
:10D0E0000E4D0F49002244EAC9041A602A60086004
:10D0F0001C60BDE8F8830B4B0B4D0C49F2E700BFF9
:10D10000001BB740006CDC026006F00000800340AA
:10D11000048003400880034000800B4004800B40E3
:10D1200008800B40009003400490034008900340A7
:10D13000212801D8FFF73CBD704700BF212806D841
:10D14000044B53F8303093F80002C0B2704700200F
:10D15000704700BF60380100212801D8FFF74ABDA1
:10D16000704700BF72B60C490C4B0D4A1B6808682B
:10D17000126862B6520102D5322B88BF01300949CC
:10D18000C3F5BB334FF47A72FF33A1FB031302FBE9
:10D1900000F000EB93107047F89EFF1F18E000E0CE
:10D1A00004ED00E0ABAAAAAA2DE9F843054672B641
:10D1B000204F214B214A1B683C68126862B652011D
:10D1C00002D5322B88BF013495B3C3F5BB331C4E57
:10D1D000DFF86490DFF86480FF334FF47A72A6FBC7
:10D1E000031302FB04F404EB931472B6D9F8001095
:10D1F0003A68D8F800E062B6C1F5BB33FF33A6FB4E
:10D2000003031EF0806FC4EB93134FF47A7002D0C7
:10D21000322988BF013200FB0233B3F57A7F04D391
:10D22000013D05D004F57A74DFE701F029FCDCE765
:10D23000BDE8F883F89EFF1F18E000E004ED00E071
:10D24000ABAAAAAAF8B52D4B2D49DFF8D0E0DFF83C
:10D25000D0C02C4E2C4D2D4C2D4A2E4F4FF400009B
:10D2600018604FF0807018604FF0007018604FF039
:10D27000806018604FF0006018600020086028236C
:10D280004BF6FF71CCF80010CEF80030336013601D
:10D290002B6023603B60B3629362092245F8242C23
:10D2A000C4F8D80F05F57F65C7F8D41F07F5FF2729
:10D2B00007F5FA67C6F8F83F2B6006F5FF26C4F8B5
:10D2C000D42F05F5FD2504F5FF24386006F2F47629
:10D2D0001148316005F5FF6504F5FD642B6023609E
:10D2E0000260FFF76BF91920FFF75EFF00F0B6FF51
:10D2F00040F21310BDE8F840FFF756BF08E100E028
:10D300000480034014800340248003402C800340A9
:10D310001C8003403480034000800B400C8003409D
:10D32000088003402DE9F84F214B1B6807460BB1DD
:10D3300001221A70DFF888901E4D99F80040DFF83E
:10D3400084801D4E0134272C8ABF4FF0000A5FFAFB
:10D3500084FA5446AB462B78A34216D1FFF7E2FB82
:10D3600040281FDC33791B06F5D59BF800300133CC
:10D37000272B86BF00221346DAB218F80330DBB23F
:10D38000F3712A702B78A342E8D00C490A4BFFB204
:10D3900008F804700120AC22087089F800A0DA7047
:10D3A000BDE8F88FFF28D6DD01F06AFBD3E700BFA8
:10D3B000709FFF1F6D9FFF1F00C006406C9FFF1FE7
:10D3C000749FFF1F049FFF1F1C4BDFF894C01A6857
:10D3D0001B49F0B542F480521A4D1A60DFF884E020
:10D3E000194F1A4E1A4C00238CF800304FF451722A
:10D3F0002B701F2840F213358EF800303B703370CD
:10D4000025600A6012D819460124124A124D117083
:10D410001248547000212C27402693724FF4003498
:10D4200091701174D7702E700460F0BDC0F3443158
:10D43000C0F3471400F01F03E7E700BF3480044047
:10D440000CC00440019FFF1F6D9FFF1F6C9FFF1FBB
:10D4500008C0044000C0064031E400E004E100E000
:10D46000009FFF1F749FFF1F034B1B68DB0401D548
:10D47000FFF758BF704700BF3480044010B5044C1C
:10D48000237823B101F0FCFA2378002BFAD110BDE8
:10D490006C9FFF1F054A064B10781B78C0B2DBB2A9
:10D4A000984238BF4030C01A704700BF009FFF1F2E
:10D4B000019FFF1F30B42B4B1A7994061FD52A48C1
:10D4C000DA790378294901333F2B0978C8BF002353
:10D4D0008B42D2B203D0264CD9B2E2540170254A15
:10D4E000116861B1244A1278D2B2934236BFC2F1B8
:10D4F00040029B1A9B18272BC4BF01230B70194AAB
:10D50000D378DBB2180611D45A060DD5154B1B790A
:10D510005B0609D5194B1A491B6800220A7003B132
:10D520001A70104B2C22DA7030BC70471179090642
:10D53000EAD5144910480C780178C9B28C420DD054
:10D540004A1C272A84BF00210A460F4D054C98BF6C
:10D55000D1B2AA5CD2B2E2710170D5E76C21D17070
:10D56000D2E700BF00C00640009FFF1F019FFF1FC2
:10D570002C9FFF1FFC9EFF1F6D9FFF1F709FFF1FB3
:10D580006C9FFF1F749FFF1F049FFF1F21282FD830
:10D59000184B195CFF292BD0174B184ADFF870C0C5
:10D5A00003EBC000F0B54368DFF868E0144F154D99
:10D5B000154E00241C60DEF80030012043F02003EB
:10D5C0008840CEF8003014604FF4A07338602E60AD
:10D5D000C2F800C0013BFDD113689B05FCD4202399
:10D5E000013BFDD1094B09B233F8110080B2F0BD07
:10D5F000002070477039010060380100005004407D
:10D60000085004400450044000000203005104404C
:10D6100080014A0038800440431E032B14D872B6A0
:10D620000A4951F8230068B170B4094C058834F8F0
:10D630001320466841F82360521B24F8132062B679
:10D6400070BC704762B6704700207047D09FFF1FC4
:10D6500014A2FF1F013803280BD872B6074B53F8EA
:10D66000203043B100205B680130002BFBD162B653
:10D670007047002070471846F9E700BF24A0FF1F3D
:10D6800030B472B62B4A13781D0706D52A4B196A97
:10D69000002936D0996A002941D053781C0706D555
:10D6A000254B196C00293ED0996C002939D093780C
:10D6B000190705D5204B196E002936D0996E89B10E
:10D6C000D3781B0707D51C4BD3F880207AB3D3F847
:10D6D000882011213AB162B6184B00221A7030BC72
:10D6E00000F04ABE0D21154C154D227843F83150FB
:10D6F00003EBC1030830013A5860227062B630BCB7
:10D70000704704220D4C0F4D217843F8325003EB43
:10D71000C20308304A1E5860227062B6EFE7052146
:10D72000E1E70921DFE70822ECE70C22EAE7102213
:10D73000E8E700BF943901000080FF1F4DA0FF1FE4
:10D74000C800400088004000431E032B1DD81B4A20
:10D75000400140F0100030B4104472B6184CE25C46
:10D76000032A1BD8DFE802F00212151703220D88E6
:10D77000E25410F0080F14BFC823882343EA05437E
:10D7800008310360416062B630BC70470830022245
:10D79000EDE70522EBE708300422E8E7094A52F8F2
:10D7A000230038B1084A52F82300416042F82310A0
:10D7B00062B6E9E742F82310034AF7E70080FF1F4B
:10D7C0005CA0FF1F24A0FF1F34A0FF1F00BE7047F6
:10D7D0002DE9F04FDFF818B3DFF818A387B044E065
:10D7E000AD4F4FEA930807EBC809013ED9F8042072
:10D7F00003F00803F6B2A2F1080003F0FF04002BC7
:10D8000040F0018157F838301B0C99B222F8081CFF
:10D81000002B00F0EF80A14B22F8064C42F8044C9C
:10D8200053F82620002A00F0CF819D4D55F8263070
:10D8300058609C4C45F8260034F81630194424F8FA
:10D84000161000F079FD002800F0C281964A974B2F
:10D8500019F0080F00F1080018BF1346C9F80400BA
:10D8600047F8383008238BF800309BF80040E4B2CA
:10D8700065071CD58E4B1B78B3B18E490A7802F030
:10D88000FF0322B1013BDBB20B7003B900BE8A4932
:10D890000A7802F0FF032AB1013BDBB20B70002BC8
:10D8A00000F0688100F066FE04238BF8003004F07D
:10D8B000080303F0FF02002B00F0C9809AF8003043
:10D8C000DBB21E098CD19A08DFF8CC9159F83210DE
:10D8D00009EBC200C1F38301013940680C2900F251
:10D8E0008580DFE801F07A7A8383838383834683AC
:10D8F000838307000168714D4068714F714E686005
:10D90000296088B240F281610024674B49F83230C7
:10D910004FF0010E88423C60C9F81040C9F8184029
:10D9200086F800E05C4A00F2E780B0F5D06F80F046
:10D930001B82B0F5817F00F0D98100F269818028D7
:10D9400000F02A82822840F0D781A98801F07F0167
:10D95000042900F2D1815C485C4A890008441470B3
:10D96000547001788C0740F1608382F800E0022156
:10D9700073E1534F3A682AB3554B524E55481988B4
:10D980003478057840298E4645F0020828BF4FF0CC
:10D99000400E002C84F001043470CEEB01010CBF6A
:10D9A0008824C82409EBC80689B285F0010544EA39
:10D9B0000E447260198049F838407244057000299D
:10D9C00065D03A603D4B1A88B2F5A06F0ED10021A8
:10D9D0009A785970404B1A7008E038493F4C0D68EE
:10D9E000A54200F09880304949F832103C4A0123A2
:10D9F000137037E72C4A2D4B19F0080F18BF134648
:10DA000047F838302EE700F0B7FC364A364952F86E
:10DA10002630002B00F0E38058688C5D42F8260029
:10DA200003F10802C9F80420032C05D8DFE804F04C
:10DA30002C02292602228A551A8819F0080F0CBFD9
:10DA40008823C82343EA024347F838300AE7E0074F
:10DA500000F19380210600F1D180A20706D5234A68
:10DA6000234913780220DBB213700870E30602D555
:10DA70001F4B10221A7007B0BDE8F08F04228A55A0
:10DA8000DAE705228A55D7E703228A55D4E7BEF1A3
:10DA9000400F18BF002294E70080FF1FD09FFF1F98
:10DAA0007C9FFF1F14A2FF1FC80040008800400099
:10DAB00058A0FF1FE19FFF1FCCA0FF1F44A0FF1F26
:10DAC000789FFF1FE09FFF1FC020074050A0FF1F4F
:10DAD0008C9FFF1F4CA0FF1F9820074021090003C7
:10DAE0009420074024A0FF1F5CA0FF1F8820074050
:10DAF0008020074090200740B0F5106F00F07C8137
:10DB000040F2A38040F62112904240F07B82A54A69
:10DB1000012313706AE74C68A3498C427FF463AF1A
:10DB20000178A9297FF45FAF417845297FF45BAF85
:10DB30008178C2297FF457AFC1786B297FF453AF46
:10DB40009A489B4E0178347881F00105002C41F011
:10DB5000020105700CBF8820C82084F0010449F838
:10DB6000310009EBC10193483470002505244D6054
:10DB7000047038E700F064FF94E68F4B89488B49C6
:10DB80001A614FF0020E80F800E08C4F0A708C4949
:10DB9000196099608B4E8C4D8C4C9A610D213970B7
:10DBA000FF213170DFF84CE229702270884D894ADC
:10DBB0008EF800109F27012406F8047C5D60047035
:10DBC000DA6007B0BDE8F08F43F82600824D30E6FA
:10DBD000824A47F8380013780133137042E68B5DB0
:10DBE000032B00F2BA8001A252F823F065D800009E
:10DBF00065D8000045DC00003FDC00006F49724B37
:10DC000080220D2008701A70A2077FF52FAF26E73B
:10DC100040F20232904240F0ED81AA8802F07F0289
:10DC2000042A69D86D88002D66D16449CDF804E0D6
:10DC3000920011440A7842F002020A70C1E1012305
:10DC40008B550FE600238B550CE6B0F5086F53D1CA
:10DC50006349644A097811707146ED888D4280F0FD
:10DC6000E88252480478402DAE4644F0020C28BFAA
:10DC70004FF0400E02EB0E0309EBCC01029301239F
:10DC80004A604FEA0E48CEEB050101930025C822F9
:10DC900042EA080384F0010249F83C303570027012
:10DCA000DFF814C1424BDFF8048149BBBEF1400FDD
:10DCB0007FF42DAF42F0020C09EBCC03029ADFF89F
:10DCC000F8E05A608DBB0D0445F088059DF80430DE
:10DCD0004EF83C500A4433700470134640297FF4D8
:10DCE00016AF0021404A3B60118010E7AA8802F07D
:10DCF0007F02042A40F28B81304A0F23137006E71B
:10DD00004029D7D942F002020CEBC200029E4660C5
:10DD1000BDB19DF8045035481D703346403988F830
:10DD2000004040334CF83200DCE79DF8043033709B
:10DD30000D04029B047045F0C8050B444EF83C509E
:10DD4000CCE79DF804501D70029B1D4888F80040E8
:10DD5000403940334CF83200C4E719F0080F0CBFCB
:10DD6000022303238B557DE521494A68002AC3D04D
:10DD70006C88B5F804E003E00C314A68002ABBD097
:10DD80000B88A342F8D14B887345F5D1240A032CA4
:10DD90000CBF1178098960E7124A0221147054708F
:10DDA0005BE700BF94200740010004004CA0FF1F68
:10DDB000E09FFF1FE19FFF1F0080FF1FC020074063
:10DDC00088004000882007408020074098200740B6
:10DDD000909FFF1FE49FFF1F7C9FFF1F4DA0FF1F11
:10DDE00058A0FF1F50A0FF1F8C9FFF1FC8004000BE
:10DDF000983901008C200740B248116AAC78047051
:10DE00000C0600F19881D9F82820AF49100600F1DE
:10DE1000DB81D9F83020AC49120600F1D081D9F865
:10DE20003820A949130600F1C581D9F84020A64938
:10DE3000150600F1BA81D9F84820A349140600F16B
:10DE4000AF81D9F85020A049100600F1A481D9F87B
:10DE500058209D49120600F19981D9F860209A490D
:10DE6000130600F18E81D9F868209749150600F154
:10DE70008381D9F870209449140600F17881D9F88B
:10DE800078209149100600F16D81D9F880208E49E3
:10DE9000120600F16181D9F888208B49130600F140
:10DEA0005581D9F890208849150600F14981D9F8A3
:10DEB00098208549140600F1FF808448844A8549EA
:10DEC00001908548854D864C049700230596029560
:10DED00080460F4616461D460394306828B14468B4
:10DEE00000F04AFA2046002CF9D100233360029B4F
:10DEF00038681A46002342F8253028B1446800F0FB
:10DF00003BFA2046002CF9D100223A60019A98F899
:10DF100000301146002241F8042B039A0191023B84
:10DF20004FF0000122F81510032B07D8DFE803F0AB
:10DF30005D025D024FF0010388F800300135042DC9
:10DF400006F1040607F1040708F10108C5D1654C84
:10DF5000654D2278654B049F059E002110072970AE
:10DF60001A7000F19280624962780A700021C9F843
:10DF70003010C9F838101107DFF84C816ED4A27840
:10DF80005C49DFF844810A7000211207C9F850107B
:10DF9000C9F858104BD4E27857494B4C0A70130714
:10DFA0004FF00001C9F87010C9F8781000F1AE8088
:10DFB00033780193002283F00105C9F89020C9F855
:10DFC00098200021029188468E460A464B480478E4
:10DFD00044F0020C09EBCC030393019B002B039B41
:10DFE0005A600CBF8822C82252E64FF0000388F81E
:10DFF0000030A3E7B0F5A06F7FF47EAE01230025CB
:10E000000193DEE740F621229042F7D074E66D8856
:10E01000002D7FF471AE3A49CDF804E0920011442E
:10E020000A7822F002020A70CBE7022115E600F01E
:10E0300083F9002800F0EB800830324AC8F8640009
:10E04000C8F8602000F078F9002800F0DA80083085
:10E050002D4AC9F86C00C9F868209CE700F06CF9FB
:10E06000002800F0E0800830264AC8F84400C8F8CC
:10E07000402000F061F9002800F0CF800830224AEB
:10E08000C9F84C00C9F8482079E700F055F9002894
:10E0900000F0A58008301B4AC9F82400C9F82020E8
:10E0A00000F04AF9002800F094800830164AC9F8B8
:10E0B0002C00C9F8282056E7D1F89C00083800F059
:10E0C0005BF9FAE658A0FF1F0080FF1F34A0FF1F76
:10E0D000D09FFF1F24A0FF1F5CA0FF1F7C9FFF1F7E
:10E0E00014A2FF1F943901004DA0FF1FC420074058
:10E0F000C8200740CC200740D02007404CA0FF1F7D
:10E10000C020074088004000C800400000F014F91B
:10E11000002870D008304F4AC4F88400C4F880202A
:10E1200000F00AF9002860D008304B4AC9F88C008A
:10E13000C9F888203CE7506A083800F01DF962E60B
:10E14000D1F89400083800F017F9B0E6D1F88C0047
:10E15000083800F011F9A4E6D1F88400083800F07E
:10E160000BF998E6C86F083800F006F98DE6486F9D
:10E17000083800F001F982E6C86E083800F0FCF8B3
:10E1800077E6486E083800F0F7F86CE6C86D083896
:10E1900000F0F2F861E6486D083800F0EDF856E658
:10E1A000C86C083800F0E8F84BE6486C083800F016
:10E1B000E3F840E6C86B083800F0DEF835E6486B57
:10E1C000083800F0D9F82AE6C86A083800F0D4F810
:10E1D0001FE62A78C9F8280001322A70C3E62A7897
:10E1E000C9F8200001322A705AE72A78C9F8880055
:10E1F00001322A70DCE62A78C4F8800001322A70E5
:10E200008EE72A78C9F8680001322A70C3E62A78B6
:10E21000C8F8600001322A7014E72A78C9F848006B
:10E2200001322A70ABE62A78C8F8400001322A7021
:10E230001FE740298E4628BF4FF0400E02EB0E0329
:10E2400002930123CEEB01014FEA0E480025019312
:10E25000BCE600BF88004000C8004000F8B500F0F0
:10E260008FFD294B29482A4C2A4F2B4DDFF8BCC083
:10E27000DFF8BCE0294E00221A605A609A60DA602A
:10E280001A615A619A61DA611A625A629A62DA62B2
:10E290001A635A639A63DA631A645A649A64DA6492
:10E2A0001A655A659A65DA651A665A669A66DA6672
:10E2B0001A675A679A67DA67C3F880200168C3F85B
:10E2C000842041F480210160C3F307212170C3F34E
:10E2D0000740134938701B0E2B70FF238CF8003059
:10E2E000104D8EF8003010480B700123337084F805
:10E2F000642070264FF40074102207F82C3C2E7016
:10E30000046081F8F820F8BD0080FF1F34800440CD
:10E310009C200740B0200740B420074094200740CD
:10E320001020074049E400E008E100E080200740B9
:10E3300088200740704700BF72B60D480268B2FAE5
:10E3400082F30F2B10DC4FF00041D94022EA01028A
:10E35000026062B6074803EBC303DB00C21800216A
:10E36000C15010465160704762B60020704700BF30
:10E370003C92FF1FBC83FF1F0D4B0E4AC31AA2FB2A
:10E3800003231B090F2B0CD80B4A127852B972B613
:10E390000A484FF00041026821FA03F31A43026071
:10E3A00062B67047064A1278002AF0D0FFF768B9C3
:10E3B000BC83FF1F398EE3384DA0FF1F3C92FF1F27
:10E3C00058A0FF1F38B50E4B0E4C1B682188054620
:10E3D0008BB1B1F5917F05D20B4A4B1C55549BB2C2
:10E3E000238038BD0022084898470021064A55542A
:10E3F0000123238038BDB1F5917FEDD338BD00BF37
:10E4000084A0FF1F1EA2FF1F24A2FF1F2DE9F843B7
:10E41000214E224F3168012380463B70B1B1204D1F
:10E420004B8801EB8302013300240F2BC2F80880D4
:10E430002C7004D84B8000233B70BDE8F883402348
:10E440000B800320FFF780F93460F4E7DFF8549085
:10E4500099F80030002BF0D0114D45F6215408E01A
:10E46000013C12D02B7883B900F00AFB99F80030F8
:10E470007BB10320FFF7EEF80528F1D8FFF75CFF2A
:10E48000014630600028EBD0CAE701232B70BDE8BD
:10E49000F883BDE8F88300BFA0A0FF1F74A0FF1F92
:10E4A000A4A0FF1F58A0FF1F1201F8B5D5B2A1B359
:10E4B000012943D04378044600781B0643EA004014
:10E4C00040F4704045F004068F1E3043FFF79EFF76
:10E4D000022F04F1020314D9053414F8023C14F895
:10E4E000032C14F8010C1B0443EA0223334343EAD0
:10E4F0000060033FFFF78AFF022F234604F1030465
:10E50000EBD8022F23D0012F0DD045F4774040F0F7
:10E510000500BDE8F840FFF779BF14482843BDE87F
:10E52000F840FFF773BF187845F4770545F0060506
:10E5300045EA0020BDE8F840FFF768BF03780C48C3
:10E5400045EA03452843BDE8F840FFF75FBF1A7866
:10E55000587845F0774545F0070545EA022545EA34
:10E560000040BDE8F840FFF751BF00BF06F0F700DC
:10E5700007F000F738B5084B1C7824B9074D296817
:10E5800009B14B8803B938BD9B000B800320FFF70E
:10E59000DBF82C6038BD00BF74A0FF1FA0A0FF1FD8
:10E5A0002DE9F041AD4E33680746002B00F0928014
:10E5B0001D885A88910803EB81010432AA428C68B5
:10E5C00042D25A8004F00F064FEA1428A449A6F15B
:10E5D000080208F00F00C4F30313062A00F1010536
:10E5E0000B701AD9B31E012B5FFA88F04ED9052E95
:10E5F00048D0042E00F0A481731F022B7FD90F2E68
:10E600000ED1F72842D8F02802D0964B1B883BB198
:10E61000FFF7D8FE0020BDE8F08127B1BD4202D04F
:10E620000020BDE8F081082EC4F3033300F087809A
:10E63000092E11D00A2E40F094800A2BF0D18A4B7B
:10E640008A4A1B68A02181E01846FFF795FE042046
:10E65000FEF7E2FF3060B5E7092BE1D1270E00F0AD
:10E660007B81834B814A1B689021C4F3074611705C
:10E67000EDB2FCB2002B00F09D80224631462846C8
:10E68000984797E0F02843D9F72841D0F1380E2871
:10E69000C6D801A353F820F04FE8000033E800008B
:10E6A00021E8000021E6000021E6000013E8000058
:10E6B00021E60000F3E8000021E60000BDE80000CC
:10E6C000D7E80000FBE7000021E60000E3E70000D8
:10E6D000C7E70000674B1B78002BA1D00420FEF792
:10E6E0009BFF0346306000289AD00588002D7FF4F8
:10E6F00060AFFFF741FE35602846BDE8F081FFF7C7
:10E7000061FEC4F30740FFF75DFE072E02D1200E25
:10E71000FFF758FE534B584A198858481468584D0B
:10E72000524A017000270E0AF0201F802E701070D0
:10E730000CB301225348A0470120BDE8F081082B0B
:10E740007FF46EAF504B494A1B688021C4F30746E3
:10E750001170EDB2240E6BB328462246314698471D
:10E7600028E00B2E11D10B2B7FF45AAF474B3F4AB9
:10E770001B68B021EAE7464B1B68002B00F0FB80CA
:10E78000404898470120BDE8F0810C2E40F0008100
:10E790000C2B7FF445AF3F4B344A1B68C0211170EE
:10E7A000EDB2C4F30746002B00F0C880284631467E
:10E7B000240E98473849314A314B0D7016701C7041
:10E7C0000120BDE8F081354B1B68002B00F0D6809E
:10E7D0009847C4F30746254BEDB2240E83F800801A
:10E7E000E8E72F4B1B68002BF2D12E4B1B68A3B11F
:10E7F000FE209847C4F30746EDE72B4B1B68002B20
:10E80000E6D1284B1B6843B1FC209847C4F3074668
:10E81000E1E7264B1B68002BDAD1C4F30746DAE7A1
:10E82000234B1B68C4F30746002BD4D030469847CF
:10E83000D1E7204B1A68002AEFD0260C630C06F0B3
:10E840007F0003F47E531843F6B29047C3E71A4B98
:10E850001B68C4F30746002BE8D1BCE7ACA0FF1F40
:10E8600022A2FF1F1EA2FF1F88A0FF1F1CA2FF1FC6
:10E87000BCA0FF1F58A0FF1F84A0FF1F20A2FF1FE6
:10E8800021A2FF1F24A2FF1FB4A0FF1FB8A0FF1FDB
:10E890009CA0FF1F78A0FF1F23A2FF1F64A0FF1FE3
:10E8A00068A0FF1F6CA0FF1FA8A0FF1F98A0FF1F5C
:10E8B000B0A0FF1F80A0FF1F94A0FF1F3F4B1B684D
:10E8C000002B85D13E4B1B68002BA6D0FA20984721
:10E8D000C4F307467FE73B4B1B68002B7FF478AF00
:10E8E000374B1B68002B98D0FB209847C4F3074692
:10E8F00071E7354B1B68002B7FF46AAF304B1B6808
:10E90000002B8AD0F8209847C4F3074663E70E2B04
:10E910007FF486AE2D4A2E4B1268E0211970002A32
:10E9200047D0260C610C06F07F0301F47E51194399
:10E93000EDB2A1F5005128469047F6B2240E39E712
:10E94000FFF740FDC4F30740FFF73CFD200EFFF743
:10E9500039FD0020BDE8F0811E4B1D4A1B68802157
:10E960001170EDB2C4F3074683B1314628463A46EA
:10E9700098473C461EE70120BDE8F081104B1B681C
:10E98000002B3FF44AAFFF20984746E71C4611E7AB
:10E990000D2EBCD10D2B7FF443AE0F4B0C4A1B68E0
:10E9A000D0211170EDB2C4F30746002B7FF4FEAE08
:10E9B000C4E7C4F30746EDB2240EFBE690A0FF1FA8
:10E9C0006CA0FF1F70A0FF1F60A0FF1F7CA0FF1F97
:10E9D0001CA2FF1FB4A0FF1F8CA0FF1F38B5164D4F
:10E9E0002868E0B101884488A14213DD03191B7A2D
:10E9F00083B104F10803C2180C1B002302E012F8D3
:10EA0000011F21B10133A342F9D1204638BD1C4674
:10EA1000204638BDFFF7B0FC0020286038BD074B0A
:10EA20001B780BB9002038BD0220FEF7F5FD2860E9
:10EA30000028D7D1F6E700BFC8A0FF1F58A0FF1FCE
:10EA40000D4B1B78BBB910B50C4C216803F0FF02CD
:10EA50004B883F2B07DC07330B4401F1470003F8D9
:10EA6000012F8342FBD140230B800120FEF76CFE77
:10EA70000023236010BD7047C0A0FF1FC4A0FF1F6C
:10EA800038B5224C237803B138BD01232370FFF73A
:10EA9000A5FF70BB00F048F840BB00F0DBF810BBEE
:10EAA000FEF7F8FCE0B900232370EFF30583002B99
:10EAB000EAD1EFF3108172B6154B1868E0B1154C2E
:10EAC0002278CAB945691D6001232370C5B1AA61C6
:10EAD00001B962B600254577836898472570D3E76A
:10EAE00000F020F8DFE700F01BF8D9E700F016F897
:10EAF000D3E7FFF71FFCCDE70029C5D162B638BDCB
:10EB0000054B1D600029E5D1E3E700BFCDA0FF1F45
:10EB1000E49EFF1FE89EFF1FE09EFF1F704700BF9F
:10EB2000704700BF704700BF054A064B10781B783E
:10EB3000C0B2DBB2984238BF4030C01A704700BF45
:10EB4000D4A0FF1FD5A0FF1FF0B4384B1A7912F0E4
:10EB5000300F2CD072B6997D01F0FF0200293DD014
:10EB600062B6334F334938780D78334E1C46C0B205
:10EB7000EDB2431C402BE17928BF0023AB4202F1E8
:10EB8000FF32C9B21CBFF154184612F0FF02F0D197
:10EB90002A4B1B68C2B23A704BB1A84236BFC5F1CE
:10EBA0004005401B40192728C4BF01221A701F4985
:10EBB000CA78D2B2150616D452060DD51B4B1B7956
:10EBC0005B0609D51E4B1F491B6800220A7003B162
:10EBD0001A70164B3C22DA70F0BC70474022D9798B
:10EBE0005A7462B6E3E70B791C06E5D5164B174E4F
:10EBF0001C783378E4B2DBB29C420ED0144D01E0B5
:10EC0000A3420AD00133402B28BF00230879E85CD7
:10EC1000C0B2C871087D0728F2D9DBB2034933704E
:10EC20000B79180644BF7C23CB70C5E700A00640D3
:10EC3000D4A0FF1FD5A0FF1F18A1FF1FD0A0FF1F4A
:10EC40005CA1FF1F58A1FF1F60A1FF1F59A1FF1F5B
:10EC5000D8A0FF1F054A064B10781B78C0B2DBB264
:10EC6000984238BF4030C01A704700BFD4A1FF1F80
:10EC700069A1FF1FF0B4384B1A7912F0300F2CD075
:10EC800072B6997D01F0FF0200293DD062B6334F84
:10EC9000334938780D78334E1C46C0B2EDB2431C70
:10ECA000402BE17928BF0023AB4202F1FF32C9B209
:10ECB0001CBFF154184612F0FF02F0D12A4B1B681A
:10ECC000C2B23A704BB1A84236BFC5F14005401BF5
:10ECD00040192728C4BF01221A701F49CA78D2B22E
:10ECE000150616D452060DD51B4B1B795B0609D5AC
:10ECF0001E4B1F491B6800220A7003B11A70164B85
:10ED00003C22DA70F0BC70474022D9795A7462B65E
:10ED1000E3E70B791C06E5D5164B174E1C783378C4
:10ED2000E4B2DBB29C420ED0144D01E0A3420AD003
:10ED30000133282B28BF00230879E85CC0B2C871D2
:10ED4000087D0728F2D9DBB2034933700B79180626
:10ED500044BF7C23CB70C5E700B00640D4A1FF1FA1
:10ED600069A1FF1F94A1FF1F64A1FF1FD8A1FF1F6E
:10ED700068A1FF1FDCA1FF1FD5A1FF1F6CA1FF1F12
:10ED800070B584B072B6194B194D1A4870224126DD
:10ED90000F2480211A702E701A460470197013788F
:10EDA0001B06FCD5144B186862B6144B144C9842E1
:10EDB00098BF00EB800001A998BF40000A22FDF730
:10EDC000CFFE01A92046002311F8012B01333AB1EF
:10EDD0000A2B20F8022FF7D11623237004B070BD40
:10EDE0005B00DBB2237004B070BD00BF00000240C6
:10EDF0000700024006000240080002407F9698008B
:10EE00000893FF1FFFFFFFFF2DE9F043DFF8EC80C1
:10EE10008BB006460F4600F073F898F900300133C6
:10EE200004460D4637D03046394600F0DFF9002859
:10EE300031D02BA3D3E900233046394600F026FE1B
:10EE4000814668BB28A3D3E900233046394600F049
:10EE5000FFFD00B398F90030254ACDF82090042436
:10EE600000200021022BCDE90467CDE90267009460
:10EE70000192CDE906012CD0684600F0BDF940B3FF
:10EE8000089B1BB101F0AAF9089B0360DDE90601AC
:10EE90000BB0BDE8F083204629460BB0BDE8F083F7
:10EEA000134A98F90030019203210022CDE904674A
:10EEB000CDE90267009108922BB90E4B4FF06042EA
:10EEC000CDE90623D8E70C490020022BCDE9060145
:10EED000D2D101F083F922230360D1E7AFF30080A0
:10EEE000EF39FAFE422E864051302DD5104987C0A9
:10EEF000043A0100FFFFEF470000F07F1E93FF1F61
:10EF00002DE9F04FB04F21F00042BA4283B00C46D9
:10EF10004FEAD17605460DD9AC4FBA4225D9C1F397
:10EF20001303034340F0EF800EB10020014603B00D
:10EF3000BDE8F08FA64B9A4200F2CC80A54B9A42D6
:10EF400000F2DE808AA3D3E9002300F05DF90022FD
:10EF5000A14B00F09BFD002800F0058128462146CA
:10EF600000229D4B00F050F9E1E783A3D3E9002391
:10EF700000F08CFD002840F0CB802846214680A37D
:10EF8000D3E9002300F064FD0028CED1934B28463E
:10EF900003EBC60821467CA3D3E9002300F0E6FA80
:10EFA000D8E9002300F030F900F07AFD804600F047
:10EFB00077FA77A3D3E9002306460F4600F0D6FA86
:10EFC00002460B462846214600F01CF972A3D3E9FD
:10EFD0000023CDE900013046394600F0C7FA8246E9
:10EFE0008B4652465B46DDE9000100F00BF9054611
:10EFF0000C462A4623462846214600F0B7FA68A365
:10F00000D3E9002306460F4600F0B0FA66A3D3E921
:10F01000002300F0F7F832463B4600F0A7FA64A35D
:10F02000D3E9002300F0F0F832463B4600F09EFAA8
:10F0300061A3D3E9002300F0E5F832463B4600F037
:10F0400095FA5FA3D3E9002300F0DEF832463B4691
:10F0500000F08CFA02460B462846214600F0D2F812
:10F0600006460F462846214632463B46B8F1000F79
:10F0700056D000F07BFA324604460D463B4600204F
:10F080004FF0804100F0BEF802460B46204629466C
:10F0900000F096FB02460B465046594600F0B2F887
:10F0A000DDE9002300F0AEF80B4602464A49002095
:10F0B00000F0A8F86FF47F7398454FDA08F57A7876
:10F0C00001EB085100224FF0B87300F04FFA03B083
:10F0D000BDE8F08F424B9A423FF658AF414BF400E7
:10F0E0002344D3E9002300F08DF83F4BC6F101081B
:10F0F0001C44CDE90001D4E900ABC6EB080870E779
:10F100004FF0000875E702460B4600F07DF80EE769
:10F1100017A3D3E900231046194600F027FA06E7A3
:10F1200000F024FA0022804689464FF080433046A2
:10F13000394600F067F802460B464046494600F063
:10F140003FFB2A46234600F05DF802460B460020AE
:10F15000214900F057F803B0BDE8F08F01EB0851EA
:10F1600003B0BDE8F08F804643E700BFAFF30080F7
:10F170009C7500883CE4377EEF39FAFE422E8640CB
:10F1800051302DD5104987C0FE822B654715F73FBA
:10F190000000E0FE422EE63F763C7935EF39EA3D4D
:10F1A000D0A4BE726937663EF16BD2C541BDBB3E8D
:10F1B0002CDE25AF6A56113F93BDBE166CC1663F6B
:10F1C0003E5555555555C53F412E8640FFFFEF7FB3
:10F1D000422ED63FFFFF2F3E0000F03F083A0100CD
:10F1E000B1A2F03F283A0100183A010041F0004175
:10F1F00001F58010C00F70470020704781F000417A
:10F2000002E000BF83F0004330B54FEA41044FEA0B
:10F21000430594EA050F08BF90EA020F1FBF54EAA6
:10F22000000C55EA020C7FEA645C7FEA655C00F042
:10F23000E2804FEA5454D4EB5555B8BF6D420CDD13
:10F240002C4480EA020281EA030382EA000083EA96
:10F25000010180EA020281EA0303362D88BF30BD36
:10F2600011F0004F4FEA01314FF4801C4CEA11318C
:10F2700002D0404261EB410113F0004F4FEA0333EB
:10F280004CEA133302D0524263EB430394EA050F76
:10F2900000F0A780A4F10104D5F1200E0DDB02FAE5
:10F2A0000EFC22FA05F2801841F1000103FA0EF279
:10F2B000801843FA05F359410EE0A5F120050EF13F
:10F2C000200E012A03FA0EFC28BF4CF0020C43FA70
:10F2D00005F3C01851EBE37101F0004507D54FF07D
:10F2E000000EDCF1000C7EEB00006EEB0101B1F5CD
:10F2F000801F1BD3B1F5001F0CD349085FEA300013
:10F300004FEA3C0C04F101044FEA445212F5800F1D
:10F3100080F09A80BCF1004F08BF5FEA500C50F1BA
:10F32000000041EB045141EA050130BD5FEA4C0C9D
:10F33000404141EB010111F4801FA4F10104E9D126
:10F3400091F0000F04BF01460020B1FA81F308BF1D
:10F350002033A3F10B03B3F120020CDA0C3208DDE9
:10F3600002F1140CC2F10C0201FA0CF021FA02F1C4
:10F370000CE002F11402D8BFC2F1200C01FA02F134
:10F3800020FA0CFCDCBF41EA0C019040E41AA2BF59
:10F3900001EB0451294330BD6FEA04041F3C1CDA21
:10F3A0000C340EDC04F11404C4F1200220FA04F041
:10F3B00001FA02F340EA030021FA04F345EA0301EB
:10F3C00030BDC4F10C04C4F1200220FA02F001FAAD
:10F3D00004F340EA0300294630BD21FA04F029462F
:10F3E00030BD94F0000F83F4801306BF81F48011C8
:10F3F0000134013D4EE77FEA645C18BF7FEA655C3B
:10F4000029D094EA050F08BF90EA020F05D054EA0C
:10F41000000C04BF1946104630BD91EA030F1EBF11
:10F420000021002030BD5FEA545C05D14000494115
:10F4300028BF41F0004130BD14F580043CBF01F508
:10F44000801130BD01F0004545F0FE4141F47001EE
:10F450004FF0000030BD7FEA645C1ABF19461046C9
:10F460007FEA655C1CBF0B46024650EA013406BFCA
:10F4700052EA033591EA030F41F4002130BD00BF89
:10F4800090F0000F04BF0021704730B54FF4806446
:10F4900004F132044FF000054FF0000150E700BFC7
:10F4A00090F0000F04BF0021704730B54FF4806426
:10F4B00004F1320410F0004548BF40424FF0000113
:10F4C0003EE700BF42004FEAE2014FEA31014FEA56
:10F4D00002701FBF12F07F4393F07F4F81F06051A5
:10F4E000704792F0000F14BF93F07F4F704730B514
:10F4F0004FF4607401F0004521F0004120E700BFA7
:10F5000050EA010208BF704730B54FF000050AE02D
:10F5100050EA010208BF704730B511F0004502D52E
:10F52000404261EB41014FF4806404F132045FEA30
:10F53000915C3FF4DCAE4FF003025FEADC0C18BFD5
:10F5400003325FEADC0C18BF033202EBDC02C2F1CB
:10F55000200300FA03FC20FA02F001FA03FE40EA5D
:10F560000E0021FA02F11444C1E600BF70B54FF05D
:10F57000FF0C4CF4E06C1CEA11541DBF1CEA13553F
:10F5800094EA0C0F95EA0C0F00F0DEF82C4481EAA7
:10F59000030621EA4C5123EA4C5350EA013518BFC7
:10F5A00052EA033541F4801143F4801338D0A0FBB4
:10F5B00002CE4FF00005E1FB02E506F00042E0FB61
:10F5C00003E54FF00006E1FB03569CF0000F18BF67
:10F5D0004EF0010EA4F1FF04B6F5007F64F540740F
:10F5E00004D25FEA4E0E6D4146EB060642EAC621A2
:10F5F00041EA55514FEAC52040EA5E504FEACE2E0F
:10F60000B4F1FD0C88BFBCF5E06F1ED8BEF1004F11
:10F6100008BF5FEA500E50F1000041EB045170BD8D
:10F6200006F0004646EA010140EA020081EA0301D1
:10F63000B4EB5C04C2BFD4EB0C0541EA045170BDCD
:10F6400041F480114FF0000E013C00F3AB8014F147
:10F65000360FDEBF002001F0004170BDC4F1000490
:10F66000203C35DA0C341BDC04F11404C4F1200511
:10F6700000FA05F320FA04F001FA05F240EA02006C
:10F6800001F0004221F0004110EBD37021FA04F6A2
:10F6900042EB06015EEA430E08BF20EAD37070BD5C
:10F6A000C4F10C04C4F1200500FA04F320FA05F0BB
:10F6B00001FA04F240EA020001F0004110EBD370BD
:10F6C00041F100015EEA430E08BF20EAD37070BD2D
:10F6D000C4F1200500FA05F24EEA020E20FA04F306
:10F6E00001FA05F243EA020321FA04F001F00041B5
:10F6F00021FA04F220EA020000EBD3705EEA430E26
:10F7000008BF20EAD37070BD94F0000F0FD101F054
:10F710000046400041EB010111F4801F08BF013C8D
:10F72000F7D041EA060195F0000F18BF704703F0CB
:10F730000046520043EB030313F4801F08BF013D52
:10F74000F7D043EA0603704794EA0C0F0CEA13550E
:10F7500018BF95EA0C0F0CD050EA410618BF52EAC8
:10F760004306D1D181EA030101F000414FF00000CE
:10F7700070BD50EA410606BF1046194652EA4306DC
:10F7800019D094EA0C0F02D150EA013613D195EA50
:10F790000C0F05D152EA03361CBF104619460AD198
:10F7A00081EA030101F0004141F0FE4141F47001A2
:10F7B0004FF0000070BD41F0FE4141F4780170BD92
:10F7C00070B54FF0FF0C4CF4E06C1CEA11541DBFF7
:10F7D0001CEA135594EA0C0F95EA0C0F00F0A7F8F9
:10F7E000A4EB050481EA030E52EA03354FEA013126
:10F7F00000F088804FEA03334FF0805545EA131339
:10F8000043EA12634FEA022245EA111545EA106500
:10F810004FEA00260EF000419D4208BF964244F197
:10F82000FD0404F5407402D25B084FEA3202B61AB6
:10F8300065EB03055B084FEA32024FF480104FF48A
:10F84000002CB6EB020E75EB030E22BFB61A7546FE
:10F8500040EA0C005B084FEA3202B6EB020E75EB91
:10F86000030E22BFB61A754640EA5C005B084FEAF9
:10F870003202B6EB020E75EB030E22BFB61A7546C6
:10F8800040EA9C005B084FEA3202B6EB020E75EBD1
:10F89000030E22BFB61A754640EADC0055EA060E92
:10F8A00018D04FEA051545EA16754FEA06164FEAD5
:10F8B000C30343EA52734FEAC2025FEA1C1CC0D181
:10F8C00011F4801F0BD141EA00014FF000004FF00E
:10F8D000004CB6E711F4801F04BF01430020B4F1CF
:10F8E000FD0C88BFBCF5E06F3FF6AFAEB5EB030C87
:10F8F00004BFB6EB020C5FEA500C50F1000041EB84
:10F90000045170BD0EF0004E4EEA113114EB5C0450
:10F91000C2BFD4EB0C0541EA045170BD41F4801123
:10F920004FF0000E013C90E645EA060E8DE60CEA2B
:10F93000135594EA0C0F08BF95EA0C0F3FF43BAF48
:10F9400094EA0C0F0AD150EA01347FF434AF95EAFF
:10F950000C0F7FF425AF104619462CE795EA0C0FE3
:10F9600006D152EA03353FF4FDAE1046194622E7B0
:10F9700050EA410618BF52EA43067FF4C5AE50EA8A
:10F9800041047FF40DAF52EA43057FF4EBAE12E77A
:10F990004FF0FF3C06E000BF4FF0010C02E000BF5B
:10F9A0004FF0010C4DF804CD4FEA410C7FEA6C5C3E
:10F9B0004FEA430C18BF7FEA6C5C1BD001B050EAE1
:10F9C000410C0CBF52EA430C91EA030F02BF90EACC
:10F9D000020F0020704710F1000F91EA030F58BF8B
:10F9E000994208BF90422CBFD8176FEAE37040F0ED
:10F9F000010070474FEA410C7FEA6C5C02D150EA8B
:10FA0000013C07D14FEA430C7FEA6C5CD6D152EA45
:10FA1000033CD3D05DF8040B704700BF844610460A
:10FA200062468C461946634600E000BF01B5FFF709
:10FA3000B7FF002848BF10F1000F01BD4DF808EDD9
:10FA4000FFF7F4FF0CBF012000205DF808FB00BFAA
:10FA50004DF808EDFFF7EAFF34BF012000205DF804
:10FA600008FB00BF4DF808EDFFF7E0FF94BF012051
:10FA700000205DF808FB00BF4DF808EDFFF7CEFF52
:10FA800094BF012000205DF808FB00BF4DF808ED91
:10FA9000FFF7C4FF34BF012000205DF808FB00BF62
:10FAA0004FEA410212F5001215D211D56FF47873A6
:10FAB000B3EB625212D94FEAC12343F0004343EA49
:10FAC000505311F0004F23FA02F018BF4042704724
:10FAD0004FF00000704750EA013005D111F00040AE
:10FAE00008BF6FF0004070474FF00000704700BF44
:10FAF0004FEA4102B2F1E04324BFB3F5001CDCF150
:10FB0000FE5C0DD901F0004C4FEAC0024CEA507087
:10FB1000B2F1004F40EB830008BF20F001007047B6
:10FB200011F0804F21D113F13872BCBF01F00040B9
:10FB3000704741F480114FEA5252C2F11802C2F1EB
:10FB4000200C10FA0CF320FA02F018BF40F001006C
:10FB50004FEAC1234FEAD32303FA0CFC40EA0C001E
:10FB600023FA02F34FEA4303CCE77FEA625307D15B
:10FB700050EA01331EBF4FF0FE4040F44000704792
:10FB800001F0004040F0FE4040F40000704700BF2C
:10FB900080F0004002E000BF81F0004142001FBF42
:10FBA0005FEA410392EA030F7FEA226C7FEA236C4B
:10FBB0006AD04FEA1262D2EB1363C1BFD218414040
:10FBC00048404140B8BF5B42192B88BF704710F0D6
:10FBD000004F40F4000020F07F4018BF404211F079
:10FBE000004F41F4000121F07F4118BF494292EAE1
:10FBF000030F3FD0A2F1010241FA03FC10EB0C000D
:10FC0000C3F1200301FA03F100F0004302D5494299
:10FC100060EB4000B0F5000F13D3B0F1807F06D346
:10FC200040084FEA310102F10102FE2A51D2B1F13E
:10FC3000004F40EBC25008BF20F0010040EA030033
:10FC40007047490040EB000010F4000FA2F10102E0
:10FC5000EDD1B0FA80FCACF1080CB2EB0C0200FA6A
:10FC60000CF0AABF00EBC25052421843BCBFD040B8
:10FC70001843704792F0000F81F4000106BF80F432
:10FC800000000132013BB5E74FEA41037FEA226CF5
:10FC900018BF7FEA236C21D092EA030F04D092F0C0
:10FCA000000F08BF0846704790EA010F1CBF0020F4
:10FCB000704712F07F4F04D1400028BF40F0004051
:10FCC000704712F100723CBF00F50000704700F071
:10FCD000004343F0FE4040F4000070477FEA226298
:10FCE00016BF08467FEA23630146420206BF5FEA69
:10FCF000412390EA010F40F4800070474FF0000369
:10FD000004E000BF10F0004348BF40425FEA000C2F
:10FD100008BF704743F0964301464FF000001CE0D7
:10FD200050EA010208BF70474FF000030AE000BF2D
:10FD300050EA010208BF704711F0004302D540426B
:10FD400061EB41015FEA010C02BF844601460020DD
:10FD500043F0B64308BFA3F18053A3F50003BCFAF8
:10FD60008CF2083AA3EBC25310DB01FA02FC6344A5
:10FD700000FA02FCC2F12002BCF1004F20FA02F2AC
:10FD800043EB020008BF20F00100704702F120029F
:10FD900001FA02FCC2F1200250EA4C0021FA02F200
:10FDA00043EB020008BF20EADC7070474FF0FF0C05
:10FDB0001CEAD0521EBF1CEAD15392EA0C0F93EA00
:10FDC0000C0F6FD01A4480EA010C400218BF5FEAA2
:10FDD00041211ED04FF0006343EA501043EA511115
:10FDE000A0FB01310CF00040B1F5000F3EBF49000F
:10FDF00041EAD3715B0040EA010062F17F02FD2A13
:10FE00001DD8B3F1004F40EBC25008BF20F00100F5
:10FE1000704790F0000F0CF0004C08BF49024CEA0C
:10FE2000502040EA51207F3AC2BFD2F1FF0340EA9E
:10FE3000C250704740F400004FF00003013A5DDC0F
:10FE400012F1190FDCBF00F000407047C2F1000250
:10FE5000410021FA02F1C2F1200200FA02FC5FEA3D
:10FE6000310040F1000053EA4C0308BF20EADC7087
:10FE7000704792F0000F00F0004C02BF400010F4F9
:10FE8000000F013AF9D040EA0C0093F0000F01F0A6
:10FE9000004C02BF490011F4000F013BF9D041EAC8
:10FEA0000C018FE70CEAD15392EA0C0F18BF93EACA
:10FEB0000C0F0AD030F0004C18BF31F0004CD8D1F4
:10FEC00080EA010000F00040704790F0000F17BF7B
:10FED00090F0004F084691F0000F91F0004F14D0C1
:10FEE00092EA0C0F01D142020FD193EA0C0F03D119
:10FEF0004B0218BF084608D180EA010000F000401C
:10FF000040F0FE4040F40000704740F0FE4040F4F6
:10FF1000400070474FF0FF0C1CEAD0521EBF1CEA95
:10FF2000D15392EA0C0F93EA0C0F69D0A2EB0302B3
:10FF300080EA010C49024FEA402037D04FF080534D
:10FF400043EA111143EA10130CF000408B4238BF12
:10FF50005B0042F17D024FF4000C8B4224BF5B1A20
:10FF600040EA0C00B3EB510F24BFA3EB510340EA6E
:10FF70005C00B3EB910F24BFA3EB910340EA9C001C
:10FF8000B3EBD10F24BFA3EBD10340EADC001B018C
:10FF900018BF5FEA1C1CE0D1FD2A3FF650AF8B4230
:10FFA00040EBC25008BF20F0010070470CF0004C3D
:10FFB0004CEA50207F32C2BFD2F1FF0340EAC25068
:10FFC000704740F400004FF00003013A37E792F029
:10FFD000000F00F0004C02BF400010F4000F013A87
:10FFE000F9D040EA0C0093F0000F01F0004C02BF82
:10FFF000490011F4000F013BF9D041EA0C0195E7EB
:020000021000EC
:100000000CEAD15392EA0C0F08D142027FF47DAF83
:1000100093EA0C0F7FF470AF084676E793EA0C0F73
:1000200004D14B023FF44CAF08466EE730F0004C71
:1000300018BF31F0004CCAD130F000427FF45CAF01
:1000400031F000437FF43CAF5FE700BF4FF0FF3C6F
:1000500006E000BF4FF0010C02E000BF4FF0010CC2
:100060004DF804CD4FEA40024FEA41037FEA226C8B
:1000700018BF7FEA236C11D001B052EA530C18BFAD
:1000800090EA010F58BFB2EB030088BFC81738BF12
:100090006FEAE17018BF40F0010070477FEA226C00
:1000A00002D15FEA402C05D17FEA236CE4D15FEAFC
:1000B000412CE1D05DF8040B704700BF8446084630
:1000C0006146FFE70FB5FFF7C9FF002848BF10F1F1
:1000D000000F0FBD4DF808EDFFF7F4FF0CBF012036
:1000E00000205DF808FB00BF4DF808EDFFF7EAFFC0
:1000F00034BF012000205DF808FB00BF4DF808ED7B
:10010000FFF7E0FF94BF012000205DF808FB00BF6F
:100110004DF808EDFFF7D2FF94BF012000205DF8F5
:1001200008FB00BF4DF808EDFFF7C8FF34BF012002
:1001300000205DF808FB00BF4FEA4002B2F1FE4F1D
:100140000FD34FF09E03B3EB12620DD94FEA002399
:1001500043F0004310F0004F23FA02F018BF404272
:1001600070474FF00000704712F1610F01D1420259
:1001700005D110F0004008BF6FF0004070474FF00D
:100180000000704742000ED2B2F1FE4F0BD34FF089
:100190009E03B3EB126209D44FEA002343F00043FD
:1001A00023FA02F070474FF00000704712F1610F20
:1001B00001D1420202D14FF0FF3070474FF00000F2
:1001C000704700BF0B460146184600F001B800BF5B
:1001D00013460A460146022000F0C4BE014B1868CF
:1001E000704700BF4897FF1F70B50F4E0F4D761B2D
:1001F000B61018BF002405D0013455F8043B9847C9
:10020000A642F9D10A4E0B4D761B03F017FCB6102F
:1002100018BF002406D0013455F8043B9847A64285
:10022000F9D170BD70BD00BF483A0100483A0100E5
:100230005C3A0100483A0100024B0146186800F0A0
:100240000BB800BF4897FF1F024B0146186800F02B
:100250004DBF00BF4897FF1F2DE9F04F01F10B057F
:10026000162D83B0064640F29F8035F0070500F159
:10027000BF80A94200F2BC8000F058FBB5F5FC7FBE
:10028000C0F09C826B0A00F0BA80042B00F28381DC
:10029000A80900F1390E4FEA4E033830C44F07EB7E
:1002A0008303A3F108015C68A14207D1ACE0002AF6
:1002B00080F2AC80E468A14200F0A680636823F07D
:1002C00003035A1B0F2AF2DDB9493C6901F1080EFC
:1002D000744500F0B381636823F003035A1B0F2AAF
:1002E00000F39981002AC1F814E0C1F810E080F20F
:1002F0009E80B3F5007F80F06781DB0803F1010C7D
:1003000001229B1002FA03F34A6851F83C80C4F8BA
:10031000088001EBCC091A43A9F10803E3604A60A5
:1003200041F83C40C8F80C40831001249C409442A2
:1003300000F28A80144206D120F0030064001442C7
:1003400000F10400FAD007EBC009CC468046DCF887
:100350000C108C4507D173E1002A80F28181C968B5
:100360008C4500F06D814B6823F003035A1B0F2A64
:10037000F2DD0C46D1F80CC054F8088F4B1945F04B
:1003800001054D6042F00101C8F80CC03046CCF8C0
:1003900008807B613B61C3F80CE0C3F808E059605A
:1003A0009A5000F0C5FA1FE0102921D800F0BEFADB
:1003B0001025062302207E4F07EB8303A3F10802DA
:1003C0005C68944200F045816368E168A56823F0A9
:1003D0000303234430465A68E96042F001028D600D
:1003E0005A6000F0A5FA0834204603B0BDE8F08F4B
:1003F00000240C232046336003B0BDE8F08F802337
:100400004FF0400E3F2049E770465DE72344E16826
:100410005A68A56842F00102E96030468D605A6072
:1004200000F086FA0834204603B0BDE8F08F23447C
:1004300030465A6842F001025A6000F079FA0834F6
:10044000204603B0BDE8F08FBC68636823F0030862
:10045000A84504D3C5EB08030F2B00F38C80554B44
:10046000DFF860911A68D9F8003001332A4404EBB0
:10047000080A00F0608102F580520F3222F47F6298
:1004800022F00F0211463046019200F04BFCB0F111
:10049000FF3F8346019A00F05881824500F2FC80BC
:1004A000454B1968DA451144196000F05381D9F8B9
:1004B0000000DFF810E101301BBFCAEB0B0A51440A
:1004C000CEF800B019601BF0070100F01781C1F1F0
:1004D0000800C1F58051834408315A44C2F30B022D
:1004E000C2EB010949463046019300F01BFC431C56
:1004F000019B00F03F81CBEB00024A4442F0010235
:100500001968C7F808B04944BC42CBF80420196008
:10051000DFF8A49016D0B8F10F0F40F2FD806268AA
:10052000A8F10C0323F00703E01802F001024FF0DA
:10053000050E1A430F2B6260C0F804E0C0F808E013
:1005400000F21C811D4BBC681A68914288BF19607B
:100550001B4B1A689142626888BF196022F003023F
:100560009542A2EB050301D80F2B04DC304600F0C6
:10057000DFF9002438E7621943F0010345F0010573
:1005800065603046BA60536000F0D2F90834204606
:1005900003B0BDE8F08F142B71D9542B00F2A48066
:1005A000280B00F16F0E4FEA4E036E3076E600BF67
:1005B0004C97FF1FE8A1FF1FECA1FF1FE4A1FF1F45
:1005C000E0A1FF1F589BFF1F5A0A042A5ED9142A74
:1005D00000F2B38002F15C0149005B3207EB810C51
:1005E00057F82110DFF8DC81ACF1080C8C4500F0E5
:1005F00088804A6822F00302934202D289688C45BF
:10060000F7D1D1F80CC07A68C4F80CC0A160CCF85E
:100610000840CC6088E6631942F0010745F0010507
:10062000656030464B610B61C3F80CE0C3F808E02D
:100630005F609A50083400F07BF9D5E64A6873E6AB
:1006400008F1010818F0030F0CF1080C7FF47FAEDD
:1006500030E0DC68A34208BF02303FF435AEB3E6B9
:100660000B440C465A68C96854F8085F42F001020E
:100670005A603046E9608D6000F05AF9B4E603F143
:100680005C0E03F15B004FEA4E0307E69A0902F1A4
:10069000390149003832A1E7BC424A4B3FF400AF70
:1006A0009C68626822F003025AE759F808399945B4
:1006B00040F0828010F0030F00F1FF30F5D17B682D
:1006C00023EA04037B6064009C423FF6BDAE002C2D
:1006D0003FF4BAAE1C4240467FF435AE64001C4283
:1006E00000F10400FAD02EE6B3F5AA7F18D8E80B83
:1006F00000F1780E4FEA4E037730CFE54FF480518A
:10070000EBE60121D8F80430921001FA02F21A4304
:10071000C8F80420614677E70123CBF8043025E7C9
:1007200040F25452934220D8A80C00F17D0E4FEABB
:100730004E037C30B2E51032A4E6542A26D81A0BB8
:1007400002F16F0149006E3248E7BC68626822F02E
:10075000030205E7CAF30B0000287FF4A8AE424469
:10076000BB6842F001025A60ECE6FE234FF07F0EB8
:100770007E2093E501224FF00009C1E604F1080153
:10078000304600F0B3FCD9F80010DBE6B2F5AA7FE2
:1007900005D8DA0B02F17801490077321EE740F202
:1007A00054518A4205D89A0C02F17D0149007C32ED
:1007B00014E7FE217E2211E77B6884E7E808431CEA
:1007C0005B00F8E54C97FF1F8842F0B50DD98B18F8
:1007D00098420AD28118002A51D09A1A13F8014D72
:1007E00001F8014D9342F9D1F0BD0F2A48D941EAF1
:1007F00000039B0746D100F1100401F110031546D8
:1008000053F8106C44F8106C53F80C6C44F80C6CF2
:1008100053F8086C44F8086C103D53F8046C44F825
:10082000046C0F2D03F1100304F11004E8D8A2F1B9
:10083000100323F00F0302F00F0E1033BEF1030F6D
:100840001944034421D91E1F0D467446043C55F833
:10085000047B46F8047F032CF8D8AEF1040424F09E
:10086000030404342344214402F0030262B1013B37
:100870000A4411F8014B03F8014F8A42F9D1F0BD47
:100880000346F3E70346F2E7F0BD7246EEE700BF2A
:1008900070B4840746D0541E002A41D0CDB203461E
:1008A00002E0621EE4B3144603F8015B9A07F8D134
:1008B000032C2ED9CDB245EA05250F2C45EA054576
:1008C00019D903F110022646103E0F2E42F8105C93
:1008D00042F80C5C42F8085C42F8045C02F1100239
:1008E000F2D8A4F1100222F00F0204F00F0410322B
:1008F000032C13440DD91E462246043A032A46F817
:10090000045BFAD8221F22F003020432134404F0DD
:1009100003042CB1C9B21C4403F8011BA342FBD150
:1009200070BC704714460346C2E700BF704700BF63
:10093000704700BF024B0A460146186800F002B833
:100940004897FF1F2DE9F04F174683B0002900F0AC
:10095000C1800E46814607F10B05FFF7E7FF56F809
:1009600004EC162D2EF00304A6F1080840D810223E
:100970001546AF4241D8944275DAC94B996808EBE5
:1009800004008842416800F0D98021F0010303444B
:100990005B68DB077DD51EF0010F35D03946484630
:1009A000FFF75AFC0746E0B156F8043C23F0010378
:1009B0004344A0F108029A4200F04481221F242AF5
:1009C00000F23181132A00F2048103463246116895
:1009D00019605168596092689A603146484600F043
:1009E00085FB4846FFF7A4FF384603B0BDE8F08F0B
:1009F00025F00705002D2A46BBDA0C230020C9F894
:100A0000003003B0BDE8F08F56F8083CC3EB080A8D
:100A1000DAF8043023F0030C04EB0C039342BDDB43
:100A20005746DAF80C1057F8080F221F242AC16025
:100A3000886000F21781132A40F212813168CAF8E7
:100A400008107168CAF80C101B2A00F22B810836B6
:100A50000AF110023168116071685160B1689160EB
:100A60003E461C46D046631B0F2B1DD8D8F80430D9
:100A700003F0010323434444C8F80430636843F09F
:100A8000010363604846FFF753FF304603B0BDE8FB
:100A9000F08F21F003012144914221DBC368826879
:100AA0000C46D3609A60DEE7D8F8042008EB050115
:100AB00002F00102154343F001020B44C8F8045050
:100AC0004A605A6842F0010208315A60484600F014
:100AD0000DFBD7E7114603B0BDE8F04FFFF7BCBBF5
:100AE0001EF0010F7FF45AAF56F8083CC3EB080A1A
:100AF000DAF8043023F0030C01EB0C0E96458BDB87
:100B0000C36882685746D3609A6057F8081FDAF8BE
:100B10000C30CB60221F242A996000F29980132A9E
:100B200062D93368CAF808307368CAF80C301B2AD7
:100B300000F2A08008360AF1100356E021F0030B02
:100B4000A34405F11000834559DA1EF0010F7FF42C
:100B500025AF56F8081CC1EB080ADAF8041021F09A
:100B6000030CE34458453FF757AF5746DAF80C10EB
:100B700057F8080F221F242AC160886000F2B48051
:100B8000132A40F2A5803168CAF808107168CAF8C3
:100B90000C101B2A00F2AF8008360AF110023168EF
:100BA000116071685160B16891600AEB0501C5EB95
:100BB0000B0242F0010299604A60DAF8043003F057
:100BC00001031D434846CAF80450FFF7B1FE3846FA
:100BD0005CE733680360736843601B2A27D800F121
:100BE000080306F10802F2E63B4632681A607268B2
:100BF0005A60B2689A603E467446D04633E708EBC6
:100C00000501C5EB0B0B4BF0010299604A6056F8E9
:100C1000043C03F001031D43484646F8045CFFF71B
:100C200087FE304632E73146FFF7CEFDD5E6B368A2
:100C30008360F368C360242A28D000F1100306F112
:100C40001002C4E650F8043C23F003031C440AE7F6
:100C5000314638467446D046FFF7B6FD3E4602E7B9
:100C60003A46F7E6314638461C46D046FFF7ACFD1B
:100C70003E46F8E6B368CAF81030F368CAF8143094
:100C8000242A1BD010360AF11803AEE7336903613A
:100C90007369436106F1180200F1180397E600BF7B
:100CA0004C97FF1FB168CAF81010F168CAF8141009
:100CB000242A0FD010360AF11802CBE63369CAF89D
:100CC00018307369CAF81C3018360AF120038CE713
:100CD0003A4664E73269CAF818207269CAF81C20DB
:100CE00018360AF12002B5E6314638460193FFF77F
:100CF0006BFD019B59E7B168CAF81010F168CAF89A
:100D00001410242A03D010360AF1180247E732697A
:100D1000CAF818207269CAF81C2018360AF1200295
:100D20003DE700BF38B5074C002305460846236061
:100D3000FBF7E0FE431C00D038BD2368002BFBD03E
:100D40002B6038BD48A3FF1FFFFFFFFFFFFFFFFF22
:100D5000FFFFFFFFFFFFFFFFFFFFFFFFFFFFFFFFA3
:100D6000FFFFFFFFFFFFFFFFFFFFFFFFFFFFFFFF93
:100D7000FFFFFFFFFFFFFFFFFFFFFFFFFFFFFFFF83
:100D800090F800F06DE9024520F007016FF0000CCB
:100D900010F0070491F820F040F049804FF0000473
:100DA0006FF00700D1E9002391F840F000F108004E
:100DB00082FA4CF2A4FA8CF283FA4CF3A2FA8CF386
:100DC0004BBBD1E9022382FA4CF200F10800A4FAED
:100DD0008CF283FA4CF3A2FA8CF3E3B9D1E9042341
:100DE00082FA4CF200F10800A4FA8CF283FA4CF378
:100DF000A2FA8CF37BB9D1E9062301F1200182FA32
:100E00004CF200F10800A4FA8CF283FA4CF3A2FA37
:100E10008CF3002BC6D0002A04BF04301A4612BA45
:100E2000B2FA82F2FDE8024500EBD2007047D1E948
:100E3000002304F00305C4F100004FEAC50514F0D7
:100E4000040F91F840F00CFA05F562EA05021CBFA8
:100E500063EA050362464FF00004A9E7002A41D087
:100E600040EA010313F00303F0B425D1032A23D988
:100E700004680D68AC421FD1043A35D0A4F10135A5
:100E800025EA040414F0803F31D1071D0D1D0DE04B
:100E900057F8043B0E68A3F10134B34224EA03047B
:100EA0000AD1043A20D014F0803F23D1032A2946E6
:100EB000384605F10405EBD803780C789C4202F122
:100EC000FF320CD182B114B916E06AB17BB110F8CF
:100ED000013F11F8014FA34202F1FF32F5D0181B78
:100EE000F0BC7047104670471046F0BC704718467B
:100EF000F0BC70470020F3E72046F1E740EA010329
:100F00009B0770B42BD1032A29D90C4603462146EE
:100F100054F8046BA6F1013525EA060515F0803F6B
:100F200006D1043A032A43F8046B2146EFD8A2B154
:100F30000C781C70013A013301313CB16AB111F8EF
:100F4000014B03F8014B013A002CF7D12AB11A44A6
:100F5000002103F8011B9A42FBD170BC7047034685
:100F6000E5E700BF2DE9F047254C2568D5F8484155
:100F70000646884692469946C4B360681F2817DC27
:100F8000431C76B104EB80050122C5F888A0D4F893
:100F9000881182401143022EC4F88811C5F80891C7
:100FA0001ED00230636044F820800020BDE8F08746
:100FB000144B03B34FF4C870FFF73EF90446D0B1A9
:100FC000D5F84831002780E88800C5F84841384600
:100FD0000123C4F88871C4F88C71002EE1D0D1E7E8
:100FE000D4F88C110A43C4F88C21DAE705F5A6740D
:100FF000C5F84841C1E74FF0FF30BDE8F08700BFBA
:10100000383A010039020100024B13B1024800F0E6
:1010100005B87047000000002910010000230146B8
:101020001A461846FFF79EBF38B5074D074C2C1BD4
:10103000A41005D0013C55F8043D9847002CF9D187
:10104000BDE8384002F00ABD0000000000000000CA
:10105000F8B5234F0C460646FFF768FCBB685D6891
:1010600025F00305291B01F6EF7121F47F6121F0C2
:101070000F01A1F58054B4F5805F07DB00213046F5
:10108000FFF750FEBB682B44984204D03046FFF770
:101090004FFC0020F8BD61423046FFF743FE0130AF
:1010A0000DD0104BBA6819682D1B45F0010530466C
:1010B000091B55601960FFF73BFC0120F8BD0021BA
:1010C0003046FFF72FFEBA68831A0F2BDEDD064C81
:1010D0000449246843F00103001B53600860D5E70E
:1010E0004C97FF1FECA1FF1F589BFF1F002945D005
:1010F0002DE9F0410D468046FFF718FC55F8047CB9
:101100006A4927F00103A5F10804E2188E685068C7
:10111000B24220F0030062D0FE0750600BD455F8B5
:10112000087CE41B01F1080EA56875453B446FD0AF
:10113000E768EF60BD6015186D68ED0742D543F0B4
:1011400001026260E350B3F5007F18D2DB085A1C3D
:101150004D6851F83270A76001209B1000FA03F32C
:1011600001EBC2001D430838E0604D6041F8324099
:10117000FC604046BDE8F041FFF7DABB70475A0A11
:10118000042A53D89A0902F139077F0002F1380581
:1011900001EB870051F827204449083890424DD090
:1011A000516821F003018B4202D292689042F7D13C
:1011B000D068E060A2608460D4604046BDE8F04141
:1011C000FFF7B6BB95683A4FBD4203443FD0D068A5
:1011D000E86043F0010285606260E350B3E7FF0717
:1011E000034407D455F8082CA41A1344A068E268F5
:1011F000C26090602F4A126843F001009342606021
:101200008C60B6D32C4B40461968FFF721FFB0E73E
:1012100011184968C90744D49168D268CA60034468
:1012200043F0010091606060E350A2E7142A17D8F0
:1012300002F15C077F0002F15B05A9E7AA104B6889
:10124000012505FA02F213434B600246B1E743F071
:1012500001024C610C61E560A5606260E35088E7C3
:10126000542A06D81A0B02F16F077F0002F16E05AF
:101270008EE7B2F5AA7F06D8DA0B02F178077F0075
:1012800002F1770584E740F25450824206D89A0C66
:1012900002F17D077F0002F17C0579E7FE277E25BC
:1012A00076E743F001026260E35062E74C97FF1F6C
:1012B0005497FF1F549BFF1FE8A1FF1F00007805F4
:1012C0003408540B800C3C0F5C12E015FA19141E04
:1012D0006022AC265C2B0C30BC34023AFF3FFFFF8F
:1012E000FDFFFFFFFBFFFFFFF8FFFFFFFDFFFFFF1D
:1012F000FBFFFFFFF8FFFFFFFDFFFFFFFAFFFFFF10
:10130000F7FFFFFFFDFFFFFFFBFFFFFFF7FFFFFF03
:10131000FCFFFFFFFBFFFFFFF7FFFFFFFDFFFFFFEE
:10132000FAFFFFFFF7FFFFFFFDFFFFFFFBFFFFFFE0
:10133000F8FFFFFFFDFFFFFFFBFFFFFFF8FFFFFFD1
:10134000FDFFFFFFFAFFFFFFF7FFFFFFFCFFFFFFBF
:10135000FBFFFFFFF7FFFFFFFDFFFFFFFBFFFFFFAF
:10136000F7FFFFFFFDFFFFFFFAFFFFFFF7FFFFFFA4
:10137000FDFFFFFFFBFFFFFFF7FFFFFFFDFFFFFF8D
:10138000FBFFFFFFF7FFFFFFFDFFFFFFFAFFFFFF80
:10139000F7FFFFFFFDFFFFFFFAFFFFFFF8FFFFFF73
:1013A000FDFFFFFFFAFFFFFFF7FFFFFFFDFFFFFF5E
:1013B000FAFFFFFFF7FFFFFFFDFFFFFFFAFFFFFF51
:1013C000F8FFFFFFFDFFFFFFFAFFFFFFF8FFFFFF42
:1013D000FDFFFFFFFAFFFFFFF7FFFFFFFCFFFFFF2F
:1013E000FBFFFFFFF7FFFFFFFDFFFFFFFAFFFFFF20
:1013F000F7FFFFFFFDFFFFFFFAFFFFFFF7FFFFFF14
:10140000FEFFFFFFFBFFFFFFF8FFFFFFFEFFFFFFF9
:10141000FBFFFFFFF8FFFFFFFDFFFFFFFAFFFFFFEE
:10142000F7FFFFFFFCFFFFFFFAFFFFFFF7FFFFFFE4
:10143000FCFFFFFFFAFFFFFFF7FFFFFFFDFFFFFFCE
:10144000FAFFFFFFF7FFFFFFFDFFFFFFF9FFFFFFC1
:10145000F7FFFFFFFDFFFFFFF9FFFFFFF7FFFFFFB4
:10146000FDFFFFFFFAFFFFFFF7FFFFFFFDFFFFFF9D
:10147000FAFFFFFFF7FFFFFFFDFFFFFFFAFFFFFF90
:10148000F6FFFFFFFDFFFFFFFAFFFFFFF7FFFFFF84
:10149000FEFFFFFFFBFFFFFFF7FFFFFFFEFFFFFF6A
:1014A000FBFFFFFFF7FFFFFFFDFFFFFFFAFFFFFF5F
:1014B000F7FFFFFFFDFFFFFFFBFFFFFFF8FFFFFF51
:1014C000FDFFFFFFFBFFFFFFF8FFFFFFFDFFFFFF3B
:1014D000FAFFFFFFF7FFFFFFFCFFFFFFF9FFFFFF32
:1014E000F7FFFFFFFCFFFFFFF9FFFFFFF7FFFFFF25
:1014F000FDFFFFFFFAFFFFFFF7FFFFFFFDFFFFFF0D
:10150000FAFFFFFFF7FFFFFFFDFFFFFFF9FFFFFF00
:10151000F6FFFFFFFDFFFFFFFAFFFFFFF7FFFFFFF3
:10152000D81A0100B41A0100901A01006C1A0100C7
:1015300024170100E015010004160100281601001F
:101540004C1601008C180100B0180100BC120100FB
:101550004817010000000000070000000C00000018
:101560001000000013000000180000001C00000024
:1015700000000000070000000C0000001300000045
:10158000180000001F000000240000000000000000
:101590000C000000180000002400000030000000D3
:1015A0003C0000004800000000000000FBFFFFFFBF
:1015B000F4FFFFFFEFFFFFFFE8FFFFFFE3FFFFFF89
:1015C000DCFFFFFF00000000F4FFFFFFE8FFFFFF6C
:1015D000DCFFFFFFD0FFFFFFC4FFFFFFB8FFFFFFEF
:1015E0000000580246056608540BD80E5C12E01540
:1015F000FA19141E6022AC265C2B0C30BC34023A63
:10160000FF3FFFFF0000900120031405D0075A0A96
:10161000AC0DCC10B4146A18E81C342180252A2B98
:1016200070301437FF3FFFFF0000C800F40184034F
:10163000140508072E091C0CD80EF811AE159619C2
:10164000401F1C25F22B5834FF3FFFFF00006400B1
:10165000C8009001BC021A04DC059E07F609800C44
:10166000A00F2413A2174C1D5424442FFF3FFFFF4B
:10167000FBFFFFFFF8FFFFFFF4FFFFFFFAFFFFFF95
:10168000F7FFFFFFF4FFFFFFFDFFFFFFF9FFFFFF85
:10169000F4FFFFFFFAFFFFFFF7FFFFFFF4FFFFFF7D
:1016A000FCFFFFFFF7FFFFFFF4FFFFFFFBFFFFFF64
:1016B000F8FFFFFFF4FFFFFFFDFFFFFFFAFFFFFF53
:1016C000F4FFFFFFFDFFFFFFF9FFFFFFF4FFFFFF48
:1016D000FDFFFFFFF8FFFFFFF4FFFFFFFCFFFFFF31
:1016E000F7FFFFFFF4FFFFFFFBFFFFFFF8FFFFFF28
:1016F000F4FFFFFFFCFFFFFFF7FFFFFFF4FFFFFF1B
:1017000040067805B004E80384032003BC025802B5
:10171000F40190012C01FA00C80096006400320028
:101720001900FFFF0000FF03FF07FF0BFF0FFF1370
:10173000FF17FF1BFF1FFF23FF27FF2BFF2FFF3389
:10174000FF37FF3BFF3FFFFF0000D007800CD80EA4
:101750000010C012EC130C17FA19141E6022AC26EC
:101760005C2B0C30BC34023AFF3FFFFFFBFFFFFF56
:10177000F8FFFFFFF4FFFFFFFAFFFFFFF7FFFFFF98
:10178000F4FFFFFFFDFFFFFFF9FFFFFFF4FFFFFF87
:10179000FAFFFFFFF7FFFFFFF4FFFFFFFCFFFFFF74
:1017A000F7FFFFFFF4FFFFFFFBFFFFFFF8FFFFFF67
:1017B000F4FFFFFFFDFFFFFFFAFFFFFFF4FFFFFF56
:1017C000FBFFFFFFF8FFFFFFF4FFFFFFFDFFFFFF41
:1017D000F8FFFFFFF4FFFFFFFCFFFFFFF7FFFFFF36
:1017E000F4FFFFFFFBFFFFFFF8FFFFFFF4FFFFFF2A
:1017F000FCFFFFFFF7FFFFFFF4FFFFFFFBFFFFFF13
:10180000F8FFFFFFF6FFFFFFFAFFFFFFF8FFFFFF04
:10181000F6FFFFFFFDFFFFFFFBFFFFFFF9FFFFFFED
:10182000FDFFFFFFF9FFFFFFF7FFFFFFFEFFFFFFD9
:10183000FCFFFFFFF7FFFFFFFBFFFFFFF8FFFFFFCE
:10184000F6FFFFFFFCFFFFFFFAFFFFFFF6FFFFFFC2
:10185000FDFFFFFFFBFFFFFFF9FFFFFFFCFFFFFFA7
:10186000FAFFFFFFF6FFFFFFFEFFFFFFFCFFFFFF9A
:10187000F7FFFFFFFBFFFFFFF8FFFFFFF6FFFFFF94
:10188000FEFFFFFFFCFFFFFFF7FFFFFF0000580216
:1018900046056608540BD80E5C127017FC21F82A16
:1018A00070305834DC37663A8C3C803EFF3FFFFF97
:1018B0000000580246056608540BA00FD4172823D1
:1018C000F82A442F643284354038663A8C3C803E96
:1018D000FF3FFFFF00000000070000000C000000B9
:1018E00010000000130000001A0000001F0000009C
:1018F00000000000070000000C00000010000000C5
:1019000013000000180000001C0000002C0113014F
:10191000FA00E100C800AF0096007D0064004B00B3
:101920003200190000000000CDCC4C3DCDCCCC3DA8
:101930009A99193ECDCC4C3E0000803E9A99993E32
:101940003333B33ECDCCCC3E6666E63EFBFFFFFFB5
:10195000F7FFFFFFF6FFFFFFFBFFFFFFF7FFFFFFB4
:10196000F6FFFFFFFBFFFFFFF7FFFFFFF6FFFFFFA5
:10197000FDFFFFFFFCFFFFFFF8FFFFFFFDFFFFFF85
:10198000FCFFFFFFF8FFFFFFFDFFFFFFFCFFFFFF76
:10199000F8FFFFFFFBFFFFFFF7FFFFFFF6FFFFFF73
:1019A000FBFFFFFFF7FFFFFFF6FFFFFFFBFFFFFF60
:1019B000FAFFFFFFF8FFFFFFFCFFFFFFF9FFFFFF4C
:1019C000F8FFFFFFFDFFFFFFFCFFFFFFF8FFFFFF3A
:1019D000FCFFFFFFFAFFFFFFF7FFFFFFFBFFFFFF2B
:1019E000F7FFFFFFF4FFFFFFFBFFFFFFF7FFFFFF26
:1019F000F4FFFFFFFBFFFFFFF7FFFFFFF4FFFFFF19
:101A0000FDFFFFFFF8FFFFFFF4FFFFFFFDFFFFFFFC
:101A1000F8FFFFFFF4FFFFFFFDFFFFFFF8FFFFFFF1
:101A2000F4FFFFFFFBFFFFFFF7FFFFFFF4FFFFFFE8
:101A3000FBFFFFFFF7FFFFFFF4FFFFFFFBFFFFFFD1
:101A4000F8FFFFFFF4FFFFFFFCFFFFFFF9FFFFFFC1
:101A5000F4FFFFFFFDFFFFFFF8FFFFFFF4FFFFFFB5
:101A6000FCFFFFFFF7FFFFFFF4FFFFFF000078051B
:101A7000220B0410B4143219B01DFC214826FE2993
:101A8000822D383126344637663A223DFF3FFFFF2C
:101A90000000D007100E88133219AA1E28237427BD
:101AA0005C2B442F643284354038663A8C3C803E4F
:101AB000FF3FFFFF0000540BEC13FA1908201C2510
:101AC0003629EC2C0C302C33E8357238663AF63B6C
:101AD000863D163FFF3FFFFF0000CC10581BFC2146
:101AE000AC26C62A7C2E3831F4334C36A438983ACA
:101AF0005A3C543D803E7A3FFF3FFFFF000000000C
:101B0000070000000C00000010000000130000009F
:101B1000180000001A000000070000000C00000080
:101B20001000000013000000180000001A00000060
:101B30001F000000FBFFFFFFF7FFFFFFF4FFFFFFA9
:101B4000FBFFFFFFF7FFFFFFF4FFFFFFFDFFFFFFBE
:101B5000F7FFFFFFF4FFFFFFFDFFFFFFF8FFFFFFB1
:101B6000F4FFFFFFFAFFFFFFF7FFFFFFF4FFFFFFA8
:101B7000FBFFFFFFF7FFFFFFF4FFFFFFFBFFFFFF90
:101B8000F7FFFFFFF4FFFFFFFBFFFFFFF7FFFFFF84
:101B9000F4FFFFFFFDFFFFFFF8FFFFFFF4FFFFFF74
:101BA000FDFFFFFFF8FFFFFFF4FFFFFFFDFFFFFF5B
:101BB000F8FFFFFFF4FFFFFFFAFFFFFFF8FFFFFF53
:101BC000F4FFFFFF581C0100289CFF1F0000FF0FBF
:101BD000E49DFF1F0000FF0FB5550000181C010019
:101BE0002C9CFF1F7805D007AA9DFF1F7805D00702
:101BF00039550000241C0100DC9DFF1F32005E01EE
:101C0000000000000000000055550000544852003C
